:020000020000FC
:0C0000000C941D050C94B1490C94BA49F5
:10000C000C9400000C9400000C9400000C94000064
:10001C000C9400000C9400000C9400000C94000054
:10002C000C9400000C9494950C9400000C9400001B
:10003C000C9400000C94C7390C9400000C94000034
:10004C000C9400000C9400000C94A3D20C94D1D20C
:10005C000C9400000C9400000C949A3A0C94000040
:10006C000C9400000C9400000C9400000C94000004
:10007C000C9400000C9400000C9400000C940000F4
:10008C000C9400000C94000000000000010203041A
:10009C0000060705E2BD4FB20FA68099938CE07F56
:1000AC008973C367B85C7A522049AA401039503220
:1000BC00512C08276622521EC51AA717EC148D1254
:1000CC007C10A90E0F0DAB0B1202010EFFFF13FFDC
:1000DC00FFFFFF11161003FF0D0B0006FFFF0C00B6
:1000EC00060209010D0B0711031405120E18160C4C
:1000FC0017130408100F0A0017120B11090D05082D
:10010C00130714010C190410030215060A0E0F0034
:10011C0000000101010100000000000101010100CB
:10012C000101000000000100FFFF00FFFFFF01FFC5
:10013C00FFFFFF02030405FFFF06FFFFFFFFFF00A9
:10014C00436F4465496E466F00C802100100000FF2
:10015C00AA558A617567203331203230323620310E
:10016C00303A33353A3531000067010165640000DF
:10017C000001010102020203030304040405050546
:10018C0006060607070741424341424341424341A9
:10019C0042434142434142434142434142430000B6
:1001AC000000EF006A029008000000000000000050
:1001BC000000000000000000000000000000000033
:1001CC00000000000000000000000000640023019B
:1001DC00C602D504820F00000000000000000000E1
:1001EC000000000000000000000000000000000003
:1001FC0000000000000000000000F000F0005402BD
:10020C00D203F6090000000000000000000000000E
:10021C0000000000000000000000000000000000D2
:10022C0000000000000000002A03C8032105E306BB
:10023C004D10000000000000000000000000000055
:10024C0000000000000000000000000000000000A2
:10025C000000000000000101FE0102FD0104FB0191
:10026C0008F701807F0140BF0120DF0110EF008003
:10027C007F0040BF0020DF0010EF0001FE0002FDF8
:10028C000004FB0008F70B0A090C0D100E0F1B1ACB
:10029C00191C1D001E1F02060B0C0D0E1100000078
:1002AC004C01000043414E72783A20253033580AF5
:1002BC00000043414E696E707574436E743D257534
:1002CC002121210A0043414E2D25753A20300A0088
:1002DC0043414E2D25753A20310A0043414E2D25C0
:1002EC00753A2025750A0043414E2025750044655A
:1002FC006C61792074696D6572202575000046610A
:10030C0063746F727944656661756C740A00485049
:10031C0038343432004572724C6F67506F733D2520
:10032C00752C204E6F3D25750A004572723A2025BA
:10033C00752025750A002575204F66660A002575FF
:10034C00204F6E0A00466C6173682074696D65728B
:10035C002025750048503834343200436667537595
:10036C006D3D253034580A00205570646174656405
:10037C000A00485038343432207665722E202575A8
:10038C002E25752E2575206175672033312032306E
:10039C0032362031303A33353A35310A00536572F2
:1003AC0069616C3A2025750A00596561723A2032F0
:1003BC0030253032752C205765656B3A2025750A2F
:1003CC00004857207665723A2025632C204F7074B4
:1003DC00696F6E733A20253032580A00436C6F6394
:1003EC006B3A202530386C580A0043666743686BBB
:1003FC0053756D3A202530345820004F4B0A00209D
:10040C00457272210A004366675665724572723AEC
:10041C002025752028257529210A0045455076652B
:10042C00724572723A2025752028257529210A00FB
:10043C00526573746F7265436E743D257520257516
:10044C002025750A00446174614572723D25303275
:10045C005820253032580A004850383434320A00BB
:10046C004144436D696E4572726F725B25755D3DDB
:10047C0025752121210A0000496E707574733A00AC
:10048C002025753D257500496E2D313A2025750ABC
:10049C0000496E2D323A2025750A00496E2D333AEB
:1004AC002025750A00496E2D343A2025750A00491D
:1004BC006E2D25753A2025750A00496E412D25753E
:1004CC00204F66663A2025755B6D565D0A00496EB5
:1004DC00412D2575204F6E3A2025755B6D565D0AB2
:1004EC000053776974636820257500416E616C6FE9
:1004FC006720332E257500416E616C6F6720342E9A
:10050C00257500004B65795061643D00426C696E45
:10051C006B3A2530325820253032580A0047726128
:10052C007968696C6C2043414E6F70656E0A0047A8
:10053C0072617968696C6C204A313333390A00482E
:10054C0050393634320A004E6F6E650A00004B6526
:10055C00795061642E436F6E6E2025750A004B65D1
:10056C00795061642E4469736F6E6E6E2025750A26
:10057C0000004F75745075736850756C6C3A20257B
:10058C00750A004F757448696768536964654F6EE6
:10059C006C793A2025750A0043202532753A2025BE
:1005AC0034750043616C69627261746520004F4B55
:1005BC000A006F7574707574202575206661696CFE
:1005CC0065642121210A002532753A2025352E3209
:1005DC00665B415D0A002532753A204E6F206665D8
:1005EC0065646261636B2C204F75742D25750A0050
:1005FC002532753A20466565646261636B206572CD
:10060C00726F722C204F75742D25750A004F7574FE
:10061C007075742074657374004261747420636126
:10062C006C696220203A20257500416E616C6F6701
:10063C002063616C69623A20333D25752C20343D72
:10064C0025750043616C6962726174696F6E4D61EE
:10065C00736B3A2025580A0020202532753A253430
:10066C00752C2536752C2536752C2536752C25368E
:10067C00750042617474657279206661696C656499
:10068C002121210A00416E616C6F67206661696CE3
:10069C0065642121210A00206E6F7420636F6D70D8
:1006AC006C657465642121210A004F757452737452
:1006BC004572725B25755D0A004F75742D25753A70
:1006CC00204F6E0A004F75742D25753A20532575F1
:1006DC002D3E25752C204F6E3D25752C20536574B1
:1006EC003D25750A004144433A002025753D25758A
:1006FC00002020426174743D2575004C6F77426177
:10070C0074744F66663D2025750A004C6F77426104
:10071C0074744F6E3D20257530300A00426174743C
:10072C00657279536B697046423A20252E31665BAF
:10073C00565D0A00426174746572794642204F4BD3
:10074C003A20252E31665B565D0A002020416E61F1
:10075C002D333D202575002020416E612D343D2028
:10076C002575004F75742D25753A2025750A004F97
:10077C00757420257520474E442D31210A004F7584
:10078C007420257520474E442D32210A004F757474
:10079C00202575206C696D6974210A004F757441B0
:1007AC002D25753A205325752D3E25752C204F6E21
:1007BC003D25752C205365743D25750A004F7574C5
:1007CC0020257520474E44210A004F75742025754D
:1007DC00204C696D6974210A004F75742D25753A8A
:1007EC00205325752D3E2575205365743D25750ABE
:1007FC00004F7574707574733A0A002534753A207D
:10080C0046423D2575204144433D25752025755BA9
:10081C006D415D0A002534753A2046423D25750A26
:10082C000052657365744572726F720A004F75746D
:10083C00707574202575004F75742D25753A2053ED
:10084C0025752C204F6E3D25752025632C20257594
:10085C00305B6D415D0A00004F75747075742067D4
:10086C00726F757020257500506F776572446F77C5
:10087C006E0A0057616B6555703A2025750A0000A9
:10088C004F7574412D25753A205325752D3E2575D0
:10089C002C204F6E3D25750A000043616C69622E59
:1008AC002073746172742025755B416D705D0A0054
:1008BC0054657374206F75740A0043616C69622E01
:1008CC0020626174740A0043616C696220616E611C
:1008DC0028352C3056207265662E290A0043616C2F
:1008EC0069623F006330006331006333006336009C
:1008FC0063323000636200636100746573746F75FA
:10090C00740050615373576F5264210050573A2052
:10091C0027257327200050573A204E6F6E65200014
:10092C00204D6F64653D25750A004144433F0049E5
:10093C006E7075743F004C6F61643F004850737467
:10094C00617475733F0052526573746F7265005217
:10095C0052204F4B0A005265736574005365744FF7
:10096C0075742025753D2025750A005265736574D4
:10097C00206572726F720A004F7074696F6E3A2044
:10098C00253032580A0052657365740A00504320B2
:10099C004F4B0A005043204F6C64210A00005365F2
:1009AC00712025633A20004F66660A0025630A0011
:1009BC0053657175656E63652025750020204F4B5E
:1009CC000A0020204661696C65642121210A00001F
:1009DC0056696E2D25753A2025750A005669727474
:1009EC0075616C202575000057697065723A20534B
:1009FC0025752D3E5325750A000001002D4E414EE4
:100A0C0000494E4600002D4E414E000001000200F0
:100A1C00AA0200000700BC031A0300000700C3036E
:100A2C006003000001008F0E060A00000000F8941D
:100A3C00EE27EFBBF1E0F5BFE5BFE0937400E09368
:100A4C0075008DE0A2E0BB27ED938A95E9F780EF66
:100A5C009FE0A0E0B1E0ED930197E9F7E8E1FAE05F
:100A6C00D0E0DBBF87919791009781F0A791B79168
:100A7C0007901790C791D791BF01DBB7F001CBBF9F
:100A8C0007900D920197E1F7FB01EBCFE0E0EEBB95
:100A9C00EFEEEDBFE0E1EEBFCCEBD3E00C9484378E
:100AAC000E9461E4AD014093D2035093D303A5E2BD
:100ABC00B1E00E9430E6E07111F0E1E001C0E0E04D
:100ACC00AFECB3E0E170EE0F0E2EEC91ED7FE02970
:100ADC00EC93A7ECB2E00E9430E6E093D103A8ECD3
:100AEC00B2E00E9430E6E0935C04A091D103A13007
:100AFC0010F0AD3008F004C0E091CF03E46003C007
:100B0C00E091CF03EB7FE093CF03E1E0E093D800DB
:100B1C00FA01E436A0E0FA0741F4E2E1E093E200E6
:100B2C00ECE0E093E300E7E335C0ED37A0E0FA0733
:100B3C0041F4EEE0E093E200ECE0E093E300E7E365
:100B4C0029C0E83CA0E0FA0741F4E8E0E093E200B9
:100B5C00ECE0E093E300E7E31DC0EA3FA0E0FA0716
:100B6C0041F4E6E0E093E200ECE0E093E300E7E33D
:100B7C0011C0E43FA1E0FA0711F4E6E005C0E83E3D
:100B8C00A3E0FA0749F4E2E0E093E200E4E0E0934A
:100B9C00E300E3E1E093E40010E1103F88F41093EC
:100BAC00ED002EEE30E0E8EFF0E02E173F0730F4CA
:100BBC00D901E0E0EC932F5F3F4FF5CF105FEDCF05
:100BCC00E091D800E260E093D80010E4103FA0F46C
:100BDC001093ED002EEE30E0E8EFF0E02E173F071B
:100BEC0030F4D901E0E0EC932F5F3F4FF5CFE8E80C
:100BFC00E093EF00105FEACF0E9468E42696089518
:100C0C0064970E9461E4E091D003E03009F414C2CF
:100C1C00E17089F0E0E0E093ED00E091EE00E17529
:100C2C0051F0E091D003EE7FE093D003E0E0E0934D
:100C3C00EE00E093EF00E091D003E27089F0E0E188
:100C4C00E093ED00E091EE00E17551F0E091D003FE
:100C5C00ED7FE093D003E0E0E093EE00E093EF0053
:100C6C00E091D003E47089F0E0E2E093ED00E091D4
:100C7C00EE00E17551F0E091D003EB7FE093D003EF
:100C8C00E0E0E093EE00E093EF00E091D003E87039
:100C9C0089F0E0E3E093ED00E091EE00E17551F0B6
:100CAC00E091D003E77FE093D003E0E0E093EE0027
:100CBC00E093EF00A091D003AF3009F4BDC1A09137
:100CCC005604E0915704EA1709F4B6C1A4EDB3E059
:100CDC00E0915604F0E0BD01ADE0B0E00E9416E5F5
:100CEC00DB01AE0FBF1FEC91E071B1F041E0A4ED60
:100CFC00B3E0E0915604F0E0BD01ADE0B0E00E943D
:100D0C0016E5DB01AE0FBF1F11960E94D3E5EB8BEE
:100D1C00FC8B6D8B7E8B13C040E0A4EDB3E0E091B7
:100D2C005604F0E0BD01ADE0B0E00E9416E5DB0139
:100D3C00AE0FBF1F1196ED91FD91EF8BF88FA4EDC7
:100D4C00B3E0E0915604F0E0BD01ADE0B0E00E94EC
:100D5C0016E5DB01AE0FBF1FEC91EF700E2F098F64
:100D6C00403019F0E98DE061E98FE091D003E1703A
:100D7C0009F051C0E0E0E093ED00E98DE093EF0065
:100D8C004030D1F0EB89EE0FEE0FEE0FE093F00058
:100D9C00AB89BC89E5E00E949CE4E093F100AB894F
:100DAC00BC898D899E89EDE00E94C4E4E093F20039
:100DBC00E5E10E94C4E40AC0EF89E295E07FEE0F02
:100DCC00E093F200EF89F88D0E94EFE4E093F300DA
:100DDC0010E01017B0F4A4EDB3E0E0915604F0E08D
:100DEC00BD01ADE0B0E00E9416E5DB01AE0FBF1F08
:100DFC001596EE27A10FBE1FEC91E093FA001F5F32
:100E0C00E8CFE98DE05CE093EF00E091D003E16086
:100E1C00E093D00303C1E091D003E27009F051C01C
:100E2C00E0E1E093ED00E98DE093EF004030D1F08C
:100E3C00EB89EE0FEE0FEE0FE093F000AB89BC895F
:100E4C00E5E00E949CE4E093F100AB89BC898D89BC
:100E5C009E89EDE00E94C4E4E093F200E5E10E947B
:100E6C00C4E40AC0EF89E295E07FEE0FE093F20054
:100E7C00EF89F88D0E94EFE4E093F30010E0101777
:100E8C00B0F4A4EDB3E0E0915604F0E0BD01ADE0A8
:100E9C00B0E00E9416E5DB01AE0FBF1F1596EE27E2
:100EAC00A10FBE1FEC91E093FA001F5FE8CFE98D14
:100EBC00E05CE093EF00E091D003E260E093D003BC
:100ECC00ADC0E091D003E47009F051C0E0E2E093D2
:100EDC00ED00E98DE093EF004030D1F0EB89EE0F9F
:100EEC00EE0FEE0FE093F000AB89BC89E5E00E94B9
:100EFC009CE4E093F100AB89BC898D899E89EDE07F
:100F0C000E94C4E4E093F200E5E10E94C4E40AC04C
:100F1C00EF89E295E07FEE0FE093F200EF89F88D18
:100F2C000E94EFE4E093F30010E01017B0F4A4ED8E
:100F3C00B3E0E0915604F0E0BD01ADE0B0E00E94FA
:100F4C0016E5DB01AE0FBF1F1596EE27A10FBE1FD6
:100F5C00EC91E093FA001F5FE8CFE98DE05CE09341
:100F6C00EF00E091D003E460E093D00357C0E09130
:100F7C00D003E87009F051C0E0E3E093ED00E98D97
:100F8C00E093EF004030D1F0EB89EE0FEE0FEE0F57
:100F9C00E093F000AB89BC89E5E00E949CE4E0930F
:100FAC00F100AB89BC898D899E89EDE00E94C4E477
:100FBC00E093F200E5E10E94C4E40AC0EF89E295F7
:100FCC00E07FEE0FE093F200EF89F88D0E94EFE4E2
:100FDC00E093F30010E01017B0F4A4EDB3E0E0914F
:100FEC005604F0E0BD01ADE0B0E00E9416E5DB0177
:100FFC00AE0FBF1F1596EE27A10FBE1FEC91E0930D
:10100C00FA001F5FE8CFE98DE05CE093EF00E09120
:10101C00D003E860E093D00301C00EC0E091560409
:10102C00EF5FE0935604E150A0915604AA3018F0FB
:10103C00E0E0E093560443CEE0E05E2F2E2F30E448
:10104C00303F08F032C13093ED00E091EE00E072D9
:10105C0009F41EC1E091EF00EF700E2EEE81E07FDF
:10106C00E029EE83EF70E93020F0EE81E07FE8605C
:10107C00EE83E091EF00E07109F46DC0E091F300B4
:10108C00FF2766277727EB8BFC8B6D8B7E8BAB89D1
:10109C00BC898D899E89E8E00E94ADE4EB8BFC8BCA
:1010AC006D8B7E8BE091F200AB89BC898D899E891A
:1010BC00FF2766277727EA2BFB2B682B792BEB8BEB
:1010CC00FC8B6D8B7E8BAB89BC898D899E89E8E00E
:1010DC000E94ADE4EB8BFC8B6D8B7E8BE091F10071
:1010EC00AB89BC898D899E89FF2766277727EA2BD8
:1010FC00FB2B682B792BEB8BFC8B6D8B7E8BAB8955
:10110C00BC898D899E89E5E00E94ADE4EB8BFC8B5C
:10111C006D8B7E8BE091F000F0E00E94E6E4AB89F1
:10112C00BC898D899E896F2F660F660B762FEA2BF3
:10113C00FB2B682B792BEB8BFC8B6D8B7E8BEE81D9
:10114C00E061EE83EB89FC896D897E89EF83F887FA
:10115C0069877A871DC0E091F300F0E0EF8BF88F80
:10116C000E94DDE4EF8BF88FE091F200F0E0F59552
:10117C00E7950E94E4E4AF89B88DEA2BFB2BEF8B4B
:10118C00F88FEE81EF7EEE83EF89F88DEF83F88791
:10119C0010E0EE81EF701E1758F4E12FF0E0DE0145
:1011AC001B96AE0FBF1FE091FA00EC931F5FF1CFBF
:1011BC002F5FE091CF03E17081F0E0EBF2E060E0B3
:1011CC0070E00E94EEE5EB8DFC8D662777270E9480
:1011DC00EEE584E00E94E8E32896A091D103A030CC
:1011EC0069F0AF89B88D109749F4EE81EF70E23059
:1011FC0028F0E091D103AC85EA1709F017C0EB8514
:10120C00F0E0E130A0E0FA0721F4E091CF03EB7FAE
:10121C000BC0E230A0E0FA0721F0E038A0E0FA07BA
:10122C0029F4E091CF03E460E093CF03E091CF0386
:10123C00E47069F5DE0116960E943E1EE0915C0A90
:10124C00E27021F0DE0116960E94BC98E091BB077B
:10125C00F0E0E130A0E0FA0729F4DE0116960E94D6
:10126C00634B15C0E230A0E0FA0721F0E330A0E0B8
:10127C00FA0729F4DE0116960E94245B08C0E430BC
:10128C00A0E0FA0721F4DE0116960E94136305C054
:10129C00E091EE00EE7039F05F5FE0E0E093EE007D
:1012AC00E0E8E093EF00305FCBCE222319F4552316
:1012BC0009F45AC02130E0F0E091CE03E03041F463
:1012CC00E0911B09E062E0931B09E0E0E093160952
:1012DC00EEE1E093CE03E091CF03E27049F0A2E39C
:1012EC00B1E00E942CE6FF70E093540EF093550E83
:1012FC00A0915804B0915904A13FEFEFBE0740F400
:10130C00A0915A04B0915B04A13FEFEFBE0760F1CE
:10131C00E0915804F0915904F695E795E093580440
:10132C00F0935904E0915A04F0915B04F695E7951B
:10133C00E0935A04F0935B04A0915804B0915904C3
:10134C00E22FF0E0EA0FFB1FE0935804F0935904EE
:10135C00A0915A04B0915B04E52FF0E0EA0FFB1F5B
:10136C00E0935A04F0935B040E9468E46A96089533
:10137C00BA93AA9324970E9461E4E091CF03E4709E
:10138C0009F07FC1E0916304E07821F0AA85BB8568
:10139C000E943E1EAA85BB85EC91EF700E2F202F6C
:1013AC00EC91E07151F031E0206111960E94D3E58F
:1013BC00EE83FF836887798706C030E0AA85BB85FA
:1013CC0011964D915C91E091D003E17009F047C00A
:1013DC00E0E0E093ED002093EF003030D1F0EE81AF
:1013EC00EE0FEE0FEE0FE093F000AE81BF81E5E063
:1013FC000E949CE4E093F100AE81BF8188859985C1
:10140C00EDE00E94C4E4E093F200E5E10E94C4E444
:10141C000CC0E0E0E093F000E42FE295E07FEE0FEB
:10142C00E093F200FA010E94EFE4E093F30010E085
:10143C00101758F4AA85BB851596EE27A10FBE1F71
:10144C00EC91E093FA001F5FF3CFE22FE05CE093A6
:10145C00EF00E091D003E160E093D00312C1E09182
:10146C00D003E27009F047C0E0E1E093ED00209377
:10147C00EF003030D1F0EE81EE0FEE0FEE0FE09377
:10148C00F000AE81BF81E5E00E949CE4E093F100A6
:10149C00AE81BF8188859985EDE00E94C4E4E0931C
:1014AC00F200E5E10E94C4E40CC0E0E0E093F0003F
:1014BC00E42FE295E07FEE0FE093F200FA010E9438
:1014CC00EFE4E093F30010E0101758F4AA85BB8505
:1014DC001596EE27A10FBE1FEC91E093FA001F5F4B
:1014EC00F3CFE22FE05CE093EF00E091D003E260F9
:1014FC00E093D003C6C0E091D003E47009F047C07C
:10150C00E0E2E093ED002093EF003030D1F0EE817B
:10151C00EE0FEE0FEE0FE093F000AE81BF81E5E031
:10152C000E949CE4E093F100AE81BF81888599858F
:10153C00EDE00E94C4E4E093F200E5E10E94C4E413
:10154C000CC0E0E0E093F000E42FE295E07FEE0FBA
:10155C00E093F200FA010E94EFE4E093F30010E054
:10156C00101758F4AA85BB851596EE27A10FBE1F40
:10157C00EC91E093FA001F5FF3CFE22FE05CE09375
:10158C00EF00E091D003E460E093D0037AC0E091E7
:10159C00D003E87009F047C0E0E3E093ED0020933E
:1015AC00EF003030D1F0EE81EE0FEE0FEE0FE09346
:1015BC00F000AE81BF81E5E00E949CE4E093F10075
:1015CC00AE81BF8188859985EDE00E94C4E4E093EB
:1015DC00F200E5E10E94C4E40CC0E0E0E093F0000E
:1015EC00E42FE295E07FEE0FE093F200FA010E9407
:1015FC00EFE4E093F30010E0101758F4AA85BB85D4
:10160C001596EE27A10FBE1FEC91E093FA001F5F19
:10161C00F3CFE22FE05CE093EF00E091D003E860C1
:10162C00E093D0032EC0E0915704EF5F1E2F1A30C9
:10163C0008F010E0E0915604E11759F4EF5FE093E5
:10164C005604E150A0915604AA3018F0E0E0E09363
:10165C005604A4EDB3E0E0915704F0E0BD01ADE019
:10166C00B0E00E9416E5E60FF71FFA93EA93EC85BB
:10167C00FD85FA93EA93ADE0B0E00E944EDD109345
:10168C0057040E9468E42C9608951A930A938D01CE
:10169C001396ED91FD91A091D203B091D303EA176B
:1016AC00FB0721F0F801A381B481FAD9E0911B0961
:1016BC00E17051F4E0911B09E160E0931B09E1E05A
:1016CC00E09316090E94003DF801E581EF70E930C6
:1016DC0018F4D80115964CDE099119910895A09132
:1016EC00CE03A13078F0E091CE03E150E093CE032D
:1016FC00E03041F4E0911B09EF7DE0931B09E0E041
:10170C00E093160908951A93A4EAB5E00E9430E616
:10171C00E0936F0E11E1163048F0A9EAB5E0EE2720
:10172C00A10FBE1F0E9430E6E03009F002C011503C
:10173C00F2CFE12FE550E093700EE0E0E093710EF4
:10174C00ABEBB5E00E9430E6E093720EA0EFB5E093
:10175C000E9430E6E093730EA5E2B6E00E9430E6FC
:10176C00E093740EAAE6B6E00E9430E6E093750EA4
:10177C00A091750EA13019F4E2E0E093750EE091A2
:10178C00750EE093760EABE6B6E00E9428E6E09389
:10179C00780EF093790E60937A0E70937B0EEFEFC8
:1017AC00E093770EAFE6B6E00E942CE6E0937C0E59
:1017BC00F0937D0E309719F4E0E0E093760EABE3F6
:1017CC00B1E00E9428E630976040704011F4E0E0F0
:1017DC000BC0AFE3B1E00E9430E6E0937E0EA09127
:1017EC007E0EA63018F0E5E0E0937E0E10E013308C
:1017FC00B0F5A0E8BEE0E12FF0E0EE0FFF1FEA0F1E
:10180C00FB1F3196FF93EF93A2E7B6E0E12FF0E0D8
:10181C00BD01A5E1B0E00E9416E5DB01AE0FBF1FD4
:10182C0014960E9430E6AF91BF91EC93A0E8BEE015
:10183C00E12FF0E0EE0FFF1FAE0FBF1FEC91E07831
:10184C00E560EC93A0E8BEE0E12FF0E0EE0FFF1FA7
:10185C00AE0FBF1FEC91EF77EC931F5FC8CF1991C0
:10186C00089563970E9461E4E0916304E07421F4AD
:10187C000E9468E469960895A091760EA13010F448
:10188C000C94B816E091760EE150E093760EEF5F73
:10189C00E091760EE03011F00C94B816E091750ED4
:1018AC00E093760EE091770EEF5FE093770EE150C8
:1018BC00A091770EAF3018F0E0E0E093770EEC8556
:1018CC00E07FE860EC87FE017196FA93EA93E0E022
:1018DC00EA93A8E0B0E00E9460DDE091770EF0E0C2
:1018EC00309709F057C1E0917C0EF0917D0EE170BC
:1018FC0009F44CC120E0E0919707E17009F02160F8
:10190C00E0919907E17009F02260E0919B07E1708A
:10191C0009F02460E0919D07E17009F02860E091E6
:10192C009F07E17009F02061E091A107E17009F0D7
:10193C002062E091A307E17009F02064E091A50713
:10194C00E17009F02068298B20E0E091A707E17095
:10195C0009F02160E091A907E17009F02260E091A3
:10196C00AB07E17009F02460E091AD07E17009F07C
:10197C002860FE017296208320E0E091A60DE074B1
:10198C0009F02160E091AE0DE07409F02260E09165
:10199C00B60DE07409F02460E091BE0DE07409F01E
:1019AC002860E091C60DE07409F02061E091CE0D45
:1019BC00E07409F02062E091D60DE07409F0206427
:1019CC00E091DE0DE07409F02068FE01739620832F
:1019DC0020E0E091E60DE07409F02160E091EE0D5D
:1019EC00E07409F02260E091F60DE07409F02460D7
:1019FC00E091FE0DE07409F02860E091060EE074B1
:101A0C0009F02061E0910E0EE07409F02062E09183
:101A1C00160EE07409F02064E0911E0EE07409F0DB
:101A2C002068FE017496208320E0E0917704E07832
:101A3C0009F02160E0918504E07809F02260E091E2
:101A4C009304E07809F02460E091A104E07809F0B7
:101A5C002860E091AF04E07809F02061E091BD04CA
:101A6C00E07809F02062E091CB04E07809F0206482
:101A7C00E091D904E07809F02068FE017596208386
:101A8C0020E0E091E704E07809F02160E091F504B2
:101A9C00E07809F02260E0910305E07809F0246019
:101AAC00E0911105E07809F02860E0911F05E078DD
:101ABC0009F02061E0912D05E07809F02062E091B9
:101ACC003B05E07809F02064E0914905E07809F0E5
:101ADC002068FE017696208320E0E0915705E0789F
:101AEC0009F02160E0916505E07809F02260E09151
:101AFC007305E07809F02460E0918105E07809F045
:101B0C002860E0918F05E07809F02061E0919D0557
:101B1C00E07809F02062E0919D05E07809F02064FE
:101B2C00E091B905E07809F02068FE0177962083F2
:101B3C0020E0E091C705E07809F02160E091D5053F
:101B4C00E07809F02260E091E305E07809F0246088
:101B5C00E091F105E07809F02860E091FF05E0786C
:101B6C0009F02061E0910D06E07809F02062E09127
:101B7C001B06E07809F02064E0912906E07809F072
:101B8C002068FE01789620830C947E16E1E0E093A9
:101B9C00770E05C0E130A0E0FA0709F0DDC0E09156
:101BAC007C0EF0917D0EE27009F4D2C0E091310907
:101BBC00E077E03321F4E0913109E47009F403C0DB
:101BCC00E6E6E98B0DC0E0913109E295E770FF275D
:101BDC0066277727EC58FE4F6F4F6BBF0690098A2C
:101BEC00E0913B09E077E03321F4E0913B09E470AC
:101BFC0009F403C0E6E6EA8B0DC0E0913B09E295DF
:101C0C00E770FF2766277727EC58FE4F6F4F6BBFA7
:101C1C0006900A8AE0914509E077E03321F4E091DF
:101C2C004509E47009F403C0E6E6EB8B0DC0E091C6
:101C3C004509E295E770FF2766277727EC58FE4F9A
:101C4C006F4F6BBF06900B8AE0914F09E077E03342
:101C5C0021F4E0914F09E47009F403C0E6E6EC8B43
:101C6C000DC0E0914F09E295E770FF2766277727B3
:101C7C00EC58FE4F6F4F6BBF06900C8AE0915909E0
:101C8C00E077E03321F4E0915909E47009F403C0E2
:101C9C00E6E6ED8B0DC0E0915909E295E770FF2760
:101CAC0066277727EC58FE4F6F4F6BBF06900D8A57
:101CBC00E0916309E077E03321F4E0916309E4708B
:101CCC0009F403C0E6E6EE8B0DC0E0916309E295E2
:101CDC00E770FF2766277727EC58FE4F6F4F6BBFD7
:101CEC0006900E8AE0916D09E077E03321F4E091E3
:101CFC006D09E47009F403C0E6E6EF8B0DC0E091CA
:101D0C006D09E295E770FF2766277727EC58FE4FA1
:101D1C006F4F6BBF06900F8AE0917709E077E03345
:101D2C0021F4E0917709E47009F403C0E6E6E88F4A
:101D3C000DC0E0917709E295E770FF2766277727BA
:101D4C00EC58FE4F6F4F6BBF0690088E0C947E16AE
:101D5C00E2E0E093770E05C0E230A0E0FA0709F06C
:101D6C00DCC0E0917C0EF0917D0EE47009F4D1C0E2
:101D7C00E0918109E077E03321F4E0918109E4708E
:101D8C0009F403C0E6E6E98B0DC0E0918109E29508
:101D9C00E770FF2766277727EC58FE4F6F4F6BBF16
:101DAC000690098AE0918B09E077E03321F4E09109
:101DBC008B09E47009F403C0E6E6EA8B0DC0E091F0
:101DCC008B09E295E770FF2766277727EC58FE4FC3
:101DDC006F4F6BBF06900A8AE0919509E077E0336C
:101DEC0021F4E0919509E47009F403C0E6E6EB8B6D
:101DFC000DC0E0919509E295E770FF2766277727DC
:101E0C00EC58FE4F6F4F6BBF06900B8AE0919F0909
:101E1C00E077E03321F4E0919F09E47009F403C00A
:101E2C00E6E6EC8B0DC0E0919F09E295E770FF2789
:101E3C0066277727EC58FE4F6F4F6BBF06900C8AC6
:101E4C00E091A909E077E03321F4E091A909E4706D
:101E5C0009F403C0E6E6ED8B0DC0E091A909E2950B
:101E6C00E770FF2766277727EC58FE4F6F4F6BBF45
:101E7C0006900D8AE091B309E077E03321F4E0910C
:101E8C00B309E47009F403C0E6E6EE8B0DC0E091F3
:101E9C00B309E295E770FF2766277727EC58FE4FCA
:101EAC006F4F6BBF06900E8AE091BD09E077E0336F
:101EBC0021F4E091BD09E47009F403C0E6E6EF8B70
:101ECC000DC0E091BD09E295E770FF2766277727E3
:101EDC00EC58FE4F6F4F6BBF06900F8AE091C7090D
:101EEC00E077E03321F4E091C709E47009F403C012
:101EFC00E6E6E88F0DC0E091C709E295E770FF2791
:101F0C0066277727EC58FE4F6F4F6BBF0690088EF5
:101F1C00EFC6E3E0E093770E05C0E330A0E0FA07EC
:101F2C0009F08EC0E0917C0EF0917D0EE87009F402
:101F3C0083C0E091D109E077E03321F4E091D1093D
:101F4C00E47009F403C0E6E6E98B0DC0E091D10919
:101F5C00E295E770FF2766277727EC58FE4F6F4F07
:101F6C006BBF0690098AE091DB09E077E03321F43E
:101F7C00E091DB09E47009F403C0E6E6EA8B0DC0DE
:101F8C00E091DB09E295E770FF2766277727EC588D
:101F9C00FE4F6F4F6BBF06900A8AE091170AE295CD
:101FAC00E770FF2766277727EC58FE4F6F4F6BBF04
:101FBC0006900B8AE0911B0AE295E770FF276627D3
:101FCC007727EC58FE4F6F4F6BBF06900C8AE09151
:101FDC001F0AE295E770FF2766277727EC58FE4F1C
:101FEC006F4F6BBF06900D8AE091230AE295E77064
:101FFC00FF2766277727EC58FE4F6F4F6BBF069075
:10200C000E8AE091270AE295E770FF27662777276B
:10201C00EC58FE4F6F4F6BBF06900F8AE0912B0A66
:10202C00E295E770FF2766277727EC58FE4F6F4F36
:10203C006BBF0690088E5CC6E4E0E093770E05C09B
:10204C00E430A0E0FA0709F074C0E0917C0EF09146
:10205C007D0EE07109F469C0E0912F0AE295E770FA
:10206C00FF2766277727EC58FE4F6F4F6BBF069004
:10207C00098AE091330AE295E770FF2766277727F4
:10208C00EC58FE4F6F4F6BBF06900A8AE091370AEF
:10209C00E295E770FF2766277727EC58FE4F6F4FC6
:1020AC006BBF06900B8AE0913B0AE295E770FF2725
:1020BC0066277727EC58FE4F6F4F6BBF06900C8A44
:1020CC00E0913F0AE295E770FF2766277727EC58E7
:1020DC00FE4F6F4F6BBF06900D8AE091430AE2955D
:1020EC00E770FF2766277727EC58FE4F6F4F6BBFC3
:1020FC0006900E8AE091470AE295E770FF27662763
:10210C007727EC58FE4F6F4F6BBF06900F8AE0910C
:10211C004B0AE295E770FF2766277727EC58FE4FAE
:10212C006F4F6BBF0690088EE3C5E5E0E093770E2A
:10213C0005C0E530A0E0FA0709F0C8C0E0917C0EBC
:10214C00F0917D0EE07209F4BDC0E0913809F09178
:10215C003909EA87FB87AA85BB85AC3EE3E1BE075C
:10216C0030F4E4E1F0E00E945CE52E2F01C02FEF8B
:10217C00298BA0913E09A63319F4E0E0EA8B16C036
:10218C00E0914209F0914309EA87FB87AA85BB8558
:10219C00AC3EE3E1BE0730F4E4E1F0E00E945CE524
:1021AC002E2F01C02FEFFE0172962083E0914C0977
:1021BC00F0914D09EA87FB87AA85BB85AC3EE3E12C
:1021CC00BE0730F4E4E1F0E00E945CE52E2F01C084
:1021DC002FEFFE0173962083A0915209A63319F4B8
:1021EC00E0E0EC8B16C0E0915609F0915709EA87B4
:1021FC00FB87AA85BB85AC3EE3E1BE0730F4E4E186
:10220C00F0E00E945CE52E2F01C02FEFFE017496CA
:10221C002083E0916009F0916109EA87FB87AA8528
:10222C00BB85AC3EE3E1BE0730F4E4E1F0E00E9494
:10223C005CE52E2F01C02FEFFE0175962083E091F7
:10224C006A09F0916B09EA87FB87AA85BB85AC3ECE
:10225C00E3E1BE0730F4E4E1F0E00E945CE52E2FF0
:10226C0001C02FEFFE0176962083E0917409F09166
:10227C007509EA87FB87AA85BB85AC3EE3E1BE07FF
:10228C0030F4E4E1F0E00E945CE52E2F01C02FEF6A
:10229C00FE0177962083E0917E09F0917F09EA8711
:1022AC00FB87AA85BB85AC3EE3E1BE0730F4E4E1D5
:1022BC00F0E00E945CE52E2F01C02FEFFE01789616
:1022CC00208316C5E6E0E093770E05C0E630A0E06B
:1022DC00FA0709F0BAC0E0917C0EF0917D0EE07423
:1022EC0009F4AFC0E0918809F0918909EA87FB876E
:1022FC00AA85BB85AC3EE3E1BE0730F4E4E1F0E037
:10230C000E945CE52E2F01C02FEF298BE0919209E2
:10231C00F0919309EA87FB87AA85BB85AC3EE3E184
:10232C00BE0730F4E4E1F0E00E945CE52E2F01C022
:10233C002FEFFE0172962083E0919C09F0919D098C
:10234C00EA87FB87AA85BB85AC3EE3E1BE0730F488
:10235C00E4E1F0E00E945CE52E2F01C02FEFFE01BE
:10236C0073962083E091A609F091A709EA87FB8771
:10237C00AA85BB85AC3EE3E1BE0730F4E4E1F0E0B6
:10238C000E945CE52E2F01C02FEFFE017496208376
:10239C00E091B009F091B109EA87FB87AA85BB856A
:1023AC00AC3EE3E1BE0730F4E4E1F0E00E945CE512
:1023BC002E2F01C02FEFFE0175962083E091BA09F4
:1023CC00F091BB09EA87FB87AA85BB85AC3EE3E1AC
:1023DC00BE0730F4E4E1F0E00E945CE52E2F01C072
:1023EC002FEFFE0176962083E091C409F091C50988
:1023FC00EA87FB87AA85BB85AC3EE3E1BE0730F4D8
:10240C00E4E1F0E00E945CE52E2F01C02FEFFE010D
:10241C0077962083E091CE09F091CF09EA87FB876C
:10242C00AA85BB85AC3EE3E1BE0730F4E4E1F0E005
:10243C000E945CE52E2F01C02FEFFE0178962083C1
:10244C0057C4E7E0E093770E05C0E730A0E0FA0749
:10245C0009F088C0E0917C0EF0917D0EE07809F4D3
:10246C007DC0A091D409A63319F4E0E0E98B14C027
:10247C00E091D809F091D909EA87FB87AA85BB8539
:10248C00AC3EE3E1BE0730F4E4E1F0E00E945CE531
:10249C002E2F01C02FEF298BA091DE09A63319F442
:1024AC00E0E0EA8B16C0E091E209F091E309EA87DB
:1024BC00FB87AA85BB85AC3EE3E1BE0730F4E4E1C3
:1024CC00F0E00E945CE52E2F01C02FEFFE0172960A
:1024DC002083E091170AE295E7704E2F423011F0FD
:1024EC00433011F4EFE001C0E0E0EB8BE0911B0A0C
:1024FC00E295E7704E2F423011F0433011F4EFE0CB
:10250C00EC8BE0911F0AE295E7704E2F423011F0F0
:10251C00433011F4EFE0ED8BE091230AE295E77084
:10252C004E2F423011F0433011F4EFE0EE8BE0917E
:10253C00270AE295E7704E2F423011F0433011F428
:10254C00EFE0EF8BE0912B0AE295E7704E2F4230D3
:10255C0011F0433011F4EFE0E88FCAC3E8E0E093E8
:10256C00770E05C0E830A0E0FA0709F064C0E091EE
:10257C007C0EF0917D0EF17009F459C0E0912F0A98
:10258C00E295E7704E2F423011F0433011F4EFE03A
:10259C00E98BE091330AE295E7704E2F423011F04F
:1025AC00433011F4EFE0EA8BE091370AE295E770E3
:1025BC004E2F423011F0433011F4EFE0EB8BE091F1
:1025CC003B0AE295E7704E2F423011F0433011F484
:1025DC00EFE0EC8BE0913F0AE295E7704E2F423032
:1025EC0011F0433011F4EFE0ED8BE091430AE295EA
:1025FC00E7704E2F423011F0433011F4EFE0EE8BC8
:10260C00E091470AE295E7704E2F423011F04330CB
:10261C0011F4EFE0EF8BE0914B0AE295E7704E2F4F
:10262C00423011F0433011F4EFE0E88F61C3E9E080
:10263C00E093770E05C0E930A0E0FA0709F085C0F9
:10264C00E0917C0EF0917D0EF27009F47AC0A091AD
:10265C006C0EE5E0EA9FF001EA87FB87EB85E98BDE
:10266C00EA85EA8BE091690EEB8BE091680EEC8BBE
:10267C00E091E509E077E03321F4E091E509E470BD
:10268C0009F403C0E6E6ED8B0DC0E091E509E29597
:10269C00E770FF2766277727EC58FE4F6F4F6BBF0D
:1026AC0006900D8AE091EF09E077E03321F4E09198
:1026BC00EF09E47009F403C0E6E6EE8B0DC0E0917F
:1026CC00EF09E295E770FF2766277727EC58FE4F56
:1026DC006F4F6BBF06900E8AE091F909E077E033FB
:1026EC0021F4E091F909E47009F403C0E6E6EF8BFC
:1026FC000DC0E091F909E295E770FF27662777276F
:10270C00EC58FE4F6F4F6BBF06900F8AE091030A97
:10271C00E077E03321F4E091030AE47009F403C09C
:10272C00E6E6E88F0DC0E091030AE295E770FF271B
:10273C0066277727EC58FE4F6F4F6BBF0690088EBD
:10274C00D7C2EAE0E093770E05C0EA30A0E0FA07C2
:10275C0009F0B5C0E0917C0EF0917D0EF47009F497
:10276C00AAC0A091E809A63319F4E0E0E98B14C0E3
:10277C00E091EC09F091ED09EA87FB87AA85BB850E
:10278C00AC3EE3E1BE0730F4E4E1F0E00E945CE52E
:10279C002E2F01C02FEF298BA091F209A63319F42B
:1027AC00E0E0EA8B16C0E091F609F091F709EA87B0
:1027BC00FB87AA85BB85AC3EE3E1BE0730F4E4E1C0
:1027CC00F0E00E945CE52E2F01C02FEFFE01729607
:1027DC002083E091000AF091010AEA87FB87AA8521
:1027EC00BB85AC3EE3E1BE0730F4E4E1F0E00E94CF
:1027FC005CE52E2F01C02FEFFE0173962083E09134
:10280C000A0AF0910B0AEA87FB87AA85BB85AC3EC6
:10281C00E3E1BE0730F4E4E1F0E00E945CE52E2F2A
:10282C0001C02FEFFE0174962083A0912A09B0916C
:10283C002B09E4E1F0E00E945CE5EA87FB87EB857D
:10284C00ED8BEA85EE8BE0910D0AE077E03321F415
:10285C00E0910D0AE47009F403C0E6E6EF8B0DC0BD
:10286C00E0910D0AE295E770FF2766277727EC5871
:10287C00FE4F6F4F6BBF06900F8AA091100AA633C4
:10288C0019F4E0E0E88F16C0E091140AF091150AF3
:10289C00EA87FB87AA85BB85AC3EE3E1BE0730F433
:1028AC00E4E1F0E00E945CE52E2F01C02FEFFE0169
:1028BC00789620831DC2EBE0E093770E05C0EB30D9
:1028CC00A0E0FA0709F06EC0E0917C0EF0917D0E4D
:1028DC00F87009F463C020E0E091260EE07409F072
:1028EC002160E0912E0EE07409F02260E091360E2A
:1028FC00E07409F02460E0913E0EE07409F0286069
:10290C00298BE0914F0AE295E770FF27662777271E
:10291C00EC58FE4F6F4F6BBF06900A8AE091530A3A
:10292C00E295E770FF2766277727EC58FE4F6F4F2D
:10293C006BBF06900B8AE0914F0AE295E7704E2F21
:10294C00423011F0433011F4EFE001C0E0E0EC8BC9
:10295C00E091530AE295E7704E2F423011F043306C
:10296C0011F4EFE001C0E0E0ED8BE091620AE17060
:10297C0021F0E091630AE695EE8BE0916A0AE17032
:10298C0021F0E0916B0AE695EF8BE091720AE17011
:10299C0021F0E091730AE695E88FAAC1ECE0E09390
:1029AC00770E04C0EC30A0E0FA07C9F5E0917C0E7C
:1029BC00F0917D0EF07179F1E2E0E98BE0E1EA8BC8
:1029CC00A6E1B0E00E9430E6EB8BA5E1B0E00E94FE
:1029DC0030E6EC8BE0917A0AE17021F0E0917B0A11
:1029EC00E695ED8BE091820AE17021F0E091830A8B
:1029FC00E695EE8BE0918A0AE17021F0E0918B0A6A
:102A0C00E695EF8BE091920AE17021F0E091930A48
:102A1C00E695E88F6DC1EDE0E093770E05C0ED30E3
:102A2C00A0E0FA0709F09FC0E0917C0EF0917D0EBA
:102A3C00F07209F494C0E0917F0EEF5FE0937F0E8B
:102A4C00E150E98B20E0E0916B0EE07209F021601F
:102A5C00E0916B0EE07409F02260E0912509E170C1
:102A6C0009F02460E0912509E27009F02860E091FA
:102A7C002509E07209F02061E0912409E07809F061
:102A8C002062A5E3B1E00E9430E6A0915D0EAE1786
:102A9C0008F02064A091CE03A13008F02068FE015C
:102AAC0072962083E091550EEB8BE091540EEC8BDB
:102ABC00E0E01E2F2E2F51E0183060F4A3E01A9F97
:102ACC00F001ED5BF84FE081E27009F0252B1F5F00
:102ADC00550FF2CFFE017596208320E018E051E0EF
:102AEC00103160F4A3E01A9FF001ED5BF84FE08128
:102AFC00E27009F0252B1F5F550FF2CFFE01769681
:102B0C00208320E010E151E0143160F4A3E01A9F1F
:102B1C00F001ED5BF84FE081E27009F0252B1F5FAF
:102B2C00550FF2CFFE0177962083E0E01E2F2E2F5B
:102B3C0051E0153080F4E12FAFE7B7E0F0E00E94F0
:102B4C00DFE4AE0FBF1F1396EC91E17009F0252B5B
:102B5C001F5F550FEECFFE0178962083C9C0EEE0C3
:102B6C00E093770E05C0EE30A0E0FA0709F0C0C084
:102B7C00E0917C0EF0917D0EF07409F4B4C0E091FC
:102B8C009108F09192080E94F1E4EA87FB87EB85AB
:102B9C00E98BEA85EA8BE0919308F09194080E9406
:102BAC00F1E4EA87FB87EB85EB8BEA85EC8B20E085
:102BBC00E0912509E47009F02160E0912509E870A5
:102BCC0009F02260E0912509E07109F02460E091A0
:102BDC002509E07209F02860FE0175962083E091CA
:102BEC00BB07F0E0E130A0E0FA0711F5E091BC077B
:102BFC00E078E9F0E091C507EE8BA091C607E09173
:102C0C00DE07E295E07FEA2BEF8BE091DE07F0E048
:102C1C000E94E4E4309749F4E091DF07F0E00E9471
:102C2C00DBE4309711F4E0E001C0E1E0E88F5AC03A
:102C3C00E230A0E0FA0721F0E330A0E0FA07A1F5BA
:102C4C00E091BE07E03079F1E0E01E2F3E2F0E2F11
:102C5C0035E021E0E091BD071E17E0F4A2EEB7E0ED
:102C6C00E12FF0E00E94DFE4AE0FBF1F1296EC9153
:102C7C00E17009F0022B220F203051F4E32F3F5F5B
:102C8C00F0E0DE015196EA0FFB1F008300E021E02B
:102C9C001F5FE0CF203039F0E32FF0E0DE015196DA
:102CAC00EA0FFB1F00831EC0E430A0E0FA07D1F44A
:102CBC00A091C007A130B0F0E091C307EE8B30912A
:102CCC00EB07A091C607E32FE295E07FEA2BEF8B91
:102CDC00E32FE295EF70AE2FE091EE07E295E07FE7
:102CEC00EA2BE88F05C0E0E0E093770E0C94730CB0
:102CFC00A091780EB091790E80917A0E90917B0E06
:102D0C00E091770EF0E06F2F660F660B762FEA0FCF
:102D1C00FB1F681F791FEE83FF8368877987AE815D
:102D2C00BF8188859985A030E8E0BE07E0E08E077A
:102D3C00E0E09E0740F4EC85EF7EEC87EE81FF81AE
:102D4C00ED87FE870BC0EC85E061EC87EE81FF819F
:102D5C0068857985ED87FE876F87788BDE011C96F9
:102D6C000E94BE090E9468E46996089564970E94C7
:102D7C0061E4E0916304E07409F44AC4EF81E07FFC
:102D8C00E860EF83A0917E0EA13008F450C0E09172
:102D9C007E0EE150E0937E0EEF5FE0917E0EE03010
:102DAC0009F045C0AFE3B1E00E9430E6E0937E0E3F
:102DBC00ABE3B1E00E9428E6EC8BFD8B6E8B7F8B36
:102DCC00AC89BD898E899F89A030E8E0BE07E0E020
:102DDC008E07E0E09E0740F4EF81EF7EEF83EC89F5
:102DEC00FD89E887F9870BC0EF81E061EF83EC89FF
:102DFC00FD896E897F89E887F9876A877B87A9E3D4
:102E0C00B1E00E9430E6EC87AAE3B1E00E9430E624
:102E1C00ED87E2E0EE87E0E1EF87E1E0E88BE0E0D0
:102E2C00E98BEA8BEB8BDE0117960E94BE09A09111
:102E3C006F0EA13008F421C1E0916F0EE150E093C8
:102E4C006F0EE03009F019C1FE013C96FA93EA933B
:102E5C00E0E0EA93A8E0B0E00E9460DDA4EAB5E00F
:102E6C000E9430E6E0936F0EA5EAB5E00E9428E6DA
:102E7C00EC8BFD8B6E8B7F8BAC89BD898E899F898A
:102E8C00A030E8E0BE07E0E08E07E0E09E0740F4EB
:102E9C00EF81EF7EEF83EC89FD89E887F9870BC022
:102EAC00EF81E061EF83EC89FD896E897F89E8878A
:102EBC00F9876A877B87A091700EA13090F1E09121
:102ECC00710EEF5FE093710EE150A091710EE091E5
:102EDC00700EEA1718F4E1E0E093710EE091710EB8
:102EEC00EC87A9EAB5E0F0E03496AE0FBF1F0E9464
:102EFC0030E64E2F4F3010F0463208F012C0E42F5F
:102F0C00F0E03F97AAE0B0E00E9416E5E85CF64FCF
:102F1C00DF01ED91FD91DF01E4E1F0E00E945CE561
:102F2C00EB8BAEEAB5E00E9430E64E2F4F3010F03E
:102F3C00463208F012C0E42FF0E03F97AAE0B0E070
:102F4C000E9416E5E85CF64FDF01ED91FD91DF0183
:102F5C00E4E1F0E00E945CE5EA8BADEAB5E00E94AA
:102F6C0030E64E2F4F3010F0463208F012C0E42FEE
:102F7C00F0E03F97AAE0B0E00E9416E5E85CF64F5F
:102F8C00DF01ED91FD91DF01E4E1F0E00E945CE5F1
:102F9C00E98BACEAB5E00E9430E64E2F4F3010F0D2
:102FAC00463208F012C0E42FF0E03F97AAE0B0E000
:102FBC000E9416E5E85CF64FDF01ED91FD91DF0113
:102FCC00E4E1F0E00E945CE5E88BABEAB5E00E943E
:102FDC0030E64E2F4F3010F0463208F012C0E42F7E
:102FEC00F0E03F97AAE0B0E00E9416E5E85CF64FEF
:102FFC00DF01ED91FD91DF01E4E1F0E00E945CE581
:10300C00EF87AAEAB5E00E9430E64E2F4F3010F061
:10301C00463208F012C0E42FF0E03F97AAE0B0E08F
:10302C000E9416E5E85CF64FDF01ED91FD91DF01A2
:10303C00E4E1F0E00E945CE5EE87A9EAB5E00E94CD
:10304C0030E64E2F4F3010F0463208F012C0E42F0D
:10305C00F0E03F97AAE0B0E00E9416E5E85CF64F7E
:10306C00DF01ED91FD91DF01E4E1F0E00E945CE510
:10307C00ED87DE0117960E94BE09A091720EA13059
:10308C0008F47CC0E091720EE150E093720EEF5F99
:10309C00E091720EE03009F071C0FE013C96FA939B
:1030AC00EA93E0E0EA93A8E0B0E00E9460DDABEBCD
:1030BC00B5E00E9430E6E093720EACEBB5E00E94F6
:1030CC0028E6EC8BFD8B6E8B7F8BAC89BD898E8952
:1030DC009F89A030E8E0BE07E0E08E07E0E09E07A5
:1030EC0040F4EF81EF7EEF83EC89FD89E887F98767
:1030FC000BC0EF81E061EF83EC89FD896E897F89DC
:10310C00E887F9876A877B87E0E00E2F1E2F2E2F2A
:10311C0051E0103300F5A0ECB5E0EE27A10FBE1F77
:10312C000E9430E64E2F403031F0A42F0E94EE3E2C
:10313C00E03009F0052B503859F4E22F2F5FF0E006
:10314C00DE011C96EA0FFB1F008351E000E001C07A
:10315C00550F1F5FDECFA0912A09B0912B09AC3916
:10316C00E3E6BE0728F4E4E6F0E00E945CE501C06B
:10317C00EFEFEA8BDE0117960E94BE09A091730E49
:10318C00A13008F4B9C0E091730EE150E093730ED6
:10319C00EF5FE091730EE03009F0AEC0A0EFB5E048
:1031AC000E9430E6E093730EA1EFB5E00E9428E692
:1031BC00EC8BFD8B6E8B7F8BAC89BD898E899F8947
:1031CC00A030E8E0BE07E0E08E07E0E09E0740F4A8
:1031DC00EF81EF7EEF83EC89FD89E887F9870BC0DF
:1031EC00EF81E061EF83EC89FD896E897F89E88747
:1031FC00F9876A877B87E0E00E2F1E2F2E2F51E078
:10320C00103308F06CC0A5EFB5E0EE27A10FBE1F80
:10321C000E9430E64E2F403009F451C04F3010F070
:10322C00463308F03AC0463210F5E42FF0E03F97F1
:10323C00AAE0B0E00E9416E5EF5CF64FE081E29563
:10324C00E770EE83E42FF0E03F97AAE0B0E00E9435
:10325C0016E5EF5CF64FE081E47039F4AE81A130F5
:10326C0021F0A43011F0A53009F4052B15C0E42F82
:10327C00F0E0B697A7E1BAE00E94DFE4AE0FBF1F03
:10328C00EC91E295E770EE83AE81A13021F0A43091
:10329C0011F0A53009F4052B12C0473310F04C3354
:1032AC0008F007C0A42F0E941C90E03009F0052BF9
:1032BC0006C0A42F0E94EE3EE03009F0052B5038DA
:1032CC0059F4E22F2F5FF0E0DE011C96EA0FFB1F92
:1032DC00008351E000E001C0550F1F5F91CFE091DA
:1032EC006C0EF0E03196F595E795EA8BE0E0EB8B10
:1032FC00DE0117960E94BE09A091740EA13008F44D
:10330C00BEC0E091740EE150E093740EEF5FE0915B
:10331C00740EE03009F0B3C0FE013C96FA93EA93C8
:10332C00E0E0EA93A8E0B0E00E9460DDA5E2B6E040
:10333C000E9430E6E093740EA6E2B6E00E9428E606
:10334C00EC8BFD8B6E8B7F8BAC89BD898E899F89B5
:10335C00A030E8E0BE07E0E08E07E0E09E0740F416
:10336C00EF81EF7EEF83EC89FD89E887F9870BC04D
:10337C00EF81E061EF83EC89FD896E897F89E887B5
:10338C00F9876A877B87E0E00E2F1E2F2E2F51E0E6
:10339C00103408F070C0AAE2B6E0EE27A10FBE1FF1
:1033AC000E9430E64E2F403009F455C0103220F008
:1033BC004F3010F0463308F03AC0463210F5E42F87
:1033CC00F0E03F97AAE0B0E00E9416E5EF5CF64F04
:1033DC00E081E295E770EE83E42FF0E03F97AAE0FE
:1033EC00B0E00E9416E5EF5CF64FE081E47039F432
:1033FC00AE81A13021F0A43011F0A53009F4052BD9
:10340C0015C0E42FF0E0B697A7E1BAE00E94DFE424
:10341C00AE0FBF1FEC91E295E770EE83AE81A13049
:10342C0021F0A43011F0A53009F4052B14C0103292
:10343C0020F0473310F04C3308F007C0A42F0E9443
:10344C001C90E03009F0052B06C0A42F0E94EE3E24
:10345C00E03009F0052B503859F4E22F2F5FF0E0E3
:10346C00DE011C96EA0FFB1F008351E000E001C057
:10347C00550F1F5F8DCFDE0117960E94BE0910E01D
:10348C00133008F0C5C0A0E8BEE0E12FF0E0EE0F6D
:10349C00FF1FAE0FBF1F11964C91403009F4B6C000
:1034AC00A0E8BEE0E12FF0E0EE0FFF1FAE0FBF1F54
:1034BC00EC91EF773E2FA42F0E94EE3E0E2FA0E84A
:1034CC00BEE0E12FF0E0EE0FFF1FAE0FBF1FEC913F
:1034DC00EE1FE0E0EE1FE1700E1799F031E0A0E86E
:1034EC00BEE0E12FF0E0EE0FFF1FAE0FBF1FE02F8D
:1034FC00E170E795E0E0E7950E2EEC91EF77E0298F
:10350C00EC93313008F473C03150303009F06FC097
:10351C00A1E7B6E00E9430E63E2FA2E7B6E0E12F2D
:10352C00F0E0BD01A5E1B0E00E9416E5DB01AE0FB5
:10353C00BF1F0E9428E6EC8BFD8B6E8B7F8BAC89BA
:10354C00BD898E899F89A030E8E0BE07E0E08E0738
:10355C00E0E09E0740F4EF81EF7EEF83EC89FD897C
:10356C00E887F9870BC0EF81E061EF83EC89FD8977
:10357C006E897F89E887F9876A877B87EF81E07F8F
:10358C00E860EF83A0E8BEE0E12FF0E0EE0FFF1F54
:10359C00AE0FBF1FEC91E07869F0A2E7B6E0E12F27
:1035AC00F0E0BD01A5E1B0E00E9416E5E60FF71FC3
:1035BC0035960CC0A2E7B6E0E12FF0E0BD01A5E125
:1035CC00B0E00E9416E5E60FF71F3D96E88FF98FE5
:1035DC00FE013C96FA93EA93EA8DFB8DFA93EA93FB
:1035EC00A8E00E94662ADE0117960E94BE09A0E898
:1035FC00BEE0E12FF0E0EE0FFF1FAE0FBF1FE32F79
:10360C00EF770E2EEC91E078E029EC931F5F38CF2A
:10361C000E9468E46A9608951A93A4EAB5E0E0E083
:10362C000E944CE6A5EAB5E0E0E0F0E060E070E076
:10363C000E943CE610E0123148F4A9EAB5E0EE270E
:10364C00A10FBE1F0E944CE61F5FF5CFE1E7F6E02D
:10365C00FA93EA93AAE60E949B2AE0E0F8E4FA9334
:10366C00EA93A0E5B0E00E943B2EABEBB5E0E0E0C6
:10367C000E944CE6ACEBB5E0E0E0F0E060E070E01E
:10368C000E943CE610E0103348F4A0ECB5E0EE27C5
:10369C00A10FBE1F0E944CE61F5FF5CFA0EFB5E057
:1036AC00E0E00E944CE6A1EFB5E0E0E0F0E060E085
:1036BC0070E00E943CE610E0103348F4A5EFB5E052
:1036CC00EE27A10FBE1F0E944CE61F5FF5CFA5E2AF
:1036DC00B6E0E0E00E944CE6A6E2B6E0E0E0F0E006
:1036EC0060E070E00E943CE610E0103448F4AAE27E
:1036FC00B6E0EE27A10FBE1F0E944CE61F5FF5CF70
:10370C00AAE6B6E0E0E00E944CE6ABE6B6E0E0E00C
:10371C00F0E060E070E00E943CE6AFE6B6E0EFEF70
:10372C00FFEF0E9444E6A2C21A93ADEBB2E00E94F6
:10373C002CE6DF010E945605A6ECB2E00E9430E6B2
:10374C00E170ABE1B9E0E1700E2EEC91EE7FE02977
:10375C00EC93E0E0E0931609EDE5F4E0FA93EA93DC
:10376C00E0E0EA93A6EEB2E00E9460DDA1ECB2E0EC
:10377C000E9430E6E0935E04A0915E04A53018F43C
:10378C00E5E0E0935E04A6ECB2E00E9430E6E6953C
:10379C00E170A3E6B4E0E170E795E0E0E7950E2E6A
:1037AC00EC91EF77E029EC93A2ECB2E00E9428E6D2
:1037BC00E0935F04F093600460936104709362047F
:1037CC00E0E0E0936A0410E0143308F01DC2ACECA6
:1037DC00B2E0E12FF0E0BD01AEE0B0E00E9416E5F2
:1037EC00DB01AE0FBF1F1A960E9430E6E07809F499
:1037FC0009C2ABE6B4E0E12FF0E0BD01AEE0B0E011
:10380C000E9416E5DB01AE0FBF1F1A96EC91E06823
:10381C00EC93ABE6B4E0E12FF0E0BD01AEE0B0E03C
:10382C000E9416E5E60FF71FFF93EF93ACECB2E0A6
:10383C00E12FF0E0BD01AEE0B0E00E9416E5DB0147
:10384C00AE0FBF1F0E9428E6AF91BF91ED93FD9381
:10385C006D937C93ABE6B4E0E12FF0E0BD01AEE0FC
:10386C00B0E00E9416E5E60FF71F3496FF93EF9336
:10387C00ACECB2E0E12FF0E0BD01AEE0B0E00E94B4
:10388C0016E5DB01AE0FBF1F14960E942CE6AF911C
:10389C00BF91ED93FC93ABE6B4E0E12FF0E0BD01FA
:1038AC00AEE0B0E00E9416E5E60FF71F3696FF93E8
:1038BC00EF93ACECB2E0E12FF0E0BD01AEE0B0E094
:1038CC000E9416E5DB01AE0FBF1F16960E942CE678
:1038DC00AF91BF91ED93FC93ABE6B4E0E12FF0E038
:1038EC00BD01AEE0B0E00E9416E5E60FF71F38967A
:1038FC00FF93EF93ACECB2E0E12FF0E0BD01AEE052
:10390C00B0E00E9416E5DB01AE0FBF1F18960E94B7
:10391C002CE6AF91BF91ED93FC93ABE6B4E0E12FB5
:10392C00F0E0BD01AEE0B0E00E9416E5E60FF71F37
:10393C003A96FF93EF93ACECB2E0E12FF0E0BD01CF
:10394C00AEE0B0E00E9416E5DB01AE0FBF1F1A9689
:10395C000E9430E6EF70AF91BF91EF700E2EEC919C
:10396C00E07FE029EC93ABE6B4E0E12FF0E0BD01A1
:10397C00AEE0B0E00E9416E5E60FF71F3A96FF9313
:10398C00EF93ACECB2E0E12FF0E0BD01AEE0B0E0C3
:10399C000E9416E5DB01AE0FBF1F1A960E9430E69F
:1039AC00E295E770AF91BF91E770E295E07F0E2E44
:1039BC00EC91EF78E029EC93ABE6B4E0E12FF0E08A
:1039CC00BD01AEE0B0E00E9416E5E60FF71F3B9696
:1039DC00FF93EF93ACECB2E0E12FF0E0BD01AEE071
:1039EC00B0E00E9416E5DB01AE0FBF1F1B960E94D4
:1039FC0030E6EF70AF91BF91EF700E2EEC91E07F3F
:103A0C00E029EC93ABE6B4E0E12FF0E0BD01AEE0D1
:103A1C00B0E00E9416E5E60FF71F3B96FF93EF937D
:103A2C00ACECB2E0E12FF0E0BD01AEE0B0E00E9402
:103A3C0016E5DB01AE0FBF1F1B960E9430E6E29528
:103A4C00EF70AF91BF91EF70E295E07F0E2EEC918D
:103A5C00EF70E029EC93ABE6B4E0E12FF0E0BD01B0
:103A6C00AEE0B0E00E9416E5E60FF71F3C96FF9320
:103A7C00EF93ACECB2E0E12FF0E0BD01AEE0B0E0D2
:103A8C000E9416E5DB01AE0FBF1F1C960E9430E6AC
:103A9C00E170AF91BF91E1700E2EEC91EE7FE029B9
:103AAC00EC93ABE6B4E0E12FF0E0BD01AEE0B0E0AA
:103ABC000E9416E5E60FF71F3C96FF93EF93ACECD4
:103ACC00B2E0E12FF0E0BD01AEE0B0E00E9416E5FF
:103ADC00DB01AE0FBF1F1C960E9430E6E695E1702D
:103AEC00AF91BF91E170EE0F0E2EEC91ED7FE029BE
:103AFC00EC93ABE6B4E0E12FF0E0BD01AEE0B0E05A
:103B0C000E9416E5E60FF71F3C96FF93EF93ACEC83
:103B1C00B2E0E12FF0E0BD01AEE0B0E00E9416E5AE
:103B2C00DB01AE0FBF1F1C960E9430E6E695E695B2
:103B3C00E370AF91BF91E370EE0FEE0F0E2EEC9190
:103B4C00E37FE029EC93ABE6B4E0E12FF0E0BD01BC
:103B5C00AEE0B0E00E9416E5E60FF71F3C96FF932F
:103B6C00EF93ACECB2E0E12FF0E0BD01AEE0B0E0E1
:103B7C000E9416E5DB01AE0FBF1F1C960E9430E6BB
:103B8C00E295E170AF91BF91E170E295E07F0E2E6E
:103B9C00EC91EF7EE029EC93ABE6B4E0E12FF0E0A2
:103BAC00BD01AEE0B0E00E9416E5DB01AE0FBF1F19
:103BBC001C96EC91EC70E43089F0ABE6B4E0E12FAC
:103BCC00F0E0BD01AEE0B0E00E9416E5DB01AE0F07
:103BDC00BF1F1C96EC91EC70EC3081F4ABE6B4E0BA
:103BEC00E12FF0E0BD01AEE0B0E00E9416E5DB0194
:103BFC00AE0FBF1F1C96EC91E068EC93E12FEF5FCA
:103C0C00E0936A041F5FE0CDE4E6F4E0FA93EA93F4
:103C1C00E0E4F1E0FA93EA93A5E00E94662AE091D1
:103C2C006504F091660460916704709168043097A4
:103C3C006040704021F4E0916404EF7E15C0E09187
:103C4C006404E061E0936404F0E0F695E795E370BA
:103C5C00F070E330A0E0FA0721F0E130A0E0FA07C1
:103C6C0029F4E0916404E860E093640419910895E8
:103C7C00BA93AA936D970E9461E4E0E0EE8BABA13E
:103C8C00BCA1EC91E295E1703E2F3030C1F0119661
:103C9C00ED91FD916D917D91ED8FFE8F6F8F78A3DE
:103CAC00E0915F04F0916004609161047091620492
:103CBC00AD8DBE8D8F8D98A10E940EE50CC0ABA171
:103CCC00BCA111964D915C91A0915F04B0916004E0
:103CDC00FA010E94FCE4E88FE030A9F1ABA1BCA191
:103CEC00EC91EF70E13048F0EBA1FCA1A581A17043
:103CFC0021F00E94482C0E945E8CABA1BCA1EC91DF
:103D0C00EF70E63000F120E0E1E0EA8FE98F273236
:103D1C00D0F4ABA1BCA11596EA8DF0E0AE0FBF1F9D
:103D2C00EC91A98DEA2319F0A22F0E943E77E98D20
:103D3C00EE0FE98FE03029F4EA8DEF5FEA8FE1E0D6
:103D4C00E98F2F5FE4CFE0916404E07109F43FC088
:103D5C00303079F0E0916504F0916604609167046D
:103D6C0070916804AD8DBE8D8F8D98A10E940EE56B
:103D7C0007C0A0916504B0916604FA010E94FCE4AE
:103D8C00E88FE03021F1EBA1FCA1A581A17071F0CD
:103D9C00E0916404E17021F0E0916404E77F03C0DA
:103DAC00E0916404E860E09364040DC0E091640465
:103DBC00E17021F0E0916404E86003C0E0916404D8
:103DCC00E77FE0936404E0915E04E0936904E09182
:103DDC006304EF70E23011F4E1E0EE8BA0916A0421
:103DEC00A433A0F0EEEBF2E060E070E00E94EEE5B0
:103DFC00E0916A04FF27662777270E94EEE584E0AE
:103E0C000E94E8E32896E4E3E0936A0420E0E09162
:103E1C006A042E1708F04FC5ABE6B4E0E22FF0E0D1
:103E2C00BD01AEE0B0E00E9416E5E60FF71F8F0172
:103E3C00E285E07809F43DC5303061F0D801ED91B0
:103E4C00FD916D917D91AD8DBE8D8F8D98A10E9450
:103E5C000EE507C0D801ED91FD91DF01FA010E943A
:103E6C00FCE4E88FE03009F424C5E0916304E074CD
:103E7C0009F40DC5F801E485E07171F1ACECB2E028
:103E8C00E22FF0E0BD01AEE0B0E00E9416E5DB01F0
:103E9C00AE0FBF1F1C960E9430E6E295EF70E695C0
:103EAC00E770ABA1BCA11596F0E0AE0FBF1FEC9173
:103EBC00EF93ACECB2E0E22FF0E0BD01AEE0B0E08D
:103ECC000E9416E5DB01AE0FBF1F1D960E9430E667
:103EDC00AF91EA1709F0DBC4ABE6B4E0E22FF0E0F7
:103EEC00BD01AEE0B0E00E9416E5DB01AE0FBF1FD6
:103EFC001D96E0915E04EC93E0E0E9A3EAA3F801DF
:103F0C00E385EF70E13038F1ABA1BCA11596F80157
:103F1C00E385F0E0EF70F0703197AE0FBF1FEC91BE
:103F2C00F0E0E9A3FAA3F9A1E0E0E9A3FAA3ABA1BD
:103F3C00BCA11596F801E385F0E00E94EDE4EF706A
:103F4C00F0703197AE0FBF1FEC91A9A1BAA1F0E0B0
:103F5C00EA2BFB2B0FC0ABA1BCA11596F801E38596
:103F6C00F0E00E94EDE4EF70F0703197AE0FBF1FE0
:103F7C00EC91F0E0E9A3FAA3D8011896ED91FD912C
:103F8C00A9A1BAA1EA23FB23E9A3FAA3F801E485CA
:103F9C00E17059F0F801A085B185FD01F695E79522
:103FAC00A9A1BAA1EA17FB0708F00CC0D801189612
:103FBC00ED91FD91E095F095A9A1BAA1EA2BFB2B0F
:103FCC00E9A3FAA3F801E485E295EF70E695E6958E
:103FDC00E170EF8BF801E485E17009F456C2E9A1B8
:103FEC00FAA1EB8FFC8FF801E285F0E0EF70F07036
:103FFC00E630A0E0FA0709F4C7C13097C9F4AB8DDD
:10400C00BC8D00240A160B0624F4EB8DFC8DF29665
:10401C0006C0AC8DAA232AF4EB8DFC8DF297EB8FA6
:10402C00FC8FAB8DBC8DE4E6F0E00E946FE5AAC17D
:10403C00E130A0E0FA07C9F4AB8DBC8D00240A1660
:10404C000B0624F4EB8DFC8D799606C0AC8DAA235F
:10405C002AF4EB8DFC8D7997EB8FFC8FAB8DBC8D9F
:10406C00E2E3F0E00E946FE58DC1E230A0E0FA07D8
:10407C00C9F4AB8DBC8D00240A160B0624F4EB8D11
:10408C00FC8D3A9606C0AC8DAA232AF4EB8DFC8DE0
:10409C003A97EB8FFC8FAB8DBC8DE4E1F0E00E9486
:1040AC006FE570C1E330A0E0FA07C9F4AB8DBC8DAD
:1040BC0000240A160B0624F4EB8DFC8D359606C0F5
:1040CC00AC8DAA232AF4EB8DFC8D3597EB8FFC8FEE
:1040DC00AB8DBC8DEAE0F0E00E946FE553C1E4309B
:1040EC00A0E0FA07C9F4AB8DBC8D00240A160B06B0
:1040FC0024F4EB8DFC8D339606C0AC8DAA232AF4E8
:10410C00EB8DFC8D3397EB8FFC8FAB8DBC8DE5E08D
:10411C00F0E00E946FE536C1E530A0E0FA07C9F483
:10412C00AB8DBC8D00240A160B0624F4EB8DFC8D94
:10413C00329606C0AC8DAA232AF4EB8DFC8D3297F7
:10414C00EB8FFC8FAB8DBC8DE2E0F0E00E946FE555
:10415C0019C1E730A0E0FA0741F5AB8DBC8D002406
:10416C000A160B0674F4AF3FEFE3BE071CF0EFEF3B
:10417C00FFE704C0EB8DFC8DEE0FFF1FEB8FFC8F68
:10418C0013C0AC8DAA2382F4AB8DBC8DE0E0F0ECB7
:10419C00EA17FB071CF0E0E0F0E804C0EB8DFC8DA7
:1041AC00EE0FFF1FEB8FFC8FEFC0E830A0E0FA079B
:1041BC0061F5AB8DBC8D00240A160B0684F4A9396D
:1041CC00E9E1BE071CF0EFEFFFE706C0EB8DFC8DBD
:1041DC00A5E0B0E00E9444E5EB8FFC8F15C0AC8DE0
:1041EC00AA2392F4AB8DBC8DE7E6F6EEEA17FB073B
:1041FC001CF0E0E0F0E806C0EB8DFC8DA5E0B0E033
:10420C000E9444E5EB8FFC8FBFC0E930A0E0FA07B9
:10421C0061F5AB8DBC8D00240A160B0684F4AC3C06
:10422C00ECE0BE071CF0EFEFFFE706C0EB8DFC8D5A
:10423C00AAE0B0E00E9444E5EB8FFC8F15C0AC8D7A
:10424C00AA2392F4AB8DBC8DE4E3F3EFEA17FB07E2
:10425C001CF0E0E0F0E806C0EB8DFC8DAAE0B0E0CD
:10426C000E9444E5EB8FFC8F8FC0EA30A0E0FA0788
:10427C0061F5AB8DBC8D00240A160B0684F4A636B2
:10428C00E6E0BE071CF0EFEFFFE706C0EB8DFC8D00
:10429C00A4E1B0E00E9444E5EB8FFC8F15C0AC8D1F
:1042AC00AA2392F4AB8DBC8DEAE9F9EFEA17FB0770
:1042BC001CF0E0E0F0E806C0EB8DFC8DA4E1B0E072
:1042CC000E9444E5EB8FFC8F5FC0EB30A0E0FA0757
:1042DC0061F5AB8DBC8D00240A160B0684F4AF3847
:1042EC00E2E0BE071CF0EFEFFFE706C0EB8DFC8DA4
:1042FC00A2E3B0E00E9444E5EB8FFC8F15C0AC8DBF
:10430C00AA2392F4AB8DBC8DE1E7FDEFEA17FB0716
:10431C001CF0E0E0F0E806C0EB8DFC8DA2E3B0E011
:10432C000E9444E5EB8FFC8F2FC0EC30A0E0FA0725
:10433C0059F5AB8DBC8D00240A160B0684F4A734FA
:10434C00E1E0BE071CF0EFEFFFE706C0EB8DFC8D44
:10435C00A4E6B0E00E9444E5EB8FFC8F15C0AC8D59
:10436C00AA2392F4AB8DBC8DE1E7FDEFEA17FB07B6
:10437C001CF0E0E0F0E806C0EB8DFC8DA4E6B0E0AC
:10438C000E9444E5EB8FFC8FF801E285F0E00E947F
:10439C00EDE4E770F070309769F4F801A481B58111
:1043AC00EB8DFC8DEA17FB0711F4E1E001C0E0E0B6
:1043BC00EF8B6AC0E130A0E0FA0769F4F801A48140
:1043CC00B581EB8DFC8DEA17FB0711F4E0E001C021
:1043DC00E1E0EF8B59C0E230A0E0FA07D9F4EF89A5
:1043EC00E03061F0D8011696ED91FD91AB8DBC8D4E
:1043FC00EA17FB0714F0E0E0EF8B0BC0D801149622
:10440C00ED91FD91AB8DBC8DEA17FB0714F4E1E047
:10441C00EF8B3AC0E330A0E0FA07D9F4EF89E03033
:10442C0061F0D8011696ED91FD91AB8DBC8DAE1758
:10443C00BF0714F0E0E0EF8B0BC0D8011496ED91A0
:10444C00FD91AB8DBC8DAE17BF0714F4E1E0EF8B83
:10445C001BC0E430A0E0FA07B9F4D8011496ED9132
:10446C00FD91AB8DBC8DAE17BF074CF0D8011696E5
:10447C00ED91FD91AB8DBC8DEA17FB070CF402C0DE
:10448C00E1E001C0E0E0EF8B75C1F801E285F0E0FE
:10449C00EF70F070E630A0E0FA0709F4CCC030976A
:1044AC0061F4E9A1FAA1F296E9A3FAA3A9A1BAA130
:1044BC00E4E6F0E00E945CE5BCC0E130A0E0FA0765
:1044CC0061F4E9A1FAA17996E9A3FAA3A9A1BAA189
:1044DC00E2E3F0E00E945CE5ACC0E230A0E0FA0759
:1044EC0061F4E9A1FAA13A96E9A3FAA3A9A1BAA1A8
:1044FC00E4E1F0E00E945CE59CC0E330A0E0FA0748
:10450C0061F4E9A1FAA13596E9A3FAA3A9A1BAA18C
:10451C00EAE0F0E00E945CE58CC0E430A0E0FA0731
:10452C0061F4E9A1FAA13396E9A3FAA3A9A1BAA16E
:10453C00E5E0F0E00E945CE57CC0E530A0E0FA0725
:10454C0041F4E9A1FAA13196E9A3FAA3F695E7950E
:10455C0070C0E730A0E0FA0781F4A9A1BAA1AF3F7F
:10456C00EFE7BE0728F4E9A1FAA1EE0FFF1F02C086
:10457C00EFEFFFEFE9A3FAA35EC0E830A0E0FA0783
:10458C0079F4A9A1BAA1A333E3E3BE0720F4E5E0D3
:10459C000E943EE502C0EFEFFFEFE9A3FAA34BC088
:1045AC00E930A0E0FA0779F4A9A1BAA1A939E9E1A7
:1045BC00BE0720F4EAE00E943EE502C0EFEFFFEFF9
:1045CC00E9A3FAA338C0EA30A0E0FA0779F4A9A16C
:1045DC00BAA1AC3CECE0BE0720F4E4E10E943EE55D
:1045EC0002C0EFEFFFEFE9A3FAA325C0EB30A0E088
:1045FC00FA0779F4A9A1BAA1AE31E5E0BE0720F41F
:10460C00E2E30E943EE502C0EFEFFFEFE9A3FAA35D
:10461C0012C0EC30A0E0FA0771F4A9A1BAA1AF382E
:10462C00E2E0BE0720F4E4E60E943EE502C0EFEFB4
:10463C00FFEFE9A3FAA3F801E285F0E00E94EDE4B4
:10464C00E770F070309769F4F801A481B581E9A1A5
:10465C00FAA1EA17FB0711F4E1E001C0E0E0EF8BEF
:10466C0089C0E130A0E0FA0769F4F801A481B581B2
:10467C00E9A1FAA1EA17FB0711F0E0E001C0E1E0C3
:10468C00EF8B78C0E230A0E0FA07D1F5F801E485B1
:10469C00E170D9F0EF89E03061F0D8011696ED9118
:1046AC00FD91A9A1BAA1EA17FB0714F0E0E0EF8B8A
:1046BC000BC0D8011496ED91FD91A9A1BAA1EA17EE
:1046CC00FB0714F4E1E0EF8B1AC0EF89E03061F0E6
:1046DC00D8011696ED91FD91A9A1BAA1EA17FB0795
:1046EC0010F0E0E0EF8B0BC0D8011496ED91FD912A
:1046FC00A9A1BAA1EA17FB0710F4E1E0EF8B3AC0CD
:10470C00E330A0E0FA07D9F4EF89E03061F0D8018A
:10471C001696ED91FD91A9A1BAA1AE17BF0710F0A5
:10472C00E0E0EF8B0BC0D8011496ED91FD91A9A19F
:10473C00BAA1AE17BF0710F4E1E0EF8B1BC0E43059
:10474C00A0E0FA07B9F4D8011496ED91FD91A9A156
:10475C00BAA1AE17BF0748F0D8011696ED91FD919E
:10476C00A9A1BAA1EA17FB0708F402C0E1E001C055
:10477C00E0E0EF8BF801E485E27009F448C0F80141
:10478C00E485E07419F4EF89E03009F43FC0F801D6
:10479C00E485E078F1F0D8011C96EC91EF77EC937E
:1047AC00E0916304E073E03298F0E1EDF2E060E058
:1047BC0070E00E94EEE5E22FF0E031966F2F660F6D
:1047CC00660B762F0E94EEE584E00E94E8E32896C3
:1047DC001DC0D8011C96EC91E068EC93E091630449
:1047EC00E073E03298F0ECEDF2E060E070E00E94F3
:1047FC00EEE5E22FF0E031966F2F660F660B762F09
:10480C000E94EEE584E00E94E8E3289633C0F801AC
:10481C00E485EE1FE0E0EE1FE170AE2FEF89EA17A2
:10482C0049F1D8011C96E170E795E0E0E7950E2E72
:10483C00EC91EF77E029EC93E0916304E073E032C4
:10484C00C8F0E7EEF2E060E070E00E94EEE5E22FE7
:10485C00F0E031966F2F660F660B762F0E94EEE517
:10486C00EF8DFF27662777270E94EEE588E00E94F0
:10487C00E8E32C96D8011C96EF89E170E295E07F75
:10488C00EE0FEE0F0E2EEC91EF7BE029EC93E09106
:10489C006304EF70E13059F0E0916304EF70AE2FD8
:1048AC00E22FF0E03396B0E0EA17FB0711F4E1E0F9
:1048BC00EE8B2F5FACCAE0916304EF70E23019F01D
:1048CC00EE89E030A1F1ABA1BCA1EC91EF70ED87CA
:1048DC00AD85A93010F0E8E0ED87ED85E85FEF835A
:1048EC00E6E0E887ABA1BCA1EC91E07121F0119658
:1048FC000E94D3E507C0ABA1BCA11196ED91FD912F
:10490C0066277727E987FA876B877C87FE013E96B7
:10491C00FA93EA93EDA1FEA13596FA93EA93A9894D
:10492C00BB270E944EDDDE0116960E9483A70E94D3
:10493C0068E4A59608951A930A93AFEBB2E00E942F
:10494C0030E60E2F003029F0A02F0E94EE3EE03012
:10495C0021F0E0916304E06403C0E0916304EF7B19
:10496C00E093630410E0E0916A041E1708F07DC028
:10497C00ABE6B4E0E12FF0E0BD01AEE0B0E00E94A8
:10498C0016E5DB01AE0FBF1F1D96AC91A13008F4EC
:10499C006AC0ABE6B4E0E12FF0E0BD01AEE0B0E000
:1049AC000E9416E5DB01AE0FBF1F1D96EC91E15086
:1049BC00EC93ABE6B4E0E12FF0E0BD01AEE0B0E08B
:1049CC000E9416E5DB01AE0FBF1F1D96EC91E03087
:1049DC0009F049C0ABE6B4E0E12FF0E0BD01AEE078
:1049EC00B0E00E9416E5DB01AE0FBF1F1C96EC91E8
:1049FC00F0E00E94F1E4E370F070309781F4ABE6E4
:104A0C00B4E0E12FF0E0BD01AEE0B0E00E9416E5AD
:104A1C00DB01AE0FBF1F1C96EC91EF7713C0E1309A
:104A2C00A0E0FA0701F5ABE6B4E0E12FF0E0BD0140
:104A3C00AEE0B0E00E9416E5DB01AE0FBF1F1C9686
:104A4C00EC91E068EC93ABE6B4E0E12FF0E0BD0153
:104A5C00AEE0B0E00E9416E5DB01AE0FBF1F1C9666
:104A6C00EC91EF7BEC931F5F7ECFA0916904A1309A
:104A7C0000F1E0916904E150E0936904EF5FE0918B
:104A8C006904E030B1F4E0916404F0E0F695E79548
:104A9C00E370F070309721F4E0916404E77F07C075
:104AAC00E130A0E0FA0729F4E0916404E860E093B7
:104ABC0064040C94632AA0971A93A1E4B1E0E0E09B
:104ACC00F0E060E070E00E943CE6ADEBB2E0E4EFB9
:104ADC00F1E00E9444E6AFEBB2E0E0E00E944CE66D
:104AEC00A0ECB2E00E944CE6A8ECB2E0E0E10E943F
:104AFC004CE6A1ECB2E0E5E00E944CE6A2ECB2E0A0
:104B0C00E0E0F0E060E070E00E943CE6A6ECB2E091
:104B1C000E9430E6E1600E944CE6FE017196FA9329
:104B2C00EA93E0E0EA93A0E1B0E00E9460DDFE01D0
:104B3C003196FA93EA93E0E0EA93A0E1B0E00E94A8
:104B4C0060DD10E0143308F046C1ACECB2E0E12FAC
:104B5C00F0E0BD01AEE0B0E00E9416E5DB01AE0F67
:104B6C00BF1FE0E0F0E060E070E00E943CE6ACECDF
:104B7C00B2E0E12FF0E0BD01AEE0B0E00E9416E53E
:104B8C00DB01AE0FBF1F1496E0E0F0E00E9444E69C
:104B9C00ACECB2E0E12FF0E0BD01AEE0B0E00E9481
:104BAC0016E5DB01AE0FBF1F1696E0E0F0E00E94A9
:104BBC0044E6ACECB2E0E12FF0E0BD01AEE0B0E0D9
:104BCC000E9416E5DB01AE0FBF1F1896EFEFFFEF4B
:104BDC000E9444E6ACECB2E0E12FF0E0BD01AEE0A7
:104BEC00B0E00E9416E5DB01AE0FBF1F1A960E94C3
:104BFC0030E6E07FE6600E944CE6ACECB2E0E12FE0
:104C0C00F0E0BD01AEE0B0E00E9416E5DB01AE0FB6
:104C1C00BF1F1A960E9430E6EF78E0620E944CE6C5
:104C2C00ACECB2E0E12FF0E0BD01AEE0B0E00E94F0
:104C3C0016E5DB01AE0FBF1F1A960E9430E6EF7728
:104C4C000E944CE6ACECB2E0E12FF0E0BD01AEE02E
:104C5C00B0E00E9416E5DB01AE0FBF1F1C960E9450
:104C6C0030E6EE7F0E944CE6ACECB2E0E12FF0E0D7
:104C7C00BD01AEE0B0E00E9416E5DB01AE0FBF1F38
:104C8C001B960E9430E6E07F0E944CE6ACECB2E052
:104C9C00E12FF0E0BD01AEE0B0E00E9416E5DB01D3
:104CAC00AE0FBF1F1B960E9430E6EF700E944CE6C1
:104CBC00ACECB2E0E12FF0E0BD01AEE0B0E00E9460
:104CCC0016E5DB01AE0FBF1F1C960E9430E6ED7F90
:104CDC000E944CE6ACECB2E0E12FF0E0BD01AEE09E
:104CEC00B0E00E9416E5DB01AE0FBF1F1C960E94C0
:104CFC0030E6E37F0E944CE6ACECB2E0E12FF0E052
:104D0C00BD01AEE0B0E00E9416E5DB01AE0FBF1FA7
:104D1C001C960E9430E6EF7E0E944CE6ACECB2E0B2
:104D2C00E12FF0E0BD01AEE0B0E00E9416E5DB0142
:104D3C00AE0FBF1F1C960E9430E6EF710E944CE62E
:104D4C00ACECB2E0E12FF0E0BD01AEE0B0E00E94CF
:104D5C0016E5DB01AE0FBF1F1D96E0E00E944CE68E
:104D6C00FE017196FA93EA93E3EFF2E060E070E0F3
:104D7C000E94EEE5E12FF0E031966F2F660F660B87
:104D8C00762F0E94EEE584E00E94ADE32A96E12F97
:104D9C00F0E0A0EDBCE30E94DBE4EA0FFB1FFA930A
:104DAC00EA93FE017396FA93EA93A0E10E94312DE7
:104DBC00E12FF0E0A0E1B0E40E94DDE4EA0FFB1F7C
:104DCC00FA93EA93FE013396FA93EA93A8E00E94D1
:104DDC00312D1F5FB7CE0E949A1B1881A1960895A2
:104DEC001A93E3E4F7E0FA93EA93E0E0EA93ACE396
:104DFC00B0E00E9460DD10E0143108F040C0AFE07C
:104E0C00B7E0E12FF0E0BD01A6E0B0E00E9416E5AE
:104E1C00DB01AE0FBF1F0E9430E6E03071F1A3E062
:104E2C001A9FF001ED5BF84FDF01EC91E160EC9320
:104E3C00A3E01A9FF001ED5BF84FFF93EF93AFE007
:104E4C00B7E0E12FF0E0BD01A6E0B0E00E9416E56E
:104E5C00DB01AE0FBF1F12960E942CE6DF01EEE0C5
:104E6C000E949CE4E370AF91BF91E370E295E07F08
:104E7C000E2EEC91EF7CE029EC931F5FBDCF1991C6
:104E8C0008950E9461E410E0143108F013C2A3E00D
:104E9C001A9FF001ED5BF84FE081E17009F408C254
:104EAC00AFE0B7E0E12FF0E0BD01A6E0B0E00E947A
:104EBC0016E5DB01AE0FBF1F0E9430E6AE2F0E943D
:104ECC00EE3E0E2FA3E01A9FF001ED5BF84FE08150
:104EDC00F0E00E94EDE4E370F070309709F07AC0D6
:104EEC00003009F45BC01A9FF001ED5BF84FE081D4
:104EFC00E47009F052C0AFE0B7E0E12FF0E0BD0183
:104F0C00A6E0B0E00E9416E5DB01AE0FBF1F1296C3
:104F1C000E942CE6FF73AF0100240416050688F4EA
:104F2C00A3E01A9FF001ED5BF84FDF01EC91E86014
:104F3C00EC93A3E01A9FF001EC5BF84F4083518394
:104F4C002CC0A3E01A9FF001ED5BF84FDF01EC9150
:104F5C00E77FEC93A3E01A9FF001ED5BF84FDF01C4
:104F6C00EC91E260EC93A3E01A9FF001EC5BF84F3C
:104F7C00FF93EF93AFE0B7E0E12FF0E0BD01A6E0C7
:104F8C00B0E00E9416E5DB01AE0FBF1F14960E9425
:104F9C002CE6AF91BF91ED93FC931BC0A3E01A9F3D
:104FAC00F001EC5BF84FA0E0B0E0A083B183A3E08C
:104FBC001A9FF001ED5BF84FDF01EC91E77FEC936A
:104FCC00A3E01A9FF001ED5BF84FDF01EC91ED7F50
:104FDC00EC931DC1E130A0E0FA0709F063C0A09189
:104FEC005D0EAB3008F413C1003041F4A3E01A9FFE
:104FFC00F001ED5BF84FE081E47009F452C0AFE0D2
:10500C00B7E0E12FF0E0BD01A6E0B0E00E9416E5AC
:10501C00DB01AE0FBF1F12960E942CE6FF73AF018F
:10502C0000240416050688F4A3E01A9FF001ED5B3A
:10503C00F84FDF01EC91E860EC93A3E01A9FF001CC
:10504C00EC5BF84F408351832CC0A3E01A9FF00116
:10505C00ED5BF84FDF01EC91E860EC93A3E01A9F55
:10506C00F001ED5BF84FDF01EC91E260EC93A3E013
:10507C001A9FF001EC5BF84FFF93EF93AFE0B7E0B2
:10508C00E12FF0E0BD01A6E0B0E00E9416E5DB01E7
:10509C00AE0FBF1F14960E942CE6AF91BF91ED93FB
:1050AC00FC93B5C0E230A0E0FA0709F05EC0003016
:1050BC0041F0A3E01A9FF001ED5BF84FE081E47042
:1050CC0009F052C0AFE0B7E0E12FF0E0BD01A6E07F
:1050DC00B0E00E9416E5DB01AE0FBF1F12960E94D6
:1050EC002CE6FF73AF0100240416050688F4A3E038
:1050FC001A9FF001ED5BF84FDF01EC91E860EC9347
:10510C00A3E01A9FF001EC5BF84F408351832CC055
:10511C00A3E01A9FF001ED5BF84FDF01EC91E86022
:10512C00EC93A3E01A9FF001ED5BF84FDF01EC91DB
:10513C00E260EC93A3E01A9FF001EC5BF84FFF9355
:10514C00EF93AFE0B7E0E12FF0E0BD01A6E0B0E0F7
:10515C000E9416E5DB01AE0FBF1F14960E942CE6D1
:10516C00AF91BF91ED93FC9352C0E330A0E0FA07EE
:10517C0009F04DC0A0915D0EAB3008F448C0003072
:10518C0099F0A3E01A9FF001ED5BF84FDF01EC9171
:10519C00E260EC93A3E01A9FF001EC5BF84FA0E007
:1051AC00B0E0A083B18333C0A3E01A9FF001ED5BA4
:1051BC00F84FE081E47059F11A9FF001ED5BF84F64
:1051CC00DF01EC91E77FEC93A3E01A9FF001ED5B1C
:1051DC00F84FDF01EC91E260EC93A3E01A9FF00131
:1051EC00EC5BF84FFF93EF93AFE0B7E0E12FF0E00B
:1051FC00BD01A6E0B0E00E9416E5DB01AE0FBF1FBB
:10520C0014960E942CE6AF91BF91ED93FC93A3E012
:10521C001A9FF001ED5BF84FDF01E02FE170EE0F0C
:10522C00EE0F0E2EEC91EB7FE029EC93AFE0B7E0A4
:10523C00E12FF0E0BD01A6E0B0E00E9416E5DB0135
:10524C00AE0FBF1F11960E9430E63E2F3030A1F0FA
:10525C00A3E01A9FF001ED5BF84FE081E87039F4A0
:10526C001A9FF001ED5BF84FE081E27029F0A32F5B
:10527C000E94EE3EE03009F41BC0A3E01A9FF0013F
:10528C00ED5BF84FDF01EC91E77FEC93A3E01A9F05
:10529C00F001ED5BF84FDF01EC91ED7FEC93A3E0B7
:1052AC001A9FF001EC5BF84FA0E0B0E0A083B18353
:1052BC001F5FEACD0E9468E44AC11A9310E01431D2
:1052CC0008F069C0A3E01A9FF001ED5BF84FE08194
:1052DC00E17061F01A9FF001EC5BF84FDF01ED918A
:1052EC00FC91119700240E160F0608F052C0A3E093
:1052FC001A9FF001EC5BF84FDF01ED91FD913197B6
:10530C00FE93EE93A3E01A9FF001EC5BF84FDF01E4
:10531C00ED91FC9111973097E1F5A3E01A9FF00104
:10532C00ED5BF84FE081E87059F11A9FF001ED5BED
:10533C00F84FDF01EC91E77FEC93A3E01A9FF001AB
:10534C00EC5BF84FFF93EF93AFE0B7E0E12FF0E0A9
:10535C00BD01A6E0B0E00E9416E5DB01AE0FBF1F59
:10536C0014960E942CE6AF91BF91ED93FC93A3E0B1
:10537C001A9FF001ED5BF84FDF01EC91E26008C081
:10538C00A3E01A9FF001ED5BF84FDF01EC91ED7F8C
:10539C00EC931F5F94CF0C940C2F60971A93FE0123
:1053AC003196FA93EA93E0E0EA93A0E1B0E00E9430
:1053BC0060DD10E0143108F048C0FE013196FA931C
:1053CC00EA93E0E0EA93A6E0B0E00E9460DDAFE093
:1053DC00B7E0E12FF0E0BD01A6E0B0E00E9416E5D9
:1053EC00E60FF71FFA93EA93FE013396FA93EA93CA
:1053FC00A6E081D0FE013196FA93EA93EAEFF2E04F
:10540C0060E070E00E94EEE5E12FF0E031966F2F46
:10541C00660F660B762F0E94EEE584E00E94ADE3EA
:10542C002A96E12FF0E0A0E8B2E40E94DBE4EA0F58
:10543C00FB1FFA93EA93FE013396FA93EA93A0E1E9
:10544C000E94312DA8951F5FB5CF188161960895E4
:10545C001A930A93EAE0F3E060E070E00E94EEE554
:10546C0080E00E94E8E324960FE010E0E5E4F1E030
:10547C000E171F0738F4D801E0E00E944CE60F5FCE
:10548C001F4FF4CF0E94CD31A0E0B0E0E0E50E94C8
:10549C004CE6A1E0B0E0E3E40E944CE6A2E0B0E010
:1054AC00EDE40E944CE6A3E0B0E0E0E50E944CE69F
:1054BC00A4E0B0E0E0E00E944CE609911991089557
:1054CC000E9461E40A2F2E813F814885598510E0A6
:1054DC00101778F4E12FF0E0E40FF51F0F01D9015C
:1054EC00EE27A10FBE1F0E9430E6D001EC931F5F88
:1054FC00EFCF0C94372E0E9461E40A2F2E813F814E
:10550C004885598510E0101778F4E12FF0E0E40F8E
:10551C00F51F0F01D901EE27A10FBE1FEC91D00191
:10552C000E944CE61F5FEFCF9CC30E9463E40A2FDE
:10553C002C813D8110E0101740F4D901EE27A10F0A
:10554C00BE1F0E944CE61F5FF6CF0E946AE42696AF
:10555C0008950E9461E43A2F4E815F8110E0E32FA1
:10556C00F0E03197A12FB0E0AE17BF078CF4DA0151
:10557C00EE27A10FBE1F0C91003051F0A885B98504
:10558C00EE27A10FBE1FE02F0E944CE61F5FE7CF56
:10559C00A885B985EE27A10FBE1F0E944CE6E12F0E
:1055AC0060C30E9461E43A2F4E815F8110E0E32FCB
:1055BC00F0E03197A12FB0E0AE17BF0794F4DA01F9
:1055CC00EE27A10FBE1F0E9430E60E2F003049F0CF
:1055DC00E12FA885B985F0E0EA0FFB1F00831F5F60
:1055EC00E6CFA885B985EE27A10FBE1FEC93E12F5E
:1055FC0038C32E97D1500E9463E410E0133030F57D
:10560C00FE01E250FF4FFA93EA93E0E0F0E0FA93E8
:10561C00EA93A4E1B0E06CD1E03089F0E0915B0E4C
:10562C00EE7FE0935B0EFE01E250FF4FFA93EA939C
:10563C00ACEBB3E00E9470DDE03041F005C0E091CE
:10564C005B0EE160E0935B0E1F5FD8CF133011F45B
:10565C002CD194C0E0E0F0E0E093CC03F093CD03C8
:10566C0020E030E0283EE3E03E0708F059C0203D42
:10567C00E3E03E0710F409E103C0E8EEE21B0E2F55
:10568C00FE013496FA93EA93E091CA03F091CB03AE
:10569C0060E870E0AAE0B0E00E9416E5E60FF71FA4
:1056AC00FA93EA93EAE0E09FF001DF0121D1E030C8
:1056BC00A1F110E0101788F52F5F3F4FAAE01A9F59
:1056CC00F001DE011496AE0FBF1F1696EC91E03080
:1056DC0021F1AAE01A9FF001DE011496AE0FBF1F54
:1056EC00ED91FD91A091CC03B091CD03AE17BF0706
:1056FC0090F4AAE01A9FF001DE011496AE0FBF1FC2
:10570C00ED91FC911197E093CC03F093CD03209392
:10571C00CA033093CB031F5FCDCF101708F0A2CF75
:10572C00ACECB3E0ED91FD913196FE93EE93A0912C
:10573C00CA03B091CB03A83EE3E0BE0728F0E0E03B
:10574C00E093CA03E093CB03E1E2F3E060E070E0A6
:10575C000E94EEE5E091CA03F091CB036627772710
:10576C000E94EEE5E091CC03F091CD0366277727FC
:10577C000E94EEE588E00E94E8E32C960E946AE421
:10578C006296DF5F08951A931A2F1A93E0E0EA935A
:10579C00A0E0B0E001D03AC32A970E9461E49D01D9
:1057AC0008895989E6E3F3E060E070E00E94EEE5D9
:1057BC00E52FFF27662777270E94EEE5E02FFF27CE
:1057CC00662777270E94EEE588E00E94E8E32C9696
:1057DC00543638F0ACECB9E00E942CE631960E94BD
:1057EC0044E6E091CC03F091CD03EE83FF83E0918E
:1057FC00F410F091F5106091F6107091F710E887A5
:10580C00F9876A877B875C870D872E873F8710E037
:10581C001330A0F5E091CA03F091CB0360E870E07F
:10582C00AAE0B0E00E9416E5E60FF71FFA93EA93A0
:10583C00FE013896FA93EA93AAE00DD1E030E1F03C
:10584C00ACECB3E0ED91FD913196FE93EE93AAECA6
:10585C00B3E0ED91FD913196FE93EE93A091CA03C6
:10586C00B091CB03A83EE3E0BE0728F0E0E0E09364
:10587C00CA03E093CB0302C01F5FCACF0E9468E447
:10588C0062960895E1E0F0E0E093CC03F093CD0351
:10589C00E0E0E093CA03E093CB03E0E8F0E0FA9396
:1058AC00EA93A0E1B7E2E1D108956497FE01FA937F
:1058BC00EA93E0E0EA93A4E1B0E00E9460DDFE012F
:1058CC00FA93EA93AAE1B3E080E090E00E94A8DDAD
:1058DC00E2E0E887E0E1E987E0E0F0E0FA93EA93C0
:1058EC00FE013296FA93EA93A4E1B5D0649608953A
:1058FC000E9461E4AD0110E01436C0F4A198EDB53E
:10590C00E093520EE5E0EEBDEDB5E7FFFDCFE0E034
:10591C00EEBDEDB5E7FFFDCF0EB5A19A00FF06C0B9
:10592C0080E991E00197F1F71F5FE6CF143659F447
:10593C00E885F985FA93EA93E0E0EA93DA010E94AC
:10594C0060DDE0E08EC1A198EDB5E093520EE3E08E
:10595C00EEBDEDB5E7FFFDCFEF81F070EEBDEDB51F
:10596C00E7FFFDCFEE81EEBDEDB5E7FFFDCF20E00B
:10597C0030E02417350788F4EDB5E093520EE0E0E3
:10598C00EEBDEDB5E7FFFDCFA885B985A20FB31F1E
:10599C00EEB5EC932F5F3F4FECCFA19A61C10E9403
:1059AC0061E42A2F4E815F8110E01436C0F4A19877
:1059BC00EDB5E093520EE5E0EEBDEDB5E7FFFDCFA2
:1059CC00E0E0EEBDEDB5E7FFFDCF3EB5A19A30FFAF
:1059DC0006C080E991E00197F1F71F5FE6CF14361E
:1059EC0029F4A885B985E0E0EC933BC1213008F09F
:1059FC002150A198EDB5E093520EE3E0EEBDEDB56C
:105A0C00E7FFFDCFE52FF070EEBDEDB5E7FFFDCF65
:105A1C004EBDEDB5E7FFFDCF00E00217A0F4EDB5EC
:105A2C00E093520EE0E0EEBDEDB5E7FFFDCFA885AB
:105A3C00B985EE27A00FBE1FEEB5EC93EEB5E030A6
:105A4C0011F00F5FEACFA19AA885B985EE27A00FB8
:105A5C00BE1FEC9305C10E9461E45A2F10E0513037
:105A6C0008F47AC000E00436C0F4A198EDB5E093D8
:105A7C00520EE5E0EEBDEDB5E7FFFDCFE0E0EEBD8B
:105A8C00EDB5E7FFFDCF3EB5A19A30FF06C080E92A
:105A9C0091E00197F1F70F5FE6CF043611F4E0E0E7
:105AAC00E0C0A198EDB5E093520EE6E0EEBDEDB589
:105ABC00E7FFFDCFA19A00000000A198EDB5E0939F
:105ACC00520EE5E0EEBDEDB5E7FFFDCFE0E0EEBD3B
:105ADC00EDB5E7FFFDCF3EB5A19A31FF3AC0E885A1
:105AEC00EF77A0E8AE1B2A2F521708F4252FA198A8
:105AFC00EDB5E093520EE2E0EEBDEDB5E7FFFDCF64
:105B0C00E985F070EEBDEDB5E7FFFDCFE885EEBDA4
:105B1C00EDB5E7FFFDCF00E0021780F4EDB5E093A3
:105B2C00520EAE81BF81EE27A10FBE1FEC91EEBDD0
:105B3C00EDB5E7FFFDCF0F5F1F5FEECFA19A521BB4
:105B4C00E22FF0E0A885B985EA0FFB1FE887F987FB
:105B5C0002C0E0E086C083CF83C00E9461E45A2F6C
:105B6C0010E0513008F47CC000E00436C0F4A19879
:105B7C00EDB5E093520EE5E0EEBDEDB5E7FFFDCFE0
:105B8C00E0E0EEBDEDB5E7FFFDCF3EB5A19A30FFED
:105B9C0006C080E991E00197F1F70F5FE6CF04367C
:105BAC0011F4E0E05EC0A198EDB5E093520EE6E092
:105BBC00EEBDEDB5E7FFFDCFA19A00000000A19866
:105BCC00EDB5E093520EE5E0EEBDEDB5E7FFFDCF90
:105BDC00E0E0EEBDEDB5E7FFFDCF3EB5A19A31FF9C
:105BEC003CC0E885EF77A0E8AE1B2A2F521708F4CB
:105BFC00252FA198EDB5E093520EE2E0EEBDEDB588
:105C0C00E7FFFDCFE985F070EEBDEDB5E7FFFDCF09
:105C1C00E885EEBDEDB5E7FFFDCF00E0021780F49F
:105C2C00AE81BF81EE27A10FBE1F3C91EDB5E09375
:105C3C00520E3EBDEDB5E7FFFDCF0F5F1F5FEECF00
:105C4C00A19A303069F0521BE22FF0E0A885B9859B
:105C5C00EA0FFB1FE887F98702C0E0E002C081CFA2
:105C6C00E1E00E9468E42A9608950E9461E4AD0187
:105C7C0010E000240416050608F07BC000E0043692
:105C8C00C0F4A198EDB5E093520EE5E0EEBDEDB594
:105C9C00E7FFFDCFE0E0EEBDEDB5E7FFFDCF3EB594
:105CAC00A19A30FF06C080E991E00197F1F70F5FF0
:105CBC00E6CF043611F4E0E05DC0A198EDB5E093B9
:105CCC00520EE6E0EEBDEDB5E7FFFDCFA19A000068
:105CDC000000A198EDB5E093520EE5E0EEBDEDB5F8
:105CEC00E7FFFDCFE0E0EEBDEDB5E7FFFDCF3EB544
:105CFC00A19A31FF3BC0EE81EF77A0E8AE1B2A2FB3
:105D0C00FA01B0E0EA17FB0708F4242FA198EDB5CF
:105D1C00E093520EE2E0EEBDEDB5E7FFFDCFEF8173
:105D2C00F070EEBDEDB5E7FFFDCFEE81EEBDEDB54C
:105D3C00E7FFFDCF00E0021758F4EDB5E093520EEB
:105D4C00E0E0EEBDEDB5E7FFFDCF0F5F1F5FF3CFDA
:105D5C00A19AA22FBB274A1B5B0BE22FF0E0AE816E
:105D6C00BF81EA0FFB1FEE83FF8302C0E0E002C09D
:105D7C0080CFE1E00E9468E4289608951A93EFE73B
:105D8C00F7E0FA93EA93E0E0EA93A4E1B0E00E9432
:105D9C0060DD10E01530D0F5E12FAFE7B7E0F0E0B3
:105DAC000E94DFE4EA0FFB1F0F01ABEDB6E0E12F21
:105DBC00F0E00E94DFE4AE0FBF1F0E9430E6D0017E
:105DCC00EC93E12FAFE7B7E0F0E00E94DFE4EA0FDD
:105DDC00FB1F33960F01ABEDB6E0E12FF0E00E9414
:105DEC00DFE4AE0FBF1F13960E9430E6EE1FE0E01B
:105DFC00EE1FE170D001E170EE0FEE0FEE0F0E2EE4
:105E0C00EC91E77FE029EC931F5FC4CF19910895C3
:105E1C000E9463E42A2F10E0153008F0CFC1E12F67
:105E2C00AFE7B7E0F0E00E94DFE4AE0FBF1FAC912C
:105E3C00A03081F0E12FAFE7B7E0F0E00E94DFE4A3
:105E4C00AE0FBF1F1396EC91E695E695E695E170C3
:105E5C002E1709F0B1C1E12FAFE7B7E0F0E00E94D7
:105E6C00DFE4AE0FBF1FAC910E94EE3EE03009F4B0
:105E7C0079C0E12FAFE7B7E0F0E00E94DFE4AE0FAE
:105E8C00BF1F1396EC91E47009F06BC0E12FAFE7E4
:105E9C00B7E0F0E00E94DFE4AE0FBF1F1396EC9169
:105EAC00E160EC93E12FAFE7B7E0F0E00E94DFE4B4
:105EBC00AE0FBF1F1396EC91E460EC93E12FAFE7AC
:105ECC00B7E0F0E00E94DFE4EA0FFB1F33960F010E
:105EDC00ABEDB6E0E12FF0E00E94DFE4AE0FBF1FA8
:105EEC0013960E9430E6EF77E13010F0E1E001C04C
:105EFC00E0E0D001E170EE0F0E2EEC91ED7FE02989
:105F0C00EC93E12FAFE7B7E0F0E00E94DFE4EA0F9B
:105F1C00FB1F32960F01ABEDB6E0E12FF0E00E94D3
:105F2C00DFE4AE0FBF1F13960E9430E6EF77D0016F
:105F3C00EC93E12FAFE7B7E0F0E00E94DFE4EA0F6B
:105F4C00FB1F31960F01ABEDB6E0E12FF0E00E94A4
:105F5C00DFE4AE0FBF1F11960E9430E6D001EC9328
:105F6C002BC12FC0E12FAFE7B7E0F0E00E94DFE4D8
:105F7C00AE0FBF1F1396EC91EB7FEC93E12FAFE7C5
:105F8C00B7E0F0E00E94DFE4AE0FBF1F1396EC9178
:105F9C00E270B9F4E12FAFE7B7E0F0E00E94DFE484
:105FAC00AE0FBF1F1396EC91EE7FEC93E12FAFE792
:105FBC00B7E0F0E00E94DFE4AE0FBF1F1196E0E007
:105FCC00EC93E12FAFE7B7E0F0E00E94DFE4AE0F17
:105FDC00BF1F1196AC91A13008F4EEC0E12FAFE7D2
:105FEC00B7E0F0E00E94DFE4AE0FBF1F1196EC911A
:105FFC00E150EC93E12FAFE7B7E0F0E00E94DFE473
:10600C00AE0FBF1F1196EC91E03009F0D5C0E12F17
:10601C00AFE7B7E0F0E00E94DFE4AE0FBF1F1396CE
:10602C00EC91E17009F48CC0E2E4F3E060E070E024
:10603C000E94EEE5E12FF0E031966F2F660F660BB4
:10604C00762F0E94EEE584E00E94E8E32896E12F8B
:10605C00AFE7B7E0F0E00E94DFE4AE0FBF1F13968E
:10606C00EC91EE7FEC93E12FAFE7B7E0F0E00E940C
:10607C00DFE4AE0FBF1F1396EC91E27009F442C03F
:10608C00E12FAFE7B7E0F0E00E94DFE4AE0FBF1FF7
:10609C001296AC91A130A8F1E12FAFE7B7E0F0E098
:1060AC000E94DFE4AE0FBF1F1296EC91E150EC930F
:1060BC00E12FAFE7B7E0F0E00E94DFE4AE0FBF1FC7
:1060CC001296AC91A130E8F0ABEDB6E0E12FF0E028
:1060DC000E94DFE4AE0FBF1F12960E9430E60E2F17
:1060EC00E295EF70E695E6953E2F031BE6950E1BA9
:1060FC00E12FAFE7B7E0F0E00E94DFE4EA0FFB1F0F
:10610C0001831DC0ABEDB6E0E12FF0E00E94DFE4AF
:10611C00AE0FBF1F12960E9430E60E2FE295EF7065
:10612C00E695E6953E2F031BE6950E1BE12FAFE798
:10613C00B7E0F0E00E94DFE4EA0FFB1F01833CC0F4
:10614C00EAE4F3E060E070E00E94EEE5E12FF0E0BD
:10615C0031966F2F660F660B762F0E94EEE584E06A
:10616C000E94E8E32896E12FAFE7B7E0F0E00E9449
:10617C00DFE4AE0FBF1F1396EC91E160EC93ABED37
:10618C00B6E0E12FF0E00E94DFE4AE0FBF1F1196E6
:10619C000E9430E60E2FE295EF70E695E6953E2FC5
:1061AC00031BE6950E1BE12FAFE7B7E0F0E00E9472
:1061BC00DFE4EA0FFB1F01831F5F2ECECAC160977D
:1061CC001A93FE013196FA93EA93E0E0EA93A0E188
:1061DC00B0E00E9460DD10E0153008F069C0ABED56
:1061EC00B6E0E12FF0E00E94DFE4AE0FBF1FE0E06D
:1061FC000E944CE6ABEDB6E0E12FF0E00E94DFE44C
:10620C00AE0FBF1F1196E5E00E944CE6ABEDB6E079
:10621C00E12FF0E00E94DFE4AE0FBF1F1296E5E025
:10622C000E944CE6ABEDB6E0E12FF0E00E94DFE41B
:10623C00AE0FBF1F13960E9430E6E0780E944CE62A
:10624C00ABEDB6E0E12FF0E00E94DFE4AE0FBF1F34
:10625C0013960E9430E6EF770E944CE6FE013196D1
:10626C00FA93EA93E1E5F3E060E070E00E94EEE57A
:10627C00E12FF0E031966F2F660F660B762F0E94A0
:10628C00EEE584E00E94ADE32A96E12FF0E0A0EB6E
:10629C00B1E40E94DBE4EA0FFB1FFA93EA93FE01E0
:1062AC003396FA93EA93A0E10E94312D1F5F94CFAD
:1062BC0065DD188161960895E0E0E2B9EFEFE1B990
:1062CC00E1E0E5B9E7EFE4B9E5E1E8B9EFE1E7B919
:1062DC00EAE0E0936900E0E2EBB9E8EBEAB9E2E06E
:1062EC00EEB9EEE7EDB9E0E8E0936A00E0E0E1BB7F
:1062FC00A0915E0EA33430F0EFE0E0937E00E0EF6F
:10630C00E0BB08C0E7E0E0937E00E8EFE0BBE0E82C
:10631C00E5BFE5BFE7E0E4BBEFE1E3BBE1E5ECBDE6
:10632C00E1E0EDBDE6E0E093C200E8E9E093C100F6
:10633C00E0E0E093C500E3E0E093C400EDE0E4BDF1
:10634C00E0E0E6BDEFE4E7BDE2E0E0936E00089527
:10635C00E0E0E0935D0E0E94D7390E943B6B0E94F7
:10636C0006900E94D93D0E949A1B0E94890B06DD63
:10637C000E94F6260E947CDA0E94F6D20E94E1D49A
:10638C000E94890B0E94A0950E94CE4908956097A7
:10639C00A6E2B1E00E9430E6E07F0E944CE6A6E265
:1063AC00B1E00E9430E6EF7E0E944CE6A6E2B1E03E
:1063BC000E9430E6E0620E944CE6A5E2B1E0E0E02B
:1063CC000E944CE6A7E2B1E00E944CE6A8E2B1E0E4
:1063DC000E944CE6A9E2B1E00E944CE6AAE2B1E0D0
:1063EC000E944CE6ABE2B1E00E944CE6ACE2B1E0BC
:1063FC000E944CE6ADE2B1E0E4E10E944CE6AEE274
:10640C00B1E0E0E00E944CE6AFE2B1E00E944CE665
:10641C00A0E3B1E00E944CE6A1E3B1E00E944CE69F
:10642C00FE01FA93EA93E0E0EA93A0E1B0E00E9467
:10643C0060DDFE01FA93EA93A3ECB3E00E949BDDCE
:10644C00E0E0F8E3FA93EA93FE013296FA93EA93CA
:10645C00A0E10E94312DE0E0E883E0E0F6E4FA935D
:10646C00EA93FE013296FA93EA93A1E00E94312D51
:10647C00A2E3B1E0EEE1F0E0FF700F010E942CE628
:10648C00E070F07FE029F1290E9444E6A4E3B1E03A
:10649C00E0E00E944CE6A5E3B1E0EAE00E944CE6A5
:1064AC00A6E3B1E0E0E80E944CE6A7E3B1E00E946D
:1064BC004CE6E9E3F1E0FA93EA93A7E00E949B2A09
:1064CC000E94888E0E946A900E94B9480E946125A1
:1064DC000E94121B74DE0E94D3290E9410DD0E94C0
:1064EC0061D40E9479D90E94ECA40E945E8C0E9417
:1064FC005B4B0E94482C2CDFA8E0B0E0E3E00E944C
:10650C004CE66AD1609608950E9463E4A89522E255
:10651C0031E000E010E0273DE9E03E0748F4D90106
:10652C000E9430E6F0E00E0F1F1F2F5F3F4FF3CF9E
:10653C00E7E6F3E060E070E00E94EEE5F801662724
:10654C0077270E94EEE584E00E94E8E32896A89560
:10655C00F8010E946AE424960895EF97EF97269726
:10656C000E9461E4E091600EED7FE093600EEB7FA2
:10657C00E093600EE77FE093600EE0E0E093620E44
:10658C00A8E0B0E00E9430E6E330B1F5E091600E97
:10659C00E260E093600EA2E2B1E00E9430E6E130EE
:1065AC0039F5E091600EE460E093600EADDFAF0171
:1065BC00A3E2B1E00E942CE6E887F987E985F0E0D8
:1065CC00F0E04E1B5F0BE885F985F0E0F0E04E1B28
:1065DC005F0BE885F985E417F50731F4E091600E5F
:1065EC00E860E093600E03C0E4E0E093620E03C049
:1065FC00E2E0E093620E03C0E1E0E093620E30E073
:10660C0040E050E0E2E2F1E0EE83FF83AE81BF8137
:10661C00A73DE9E0BE0708F04BC0E7EDF9E0EA1B47
:10662C00FB0BE138A0E0FA0710F010E804C0AE81D3
:10663C00E7EDEA1B1E2FFE013A96FA93EA93E2E28B
:10664C00F1E0A0E0B8E20E94FEE5EA1BFB0BA88596
:10665C00B985EA0FFB1FFA93EA93A12FBB270E947F
:10666C007E2C303071F4AA85A13031F0E091620EAD
:10667C00E061E093620E1CC0EB85FC85E887F9872E
:10668C0031E000E0011760F4E02FF0E0DE011A9633
:10669C00AE0FBF1FEC91F0E04E0F5F1F0F5FF2CFFC
:1066AC00A895EE81FF81E058FF4FEE83FF83AECFBC
:1066BC00313009F08BC0E985F0E0F0E04E1B5F0B48
:1066CC00E885F985F0704E1B5F0BE885F985E417BA
:1066DC00F50709F076C0E091600EE87009F070C023
:1066EC00AFEFBFE00E9430E6EF5F0E944CE6E09116
:1066FC00620EE064E093620EE2E2F1E0EE83FF836F
:10670C00AE81BF81A73DE9E0BE07B8F5E7EDF9E042
:10671C00EA1BFB0BE138A0E0FA0710F010E804C00C
:10672C00AE81E7EDEA1B1E2FFE013A96FA93EA932F
:10673C00E2E2F1E0A0E0B8E20E94FEE5EA1BFB0B0E
:10674C00A885B985EA0FFB1FFA93EA93A12FBB2703
:10675C000E947E2CEE81FF81FA93EA93FE013C9617
:10676C00FA93EA93A12F0E94812AA895EE81FF81CA
:10677C00E058FF4FEE83FF83C3CFC6DEAF01A3E229
:10678C00B1E00E942CE6E887F987E985F0E0F0E0BB
:10679C004E1B5F0BE885F985F0E0F0E04E1B5F0BBC
:1067AC00E885F985E417F50731F4E091600EE860AF
:1067BC00E093600E05C0E091620EE068E093620E1B
:1067CC0005C0E091620EE062E093620E0E9468E404
:1067DC00EF96EF962C960895EF97EF9724970E94DB
:1067EC0061E4E4E7F3E060E070E00E94EEE580E055
:1067FC000E94E8E32496A2E2B1E0E1E00E944CE6BC
:10680C00A3E2B1E0E0E0F0E00E9444E67DDEAF01FF
:10681C00A3E2B1E00E942CE6EE83FF83EF81F0E06F
:10682C00F0E04E1B5F0BEE81FF81F0E0F0E04E1BC1
:10683C005F0BA3E2B1E0FA010E9444E622E231E0F0
:10684C00273DE9E03E0760F5E7EDF9E0E21BF30BCD
:10685C00E138A0E0FA0710F010E803C0E7EDE21B06
:10686C001E2FFE013896FA93EA933A932A93A12F9E
:10687C000E94662AE2E2F1E0A0E0B8E20E94FEE5A6
:10688C00EA1BFB0BE20FF31FFA93EA93FE013A9615
:10689C00FA93EA93A12F0E94312D20583F4FD0CF6D
:1068AC00E091600EE460E093600EE860E093600EAF
:1068BC00E0E0E093620EE091600EE07129F0E0916F
:1068CC00600EE160E093600E0E9468E4EF96EF9634
:1068DC002A960895EF97EF9722970E9461E44A2F2A
:1068EC00403039F5A4E1B0E0E3E70E944CE6A3E2C6
:1068FC00B0E0E1E00E944CE6A4E2B0E0E0E0F0E0C1
:10690C000E9444E620E030E004E110E0E8E1F1E030
:10691C000E171F0748F4D8010E9430E6F0E02E0F46
:10692C003F1F0F5F1F4FF2CFA4E2B0E0F9010E94AE
:10693C0044E600E010E00430E1E01E0748F5E4E036
:10694C00F1E0E01BF10BE138A0E0FA0710F050E8A1
:10695C0003C0E4E0E01B5E2FFE013696FA93EA9347
:10696C00E4E1F0E0E00FF11FFA93EA93A52F0E9407
:10697C00662AF801E058F140FA93EA93FE01389642
:10698C00FA93EA93A52F0E94312D00581F4FD3CFB5
:10699C000E9468E4EF96EF96289608950E9461E4B1
:1069AC0020E030E004E110E0E8E1F1E00E171F0711
:1069BC0048F4D8010E9430E6F0E02E0F3F1F0F5F25
:1069CC001F4FF2CFA4E2B0E00E942CE6AF01E52FFE
:1069DC00F0E0F0E02E1B3F0BFA01F0E0F0E02E1B94
:1069EC003F0B4217530711F4E1E001C0E0E00E94B5
:1069FC0068E426960895EF97EF9725970E9461E437
:106A0C00E091600EEF7EE093600EE0E0DE01A957AE
:106A1C00BF4FEC93DE01A957BF4FAC91A53038F5B1
:106A2C00A0E0B0E00E9430E6E035C1F4A1E0B0E0B7
:106A3C000E9430E6E33491F4A2E0B0E00E9430E62C
:106A4C00ED3461F4A3E0B0E00E9430E6E03531F4BF
:106A5C00A4E0B0E00E9430E6E03009F001C007C0CD
:106A6C00DE01A957BF4FEC91EF5FEC93D3CFDE0162
:106A7C00A957BF4FAC91A53039F40E942E2AE09152
:106A8C00610EE160E093610EA3E2B0E00E9430E69B
:106A9C00E03061F4A4E2B0E00E942CE6309731F4CF
:106AAC00A2E2B0E00E9430E6EF3109F008C0E091BC
:106ABC00610EE260E093610EA0E00CDF0EC06EDFB1
:106ACC00E03031F0E091600EE061E093600E05C0C3
:106ADC00E091610EE460E093610EE0E0DE01AA5704
:106AEC00BF4FEC93E0E0F0E08F019F010430E1E058
:106AFC001E0708F061C0E4E0F1E0E01BF10BE138A7
:106B0C00A0E0FA0710F0E0E802C0E4E0E01BDE01D0
:106B1C00A857BF4FEC93FE013696FA93EA93F8010F
:106B2C00E058F140FA93EA93DE01A457BF4FAC91C1
:106B3C00BB270E947E2CFE01EA57FF4FE081E0301C
:106B4C00A9F4AE81A33719F4AD89A13009F008C0BE
:106B5C004E895F89E1E0DE01AA57BF4FEC9306C076
:106B6C00E091610EE860E093610E26C0E0E0DE018A
:106B7C00A957BF4FEC93FE01E857FF4FE081DE01B0
:106B8C00A957BF4FAC91AE17A0F4FE01E957FF4FC8
:106B9C00E081F0E0DE011696AE0FBF1FEC91F0E045
:106BAC002E0F3F1FDE01A957BF4FEC91EF5FEC9307
:106BBC00E2CF00581F4F9ACFE52FF0E0F0E02E1BEC
:106BCC003F0BFA01F0E0F0E02E1B3F0BDE01AA5761
:106BDC00BF4FAC91A13019F44217530709F059C0BB
:106BEC00E091600EE07109F053C0E091610EE0613C
:106BFC00E093610E00E010E00430E1E01E0798F530
:106C0C00E7EDF9E0E01BF10BE138A0E0FA0710F03A
:106C1C00E0E802C0E7EDE01BDE01A857BF4FEC93A4
:106C2C00FE013696FA93EA93F801E058F140FA9394
:106C3C00EA93DE01A457BF4FAC91BB270E947E2C78
:106C4C00E4E1F0E0E00FF11FFA93EA93FE013896CD
:106C5C00FA93EA93DE01A457BF4FAC910E94812AAC
:106C6C0000581F4FC9CF9ADEE03069F0E091600EFA
:106C7C00E061E093600EAEEFBFE00E9430E6EF5FA4
:106C8C000E944CE605C0E091610EE062E093610E5B
:106C9C0017C0E091610EE064E093610EE091600E2C
:106CAC00E07171F0A1E016DEADEFBFE00E9430E6BE
:106CBC00EF5F0E944CE6E091610EE068E093610E9C
:106CCC000E9468E4EF96EF962B960895EEE7F3E0BA
:106CDC0060E070E00E94EEE5E2E0F0E060E070E081
:106CEC000E94EEE5E0E1F0E060E070E00E94EEE58D
:106CFC00E1E0F0E060E070E00E94EEE58CE00E94E4
:106D0C00E8E36096E9EAF3E060E070E00E94EEE50B
:106D1C00A5E1B0E00E942CE6662777270E94EEE5FD
:106D2C0084E00E94E8E32896E5EBF3E060E070E095
:106D3C000E94EEE5A7E1B0E00E9430E6FF2766274F
:106D4C0077270E94EEE5A8E1B0E00E9430E6FF272D
:106D5C00662777270E94EEE588E00E94E8E32C96F0
:106D6C00EDECF3E060E070E00E94EEE5E0915E0E89
:106D7C00FF27662777270E94EEE5AAE1B0E00E9484
:106D8C0030E6FF27662777270E94EEE588E00E9411
:106D9C00E8E32C96E8EEF3E060E070E00E94EEE5AC
:106DAC00E091F410F091F5106091F6107091F710DD
:106DBC000E94EEE584E00E94E8E32896E091600EE4
:106DCC00E27009F444C0E091600EE47031F1E6EF3A
:106DDC00F3E060E070E00E94EEE5A3E2B1E00E9417
:106DEC002CE6662777270E94EEE584E00E94E8E314
:106DFC002896E091600EE87029F0E7E0F4E060E09E
:106E0C0070E004C0EBE0F4E060E070E00E94EEE5BE
:106E1C0080E00E94E8E3249619C0E2E1F4E060E02F
:106E2C0070E00E94EEE5A2E2B1E00E9430E6FF279E
:106E3C00662777270E94EEE5E1E0F0E060E070E085
:106E4C000E94EEE588E00E94E8E32C9619C0E7E288
:106E5C00F4E060E070E00E94EEE5A8E0B0E00E9493
:106E6C0030E6FF27662777270E94EEE5E3E0F0E0A7
:106E7C0060E070E00E94EEE588E00E94E8E32C966A
:106E8C00ECE3F4E060E070E00E94EEE5AFEFBFE011
:106E9C000E9430E6FF27662777270E94EEE5ADEFCC
:106EAC00BFE00E9430E6FF27662777270E94EEE5B9
:106EBC00AEEFBFE00E9430E6FF27662777270E94DF
:106ECC00EEE58CE00E94E8E36096E1E5F4E060E03A
:106EDC0070E00E94EEE5E091610EFF2766277727B0
:106EEC000E94EEE5E091620EFF27662777270E944D
:106EFC00EEE588E00E94E8E32C960895ABE0B0E064
:106F0C000E9430E6E0935E0EACE0B0E00E9430E60A
:106F1C00E0935F0ED1D90E9479A67894A1E00E94EB
:106F2C00973B0E94FF2AA89566DD17DBE091600E67
:106F3C00E07121F0E091600EE87009F405C0E09179
:106F4C00600EE160E093600E03DAA091F010B09156
:106F5C00F1108091F2109091F310AA3AE5E5BE077A
:106F6C00E0E08E07EFEF9E0719F4E4B7E0FF1AC0DC
:106F7C00EAEAF5E560E07FEFE093F010F093F110B2
:106F8C006093F2107093F310E0E0F0E060E070E8D2
:106F9C00E093F410F093F5106093F6107093F710E3
:106FAC00E093F810A2E3B1E00E942CE6FF70E093AE
:106FBC00540EF093550EA091540EB091550E1A9795
:106FCC0030F4EAE0F0E0E093540EF093550EE4B7A1
:106FDC00E3FF04C0A091F810A03009F002C0A4E0B7
:106FEC0006C0E4B7E2FF02C0A5E001C0A2E00E9427
:106FFC00C92BE0E0E4BFE093F810E4E6F4E060E0D5
:10700C0070E00E94EEE580E00E94E8E32496F09A9E
:10701C004BD2E0912409E87FE260E0932409E091EF
:10702C006304EF7CE062E0936304E2E0E093A50D7F
:10703C00E1E0E093580EA2E3B1E00E942CE6FF7071
:10704C00339770F4A2E3B1E0E3E0F0E0FF700F01DE
:10705C000E942CE6E070F07FE029F1290E9444E6C2
:10706C00E091610EE03049F0EAE0EA93E0E0EA9367
:10707C00A091610EBB270E94D22BE091620EE030F2
:10708C0049F0EBE0EA93E0E0EA93A091620EBB27B3
:10709C000E94D22BA091B30AA03071F4A0919E0B48
:1070AC00E0919F0BEA1741F4A0917A00A03021F4F3
:1070BC00A091580EA03009F005C0E1E0E3BF88951F
:1070CC00E0E0E3BFA091640EA13060F0E091640EAB
:1070DC00E150E093640EEF5FE091600EE07211F40A
:1070EC000E94370C0E940606A0914608A43038F086
:1070FC000E9468410E94A6DBE0E0E0934608A09164
:10710C00580EA13008F427C1E091580EE150E093DD
:10711C00580EEF5FE5E0E093640EA0E0F799A1E074
:10712C00E1E0EA2711F4F79801C0F79AF79BE6C063
:10713C000E9482D70E94CFDBE091600EE072D9F4FE
:10714C00E091BB07F0E0E130A0E0FA0719F40E94EF
:10715C00544D11C0E230A0E0FA0721F0E330A0E07A
:10716C00FA0719F40E947B5D06C0E430A0E0FA0730
:10717C0011F40E94EC63A1E00E940E2FA0E020FC11
:10718C00A1E0E1E0EA27E894EE2309F0689420F806
:10719C0020FE0FC00E9455D30E944727E091460E57
:1071AC00E07439F0E091460EEF7BE093460E0E94BE
:1071BC009A9AA091860EA43030F4E091860EEF5F7F
:1071CC00E093860E92C0E0E0E093860EA0E021FCF6
:1071DC00A1E0E1E0EA27E894EE2309F0689421F8B5
:1071EC0021FE83C0A895A0915D0EAF3F30F4E091D5
:1071FC005D0EEF5FE0935D0EE150A091630EA13048
:10720C0060F0E091630EE150E093630EEF5FE0916C
:10721C00630EE03011F4A0E05DDBA091530EA130C1
:10722C0030F0E091530EE150E093530E17C0E4E0C0
:10723C00E093530EABE1B9E00A2EEC91E295E170CC
:10724C00A1E0EA27A02DE170E295E07F0E2EEC91F3
:10725C00EF7EE029EC93E0E0E0931609A09145085D
:10726C00A03131F41AD10E949A9A0E942F7C11C03D
:10727C00E0914308EF70E13060F0A3E4B8E080E007
:10728C00EFE00E9422E6E0914308E061E0934308BE
:10729C0001C00AD10E948ED60E9497460E94A1245A
:1072AC000E94D2DCA0E00E940E2F0E94BC160E940D
:1072BC006329E091BB07F0E0E130A0E0FA0711F49C
:1072CC000E94EE570E9484A60E94750BA091870E17
:1072DC00A93030F4E091870EEF5FE093870E05C084
:1072EC00E0E0E093870E0E9408D7E091460EEF7B1A
:1072FC00E093460E0E94F7770E94003DE091590EF4
:10730C00F0915A0E7096E093590EF0935A0EA0918C
:10731C00590EB0915A0EA533ECE0BE07E0F0E091A7
:10732C00590EF0915A0EE553FC40E093590EF09330
:10733C005A0EA4EFB0E1ED91FD916D917D91EF5F4F
:10734C00FF4F6F4F7F4F7E936E93FE93EE930E9491
:10735C00AD900E94B18BE0914308E07121F0A091B7
:10736C004508A03109F009C0E0914308EF7EE09395
:10737C00430893D00E942F7C97D00E94E4A68ACE1B
:10738C00FFCFEA93EFB7EA93E1E0E093570EE09179
:10739C00580EEF5FE093580EE150E991EFBFE99181
:1073AC00189524970E9463E410E01731B8F5A2E316
:1073BC00B0E0E12FF0E0BD01AAE0B0E00E9416E5DC
:1073CC00DB01AE0FBF1F0E942CE60E94EFE49F0171
:1073DC002030E1E03E0788F0ECE6F4E060E070E09D
:1073EC000E94EEE5F901662777270E94EEE584E01E
:1073FC000E94E8E328962FEF30E0A5EDB8E0E12FEE
:10740C00FF2766277727EC5FFE4F6F4F6BBFE69128
:10741C00F0E0EA0FFB1F20831F5FC7CFABE1B0E0AA
:10742C000E942CE69F0100240216030690F5E6E864
:10743C00E0937A00E3E0E0937C00E6ECE0937A00E2
:10744C00E0917A00E074E1F7E0917800F091790036
:10745C000E94DFE466277727A0ECB4ED81E090E092
:10746C000E941EE5EC83FD836E837F83F901AC8162
:10747C00BD818E819F81662777270E9474E5E093FA
:10748C00680EF093690EE0E0F0E0E093660EF09386
:10749C00670E0E946AE428960895E6E8E0937A0065
:1074AC00E0E0E09342080895E6E8E0937A00E0E03B
:1074BC00E8B9E0937C00E0934408E0934508E1E0F0
:1074CC00E0934208E1E5F8E0FA93EA93E0E0EA930E
:1074DC00A0E4B0E00E9460DDE5E9F8E0FA93EA93FD
:1074EC00E0E0EA93A0E2B0E00E9460DDE5EBF8E0BA
:1074FC00FA93EA93E0E0EA93A0E2B0E00E9460DD48
:10750C00E5EFF8E0FA93EA93E0E0EA93A0E2B0E06A
:10751C000E9460DDEEECE0937A00E0914308E07F9E
:10752C00E560E093430808950A921A928A93AA930D
:10753C00BA93EA93FA93EFB7EA93E0914208F0E03A
:10754C00E130A0E0FA0739F4EFECE0937A00E2E0E6
:10755C00E0934208DCC0E230A0E0FA0709F0D7C0A3
:10756C0046B0E0914408EF5FE0934408E150E091AD
:10757C004408EF71E0934408E8B9A0914408A9319C
:10758C00D0F4EEECE0937A00A0915E0EA33460F0A0
:10759C00A0914408A83010F0A83110F0E0E001C030
:1075AC00E3E0E0937C0003C0E0E0E0937C00E1E0EA
:1075BC00E09342081CC0A0914408AE3139F4E1E0DC
:1075CC00E0937C0080E58A95F1F70EC0A091440809
:1075DC00AF3139F4E2E0E0937C0080E58A95F1F775
:1075EC0003C0E0E0E0937C00EFECE0937A00E091E4
:1075FC004408E770E093880EA7E4B8E0F0E0EA0FE7
:10760C00FB1F4082E091880EE03031F4E091460897
:10761C00EF5FE0934608E150A5E9B8E0E09144083B
:10762C00F0E0AE0FBF1FEC91E429EC93A5EBB8E0B2
:10763C00E0914408F0E0EA0FFB1F0F01A081E42D5C
:10764C00E095EA2BD001EC93A0914508A03108F00D
:10765C005EC0A5EDB8E0E0914408F0E0AE0FBF1FAE
:10766C00EC91E093880EE0917800F0917900A09174
:10767C00880EB0E0AE17BF0798F4A1E5B8E0E09132
:10768C004408F0E0EE0FFF1FEA0FFB1F0F01DF01B4
:10769C00ED91FD91DF01E0917800F091790011C03E
:1076AC00A1E5B8E0E0914408F0E0EE0FFF1FEA0F0F
:1076BC00FB1F0F01DF01ED91FD91DF01E091880EC1
:1076CC00F0E0EA0FFB1FD001ED93FC93A09144086E
:1076DC00AA3140F4A0917800B0917900A03FE3E08A
:1076EC00BE0708F40AC0A5EFB8E0E0914408F0E04A
:1076FC00AE0FBF1FEC91EF5FEC93E0914408E030CC
:10770C0031F4E0914508EF5FE0934508E150E991D1
:10771C00EFBFF991E991B991A991899119900990CB
:10772C0018951A931A2F103041F05C988BE08A95BB
:10773C00F1F75C9A8BE08A95F1F72898EDB5E09318
:10774C00520EE0E4EEBDEDB5E7FFFDCFE5E0EEBD9A
:10775C00EDB5E7FFFDCFE8E0EEBDEDB5E7FFFDCF02
:10776C00289AE0911B09ED7FE0931B09A6ECB2E08F
:10777C000E9430E6E170ABE1B9E0E1700E2EEC91C5
:10778C00EE7FE029EC93EBE1F9E0DF01F49B02C022
:10779C00F59B01C002C0E1E001C0E0E0E170E795BB
:1077AC00E0E0E7950E2EEC91EF77E029EC9328982A
:1077BC00EDB5E093520EE0E4EEBDEDB5E7FFFDCF85
:1077CC00EAE0EEBDEDB5E7FFFDCFE0911B09EEBDA4
:1077DC00EDB5E7FFFDCF289AA0915E0EA334A0F083
:1077EC002898EDB5E093520EE0E4EEBDEDB5E7FF61
:1077FC00FDCFE6E0EEBDEDB5E7FFFDCFECE0EEBD75
:10780C00EDB5E7FFFDCF13C02898EDB5E093520E10
:10781C00E0E4EEBDEDB5E7FFFDCFE6E0EEBDEDB586
:10782C00E7FFFDCFE4E0EEBDEDB5E7FFFDCF289A15
:10783C002898EDB5E093520EE0E4EEBDEDB5E7FF10
:10784C00FDCFE0E0EEBDEDB5E7FFFDCFECE0EEBD2A
:10785C00EDB5E7FFFDCF289A2898EDB5E093520ED1
:10786C00E2E4EEBDEDB5E7FFFDCFEAE0EEBDEDB530
:10787C00E7FFFDCFE0E0EEBDEDB5E7FFFDCF289AC9
:10788C002898EDB5E093520EE2E4EEBDEDB5E7FFBE
:10789C00FDCFE0E0EEBDEDB5E7FFFDCFE0E0EEBDE6
:1078AC00EDB5E7FFFDCF289A2898EDB5E093520E81
:1078BC00E4E4EEBDEDB5E7FFFDCFEAE0EEBDEDB5DE
:1078CC00E7FFFDCFE0E0EEBDEDB5E7FFFDCF289A79
:1078DC002898EDB5E093520EE4E4EEBDEDB5E7FF6C
:1078EC00FDCFE0E0EEBDEDB5E7FFFDCFE0E0EEBD96
:1078FC00EDB5E7FFFDCF289AE0912009E062E09317
:10790C002009A298EDB5E093520EE0E4EEBDEDB582
:10791C00E7FFFDCFE5E0EEBDEDB5E7FFFDCFE8E01D
:10792C00EEBDEDB5E7FFFDCFA29AA298EDB5E093C1
:10793C00520EE0E4EEBDEDB5E7FFFDCFEAE0EEBDA3
:10794C00EDB5E7FFFDCFE0912009EEBDEDB5E7FF0A
:10795C00FDCFA29AA298EDB5E093520EE0E4EEBDF5
:10796C00EDB5E7FFFDCFE0E0EEBDEDB5E7FFFDCFF8
:10797C00EFE1EEBDEDB5E7FFFDCFA29AE2E2F9E053
:10798C00DF01F29B02C0F39B01C002C0E1E001C029
:10799C00E0E0E170EE0F0E2EEC91ED7FE029EC9320
:1079AC00A298EDB5E093520EE2E4EEBDEDB5E7FF23
:1079BC00FDCFEAE0EEBDEDB5E7FFFDCFE09122098A
:1079CC00EEBDEDB5E7FFFDCFA29AA298EDB5E09321
:1079DC00520EE2E4EEBDEDB5E7FFFDCFE0E0EEBD0B
:1079EC00EDB5E7FFFDCFECEFEEBDEDB5E7FFFDCF5D
:1079FC00A29AECC1A0911609A13030F0E0911609C1
:107A0C00E150E093160918C0E3E6E09316092898B4
:107A1C00EDB5E093520EE0E4EEBDEDB5E7FFFDCF22
:107A2C00EAE0EEBDEDB5E7FFFDCFE0911B09EEBD41
:107A3C00EDB5E7FFFDCF289AA0911709A13038F0DA
:107A4C00E0911709E150E0931709EF5F18C0E3E6E6
:107A5C00E09317092898EDB5E093520EE2E4EEBDE1
:107A6C00EDB5E7FFFDCFEAE0EEBDEDB5E7FFFDCFED
:107A7C00E0911D09EEBDEDB5E7FFFDCF289AA09171
:107A8C001809A13038F0E0911809E150E093180979
:107A9C00EF5F18C0E3E6E09318092898EDB5E09382
:107AAC00520EE4E4EEBDEDB5E7FFFDCFEAE0EEBD2E
:107ABC00EDB5E7FFFDCFE0911E09EEBDEDB5E7FF9B
:107ACC00FDCF289AA0911909A13038F0E09119093D
:107ADC00E150E0931909EF5F2DC0E3E6E09319093B
:107AEC00A298EDB5E093520EE0E4EEBDEDB5E7FFE4
:107AFC00FDCFEAE0EEBDEDB5E7FFFDCFE09120094B
:107B0C00EEBDEDB5E7FFFDCFA29AA298EDB5E093DF
:107B1C00520EE0E4EEBDEDB5E7FFFDCFE0E0EEBDCB
:107B2C00EDB5E7FFFDCFE0911F09EEBDEDB5E7FF29
:107B3C00FDCFA29AA0911A09A13038F0E0911A0950
:107B4C00E150E0931A09EF5F2DC0E3E6E0931A09C8
:107B5C00A298EDB5E093520EE2E4EEBDEDB5E7FF71
:107B6C00FDCFEAE0EEBDEDB5E7FFFDCFE0912209D8
:107B7C00EEBDEDB5E7FFFDCFA29AA298EDB5E0936F
:107B8C00520EE2E4EEBDEDB5E7FFFDCFE0E0EEBD59
:107B9C00EDB5E7FFFDCFE0912109EEBDEDB5E7FFB7
:107BAC00FDCFA29A08951A93F298F398F498F59849
:107BBC00E0917E00E97FE0937E00E7E9F7E0FA933D
:107BCC00EA93E0E0EA93A8E1B0E00E9460DD10E007
:107BDC001C3008F05AC0E12FA7E9B7E0F0E0EE0F37
:107BEC00FF1FEA0FFB1F0F01ABE0B2E0EE27A10F66
:107BFC00BE1F0E9430E6E370D001E370EE0FEE0F73
:107C0C000E2EEC91E37FE029EC93E12FA7E9B7E08E
:107C1C00F0E0EE0FFF1FEA0FFB1F0F01ABE0B2E02D
:107C2C00EE27A10FBE1F0E9430E6E695E695E170A7
:107C3C00D001E170EE0F0E2EEC91ED7FE029EC936C
:107C4C00E12FA7E9B7E0F0E0EE0FFF1FAE0FBF1F6B
:107C5C00EC91F0E00E94F1E4E370F070309741F4A5
:107C6C00123011F0133011F4F49A01C0F29A0BC0D7
:107C7C00E130A0E0FA0739F4123011F0133011F4AE
:107C8C00F59A01C0F39A1F5FA3CFE89423F8EDB3E4
:107C9C00EC7FEDBBE0919707EC70EC3019F4E89AAF
:107CAC00689423F8E0919907EC70EC3019F4E99A98
:107CBC00689423F8E0919B07EC70E83031F0AFE169
:107CCC00B2E00E9430E6E37051F0E0917E00E26099
:107CDC00E0937E00E1E0E0934F08F59AF498E09190
:107CEC009D07EC70E83031F0AFE1B2E00E9430E675
:107CFC00EC7051F0E0917E00E460E0937E00E1E0F6
:107D0C00E0935008F59AF498E2E2F9E0DF01F29B77
:107D1C0002C0F39B01C002C0E1E001C0E0E0E170F1
:107D2C00EE0F0E2EEC91ED7FE029EC93E0E0E0936A
:107D3C001A09EBE1F9E0DF01F49B02C0F59B01C0ED
:107D4C0002C0E1E001C0E0E0E170E795E0E0E7951A
:107D5C000E2EEC91EF77E029EC93E0E0E09316091E
:107D6C0035C01A93E4E8F4E060E070E00E94EEE5C0
:107D7C0080E00E94E8E3249610E01C3020F5ECE84B
:107D8C00F4E060E070E00E94EEE5E12FF0E0319667
:107D9C006F2F660F660B762F0E94EEE5E12FA7E999
:107DAC00B7E0F0E0EE0FFF1FAE0FBF1FEC91E170DC
:107DBC00FF27662777270E94EEE588E00E94E8E31C
:107DCC002C961F5FDACFAAE00E94C1A619910895E4
:107DDC000E9463E43A2FE091600EE17011F03030B4
:107DEC0009F46BC2373310F03C3308F006C0E32FB4
:107DFC00F0E0F797E95AF54F3081313059F4A09102
:107E0C00680EB091690EA037E7E1BE0710F0E1E013
:107E1C0055C253C2333010F03F3008F00CC0E32F82
:107E2C00F0E03397A7E9B7E0EE0FFF1FAE0FBF1FCF
:107E3C00EC91E17043C23F3010F0363308F03CC097
:107E4C003632E8F4E32FF0E03F97AAE0B0E00E946E
:107E5C0016E5EF5CF64FE081E17079F0E32FF0E08E
:107E6C003F97AAE0B0E00E9416E5EF5CF64FE08188
:107E7C00E077E03410F4E1E001C0E0E01FC2E32F52
:107E8C00F0E0B697A7E1BAE00E94DFE4AE0FBF1FA7
:107E9C00EC91E17079F0E32FF0E0B697A7E1BAE04E
:107EAC000E94DFE4AE0FBF1FEC91E077E03410F4DA
:107EBC00E1E001C0E0E002C23C3310F0303708F0E2
:107ECC0014C0ABE6B4E0E32FF0E0FC97BD01AEE0EC
:107EDC00B0E00E9416E5DB01AE0FBF1F1C96EC91C3
:107EEC00EE1FE0E0EE1FE170E9C1303710F03438DE
:107EFC0008F011C0A6EABDE0E32FF0E0E057F04037
:107F0C000E94DDE4AE0FBF1FEC91E295EF70E69599
:107F1C00E695E170D3C1343810F0383908F00EC052
:107F2C00E32FF0E0E458F040A3E0B0E00E9416E547
:107F3C00ED5BF84FE081E695E170C0C1383910F087
:107F4C003D3908F00EC0E32FF0E0E859F040AFE700
:107F5C00B7E00E94DFE4AE0FBF1F1396EC91E17007
:107F6C00ADC13D39B9F4E091460EEF70E33079F0D4
:107F7C00E091460EEF70E43051F0E091460EEF7058
:107F8C00E13029F0E091460EEF70E63011F4E1E0BB
:107F9C0095C193C13E3969F4E091460EEF70E5301E
:107FAC0029F0E091460EEF70E23011F4E1E086C169
:107FBC0084C13F3910F0373B08F06FC0E32FEF5905
:107FCC001E2FFF2766277727E658FE4F6F4F6BBF94
:107FDC000691E12FFF2766277727EE56FE4F6F4F4E
:107FEC006BBF1691113449F5A3E00A9FF001E456DA
:107FFC00F54FE081E07FE03111F4E1E05FC1A3E0F7
:10800C000A9FF001E456F54FE081E07FE03288F002
:10801C000A9FF001E456F54FE081E770E33041F040
:10802C000A9FF001E456F54FE081E770E43009F463
:10803C0001C002C0E1E042C12FC0123401F5A3E03F
:10804C000A9FF001E456F54FE081E07FE03211F435
:10805C00E1E034C1A3E00A9FF001E456F54FE08162
:10806C00E07FE03340F00A9FF001E456F54FE081E9
:10807C00E770E43009F002C0E1E020C10DC0133418
:10808C0059F4A3E00A9FF001E456F54FE081E07F3C
:10809C00E03311F4E1E012C110C13A3B10F0363C70
:1080AC0008F009C0E32FEA5B0E2FF0E0E155F84F22
:1080BC00E081E17003C1373C10F03F3D08F0D6C0C1
:1080CC00E091BB07F0E0E130A0E0FA0709F064C0F2
:1080DC003F3C88F4E32FE75C1E2FA1E0B0E00E9448
:1080EC008BE4A091C507B0E0EA23FB23309711F095
:1080FC00E1E0E4C050C0E091BC07EF77EF3099F4B9
:10810C00363D80F4E32FEF5C1E2FA1E0B0E00E941F
:10811C008BE4A091C607B0E0EA23FB23309711F063
:10812C00E1E0CCC038C0333D88F4E32FEF5C1E2F68
:10813C00A1E0B0E00E948BE4A091C607B0E0EA2376
:10814C00FB23309711F0E1E0B9C025C03B3D88F42A
:10815C00E32FE35D1E2FA1E0B0E00E948BE4A09121
:10816C00DE07B0E0EA23FB23309711F0E1E0A6C074
:10817C0012C03F3D80F4E32FEB5D1E2FA1E0B0E079
:10818C000E948BE4A091DF07B0E0EA23FB23309739
:10819C0011F0E1E093C069C0E230A0E0FA0721F0F1
:1081AC00E330A0E0FA0789F4A2EEB7E0E32FF0E0A9
:1081BC00E75CF0400E94DFE4AE0FBF1F1296EC911B
:1081CC00E17011F0E1E07AC050C0E430A0E0FA07B1
:1081DC0009F04BC03F3C88F4E32FE75C1E2FA1E075
:1081EC00B0E00E948BE4A091C307B0E0EA23FB232C
:1081FC00309711F0E1E062C038C0333D88F4E32FD2
:10820C00EF5C1E2FA1E0B0E00E948BE4A091C607AA
:10821C00B0E0EA23FB23309711F0E1E04FC025C01A
:10822C003B3D88F4E32FE35D1E2FA1E0B0E00E94FC
:10823C008BE4A091EB07B0E0EA23FB23309711F01D
:10824C00E1E03CC012C03F3D80F4E32FEB5D1E2FFC
:10825C00A1E0B0E00E948BE4A091EE07B0E0EA232D
:10826C00FB23309711F0E1E029C027C03F3D39F4E2
:10827C00E0916B0EE07211F0E1E020C01EC0303EC8
:10828C0039F4E0916B0EE07411F0E1E017C015C009
:10829C00323059F4A5E3B1E00E9430E6A0915D0EB6
:1082AC00AE1710F0E1E00AC008C0313E31F4E091A5
:1082BC006404E87011F0E1E001C0E0E00E946AE4BF
:1082CC002496089523970E9461E4F39904C0F599CC
:1082DC0002C022FE01C003C0689422F81EC5F09BA8
:1082EC0010C0E0919707E1704E2FE0919907E17073
:1082FC00E887E0919B07E170EF83E0919D07E170C7
:10830C00EE8322FE47C0E0919707EC7009F041C064
:10831C0010919807489B02C0F19B01C027C0E091C7
:10832C009707E07111F0123008F001C012E0123022
:10833C0010F41F5F1AC01230B9F4E0919707E27085
:10834C0071F0E0919707E17021F0E0919707EE7FD3
:10835C0003C0E0919707E160E093970705C0E091B7
:10836C009707E160E09397071FE011C01B3010F0F6
:10837C0011500DC0113020F0E0919707E27009F018
:10838C0005C0E0919707EE7FE093970710E01093FC
:10839C00980743C0E0919707EC70E430F1F5109129
:1083AC009807489B12C01B3010F011500DC01130B3
:1083BC0020F0E0919707E27009F005C0E091970773
:1083CC00EE7FE093970710E026C0E0919707E071ED
:1083DC0011F0123008F001C012E0123010F41F5FDF
:1083EC0019C01230B9F4E0919707E27071F0E09186
:1083FC009707E17021F0E0919707EE7F03C0E091C1
:10840C009707E160E093970705C0E0919707E1605B
:10841C00E09397071FE01093980722FE51C0E0915C
:10842C009907EC7009F04BC010919A07499B02C058
:10843C00F19B01C031C0E0919907E07111F012304D
:10844C0008F001C012E0123010F41F5F24C0E0915C
:10845C009907E07111F0123008F001C012E01230EF
:10846C00C9F4E0919907E27081F0E0919907E1700D
:10847C0031F0A9E9B7E0EC91EE7FEC9305C0E09107
:10848C009907E160E093990705C0E0919907E160D5
:10849C00E09399071FE011C01B3010F011500DC074
:1084AC00113020F0E0919907E27009F005C0A9E9BC
:1084BC00B7E0EC91EE7FEC9310E010939A073DC07F
:1084CC00E0919907EC70E430C1F510919A07499B43
:1084DC0012C01B3010F011500DC0113020F0E09183
:1084EC009907E27009F005C0A9E9B7E0EC91EE7FBD
:1084FC00EC9310E020C0123010F41F5F1CC012303F
:10850C00C9F4E0919907E27081F0E0919907E1706C
:10851C0031F0A9E9B7E0EC91EE7FEC9305C0E09166
:10852C009907E160E093990705C0E0919907E16034
:10853C00E09399071FE010939A07E0919B07EC706A
:10854C00E830E1F5E0919108F091920834960E94A0
:10855C00EFE45E2F10919C07A9E1B2E00E9430E697
:10856C003E2FAAE1B2E00E9430E62E2F321728F5FA
:10857C00E0919B07E17089F0351768F01B3010F023
:10858C00115008C0113028F0ABE9B7E0EC91EE7F48
:10859C00EC9310E001C01FE010C0521768F01230CD
:1085AC0010F41F5F08C0123029F4E0919B07E160C2
:1085BC00E0939B071FE001C010E08CC022FE46C078
:1085CC00E0919B07EC7009F040C010919C07799BDF
:1085DC0012C01B3010F011500DC0113020F0E09182
:1085EC009B07E27009F005C0ABE9B7E0EC91EE7FB8
:1085FC00EC9310E028C0E0919B07E07111F0123071
:10860C0008F001C012E0123010F41F5F1CC01230D1
:10861C00C9F4E0919B07E27081F0E0919B07E17057
:10862C0031F0ABE9B7E0EC91EE7FEC9305C0E09153
:10863C009B07E160E0939B0705C0E0919B07E1601D
:10864C00E0939B071FE010939C0746C0E0919B07AB
:10865C00EC70E43009F040C010919C07799B29C064
:10866C00E0919B07E07111F0123008F001C012E0AC
:10867C00123010F41F5F1CC01230C9F4E0919B073C
:10868C00E27081F0E0919B07E17031F0ABE9B7E06B
:10869C00EC91EE7FEC9305C0E0919B07E160E093D9
:1086AC009B0705C0E0919B07E160E0939B071FE0EF
:1086BC0011C01B3010F011500DC0113020F0E091A2
:1086CC009B07E27009F005C0ABE9B7E0EC91EE7FD7
:1086DC00EC9310E010939C07E0919D07EC70E83050
:1086EC00E1F5E0919308F091940834960E94EFE440
:1086FC005E2F10919E07ADE1B2E00E9430E63E2F56
:10870C00AEE1B2E00E9430E62E2F321728F5E09150
:10871C009D07E17089F0351768F01B3010F011508F
:10872C0008C0113028F0ADE9B7E0EC91EE7FEC9386
:10873C0010E001C01FE010C0521768F0123010F4A6
:10874C001F5F08C0123029F4E0919D07E160E093AF
:10875C009D071FE001C010E084C022FE42C0E091E2
:10876C009D07EC70E9F510919E077A9B0FC01B30AA
:10877C0010F011500AC0E0919D07E27029F4ADE9A8
:10878C00B7E0EC91EE7FEC9310E028C0E0919D07F0
:10879C00E07111F0123008F001C012E0123010F448
:1087AC001F5F1CC01230C9F4E0919D07E27081F08C
:1087BC00E0919D07E17031F0ADE9B7E0EC91EE7F0F
:1087CC00EC9305C0E0919D07E160E0939D0705C027
:1087DC00E0919D07E160E0939D071FE010939E07D9
:1087EC0042C0E0919D07EC70E430E9F510919E07D2
:1087FC007A9B29C0E0919D07E07111F0123008F0CE
:10880C0001C012E0123010F41F5F1CC01230C9F40A
:10881C00E0919D07E27081F0E0919D07E17031F0ED
:10882C00ADE9B7E0EC91EE7FEC9305C0E0919D07CC
:10883C00E160E0939D0705C0E0919D07E160E09346
:10884C009D071FE00EC01B3010F011500AC0E091C4
:10885C009D07E27029F4ADE9B7E0EC91EE7FEC9363
:10886C0010E010939E07F09B5FC0E0919707E170BA
:10887C00E41791F0E3E9F4E060E070E00E94EEE5CB
:10888C00E0919707E170FF27662777270E94EEE5B6
:10889C0084E00E94E8E32896E0919907E170A885AE
:1088AC00EA1791F0EDE9F4E060E070E00E94EEE58B
:1088BC00E0919907E170FF27662777270E94EEE584
:1088CC0084E00E94E8E32896E0919B07E170AF8179
:1088DC00EA1791F0E7EAF4E060E070E00E94EEE560
:1088EC00E0919B07E170FF27662777270E94EEE552
:1088FC0084E00E94E8E32896E0919D07E170AE8148
:10890C00EA1791F0E1EBF4E060E070E00E94EEE534
:10891C00E0919D07E170FF27662777270E94EEE51F
:10892C0084E00E94E8E3289654E05C3008F084C1AF
:10893C00E52FA7E9B7E0F0E0EE0FFF1FAE0FBF1F6A
:10894C00EC91E1704E2F22FEA5C0E52FA7E9B7E010
:10895C00F0E0EE0FFF1FAE0FBF1FEC91EC7009F0B3
:10896C0098C0F19B02C000E011C0A7E4B8E0E52F6D
:10897C00FF2766277727EC56FF4F6F4F6BBFE691AB
:10898C00F0E0AE0FBF1FEC91E0720E2FE52FA7E9C0
:10899C00B7E0F0E0EE0FFF1FAE0FBF1F11961C915A
:1089AC00003009F44FC0E52FA7E9B7E0F0E0EE0F77
:1089BC00FF1FAE0FBF1FEC91E07111F0123008F0E9
:1089CC0001C012E0123010F41F5F3BC01230C1F531
:1089DC00E52FA7E9B7E0F0E0EE0FFF1FAE0FBF1FCA
:1089EC00EC91E27011F1E52FA7E9B7E0F0E0EE0FA2
:1089FC00FF1FAE0FBF1FEC91E17059F0E52FA7E9F7
:108A0C00B7E0F0E0EE0FFF1FAE0FBF1FEC91EE7F53
:108A1C000AC0E52FA7E9B7E0F0E0EE0FFF1FAE0F9D
:108A2C00BF1FEC91E160EC930BC0E52FA7E9B7E019
:108A3C00F0E0EE0FFF1FAE0FBF1FEC91E160EC9367
:108A4C001FE01EC01B3010F011501AC0113058F02E
:108A5C00E52FA7E9B7E0F0E0EE0FFF1FAE0FBF1F49
:108A6C00EC91E27009F00BC0E52FA7E9B7E0F0E05C
:108A7C00EE0FFF1FAE0FBF1FEC91EE7FEC9310E0DB
:108A8C00E52FA7E9B7E0F0E0EE0FFF1FEA0FFB1FA1
:108A9C001183A0C0E52FA7E9B7E0F0E0EE0FFF1FB0
:108AAC00AE0FBF1FEC91EC70E43009F093C0A7E45B
:108ABC00B8E0E52FFF2766277727EC56FF4F6F4F5F
:108ACC006BBFE691F0E0AE0FBF1FEC91E0720E2F82
:108ADC00E52FA7E9B7E0F0E0EE0FFF1FAE0FBF1FC9
:108AEC0011961C910030F9F01B3010F011501AC087
:108AFC00113058F0E52FA7E9B7E0F0E0EE0FFF1FBB
:108B0C00AE0FBF1FEC91E27009F00BC0E52FA7E987
:108B1C00B7E0F0E0EE0FFF1FAE0FBF1FEC91EE7F42
:108B2C00EC9310E04EC0E52FA7E9B7E0F0E0EE0FB4
:108B3C00FF1FAE0FBF1FEC91E07111F0123008F067
:108B4C0001C012E0123010F41F5F3BC01230C1F5AF
:108B5C00E52FA7E9B7E0F0E0EE0FFF1FAE0FBF1F48
:108B6C00EC91E27011F1E52FA7E9B7E0F0E0EE0F20
:108B7C00FF1FAE0FBF1FEC91E17059F0E52FA7E975
:108B8C00B7E0F0E0EE0FFF1FAE0FBF1FEC91EE7FD2
:108B9C000AC0E52FA7E9B7E0F0E0EE0FFF1FAE0F1C
:108BAC00BF1FEC91E160EC930BC0E52FA7E9B7E098
:108BBC00F0E0EE0FFF1FAE0FBF1FEC91E160EC93E6
:108BCC001FE0E52FA7E9B7E0F0E0EE0FFF1FEA0F7B
:108BDC00FB1F1183F09B2EC0E52FA7E9B7E0F0E057
:108BEC00EE0FFF1FAE0FBF1FEC91E170E41711F1F8
:108BFC00EBEBF4E060E070E00E94EEE5E52FF0E0D6
:108C0C0031966F2F660F660B762F0E94EEE5E52FDF
:108C1C00A7E9B7E0F0E0EE0FFF1FAE0FBF1FEC911E
:108C2C00E170FF27662777270E94EEE588E00E9417
:108C3C00E8E32C965F5F79CEF39B06C0F29904C0F3
:108C4C00F59B02C0F49B01C002C0E89414C0F399D8
:108C5C0006C0F29B04C0F59902C0F49901C002C091
:108C6C00689409C0A0E022FCA1E0E1E0EA27E894C6
:108C7C00EE2309F0689422F8F39B02C0F29901C02C
:108C8C0021C0A2E2B9E0E0E022FCE1E0E170EE0FED
:108C9C000E2EEC91ED7FE029EC93A298EDB5E093CC
:108CAC00520EE2E4EEBDEDB5E7FFFDCFEAE0EEBD1E
:108CBC00EDB5E7FFFDCFE0912209EEBDEDB5E7FF85
:108CCC00FDCFA29AF59B02C0F49901C026C0E3E641
:108CDC00E0931609ABE1B9E0E0E022FCE1E0E170E1
:108CEC00E795E0E0E7950E2EEC91EF77E029EC9319
:108CFC002898EDB5E093520EE0E4EEBDEDB5E7FF3C
:108D0C00FDCFEAE0EEBDEDB5E7FFFDCFE0911B092D
:108D1C00EEBDEDB5E7FFFDCF289A0E9468E42996D9
:108D2C00089524970E9461E423FE93C0A0918D0EB8
:108D3C00A13030F0E0918D0EE150E0938D0E89C0A2
:108D4C00E2E0E0938D0EF894E091890EF0918A0E9A
:108D5C00E0939307F0939407E0E0E093890EE0939F
:108D6C008A0EE0918B0EF0918C0EE0939507F093A8
:108D7C009607E0E0E0938B0EE0938C0E7894E091F4
:108D8C009707EC70EC3051F5A0919307B0919407D4
:108D9C0088279927E9E00E94ADE4DF01CB01EDE9DA
:108DAC00F0E060E070E00E9474E5E0939307F093CC
:108DBC009407AEECB9E00E942CE6A0919307B09119
:108DCC009407AE17BF0720F0E0919707E16003C04E
:108DDC00E0919707EE7FE093970705C0E0E0E09302
:108DEC009307E0939407E0919907EC70EC3061F5F0
:108DFC00A0919507B091960788279927E9E00E94E2
:108E0C00ADE4DF01CB01EDE9F0E060E070E00E9441
:108E1C0074E5E0939507F0939607A0EDB9E00E94F6
:108E2C002CE6A0919507B0919607AE17BF0730F0CE
:108E3C00E0919907E160E093990705C0A9E9B7E0D3
:108E4C00EC91EE7FEC9305C0E0E0E0939507E093A6
:108E5C009607AFE1B2E00E9430E6E3703E2F30306F
:108E6C0009F4B9C0A0E2B2E00E9430E62E2FA1E2D4
:108E7C00B2E00E9430E65E2F313029F4E091910887
:108E8C00F091920804C0E0919308F0919408349604
:108E9C000E94F1E4E887F98710E0163008F09BC0D7
:108EAC00A2E2B2E0EE27A10FBE1F0E9430E60E2F09
:108EBC00013008F48EC0F0E0EE83FF83EE0FFF1F4D
:108ECC00EE83FF83E12FF0E0E155F84FE081E17094
:108EDC0009F443C0E22FF0E0A885B985AE0FBF1F9F
:108EEC00EE27A50FBE1FEE81FF81AE17BF0778F0EE
:108EFC00E22FF0E0AE81BF81AE0FBF1FE52FF0E097
:108F0C00EA0FFB1FA885B985EA17FB0728F5F09B2C
:108F1C001CC0E6ECF4E060E070E00E94EEE5E12FAE
:108F2C00F0E031966F2F660F660B762F0E94EEE500
:108F3C00A889B989EAE00E943EE5662777270E9456
:108F4C00EEE588E00E94E8E32C96A12FB0E0A15555
:108F5C00B84FEC91EE7FEC933CC0E22FF0E0A8858B
:108F6C00B985AE0FBF1FEE81FF81AE17BF0758F05A
:108F7C00E22FF0E0AE81BF81EA0FFB1FA885B98517
:108F8C00EA17FB0708F425C0F09B1CC0EAEDF4E0DF
:108F9C0060E070E00E94EEE5E12FF0E031966F2F7B
:108FAC00660F660B762F0E94EEE5A889B989EAE078
:108FBC000E943EE5662777270E94EEE588E00E9436
:108FCC00E8E32C96A12FB0E0A155B84FEC91E160ED
:108FDC00EC931F5F62CFAFE1B2E00E9430E6E69502
:108FEC00E695E3703E2F303009F4B9C0A0E2B2E050
:108FFC000E9430E62E2FA1E2B2E00E9430E65E2FF6
:10900C00313029F4E0919108F091920804C0E0917C
:10901C009308F091940834960E94F1E4E887F9875C
:10902C0016E01C3008F09BC0A2E2B2E0EE27A10FC4
:10903C00BE1F0E9430E60E2F013008F48EC0F0E007
:10904C00EE83FF83EE0FFF1FEE83FF83E12FF0E033
:10905C00E155F84FE081E17009F443C0E22FF0E0F4
:10906C00A885B985AE0FBF1FEE27A50FBE1FEE81D9
:10907C00FF81AE17BF0778F0E22FF0E0AE81BF8121
:10908C00AE0FBF1FE52FF0E0EA0FFB1FA885B985D7
:10909C00EA17FB0728F5F09B1CC0E6ECF4E060E057
:1090AC0070E00E94EEE5E12FF0E031966F2F660F35
:1090BC00660B762F0E94EEE5A889B989EAE00E943A
:1090CC003EE5662777270E94EEE588E00E94E8E3FC
:1090DC002C96A12FB0E0A155B84FEC91EE7FEC93FC
:1090EC003CC0E22FF0E0A885B985AE0FBF1FEE8122
:1090FC00FF81AE17BF0758F0E22FF0E0AE81BF81C1
:10910C00EA0FFB1FA885B985EA17FB0708F425C0F1
:10911C00F09B1CC0EAEDF4E060E070E00E94EEE52C
:10912C00E12FF0E031966F2F660F660B762F0E94C1
:10913C00EEE5A889B989EAE00E943EE56627772723
:10914C000E94EEE588E00E94E8E32C96A12FB0E0A7
:10915C00A155B84FEC91E160EC931F5F62CF0E9478
:10916C0068E42A96089560971A93FE013196FA9353
:10917C00EA93E0E0EA93A0E1B0E00E9460DD10E049
:10918C001C3008F03FC0ABE0B2E0EE27A10FBE1FD1
:10919C000E9430E6EC7F0E944CE6ABE0B2E0EE279A
:1091AC00A10FBE1F0E9430E6EB7F0E944CE6FE0131
:1091BC003196FA93EA93EDEEF4E060E070E00E94F1
:1091CC00EEE5E12FF0E031966F2F660F660B762FF0
:1091DC000E94EEE584E00E94ADE32A96E12FF0E0D8
:1091EC00A0EDBAE30E94DBE4EA0FFB1FFA93EA93CB
:1091FC00FE013396FA93EA93A0E10E94312DA895D3
:10920C001F5FBECFA7E1B2E0E0E00E944CE6A8E110
:10921C00B2E0EAEF0E944CE6A9E1B2E0E4E60E947B
:10922C004CE6AAE1B2E0E6E90E944CE6ABE1B2E022
:10923C00E0E00E944CE6ACE1B2E0EAEF0E944CE6C2
:10924C00ADE1B2E0E4E60E944CE6AEE1B2E0E6E964
:10925C000E944CE6AFE1B2E00E9430E6EC7F0E9447
:10926C004CE6AFE1B2E00E9430E6E37F0E944CE6B0
:10927C00AFE1B2E00E9430E6EF700E944CE6A0E253
:10928C00B2E0E8E10E944CE6A1E2B2E0E2E00E942A
:10929C004CE6E2E2F2E0FA93EA93ACE00E949B2AFD
:1092AC0010E0163008F054C0FE013196FA93EA93A0
:1092BC00E7EFF4E060E070E00E94EEE5E12FF0E013
:1092CC0031966F2F660F660B762F0E94EEE584E0C9
:1092DC000E94ADE32A96E12FF0E0A0E4B5E40E94F1
:1092EC00DBE4EA0FFB1FFA93EA93FE013396FA9341
:1092FC00EA93A0E10E94312DFE013196FA93EA9394
:10930C00E3E0F5E060E070E00E94EEE5E12FF0E0D4
:10931C0031966F2F660F660B762F0E94EEE584E078
:10932C000E94ADE32A96E12FF0E03696A0E4B5E476
:10933C000E94DBE4EA0FFB1FFA93EA93FE013396DB
:10934C00FA93EA93A0E10E94312DA8951F5FA9CF53
:10935C00188161960895AA93BA93EA93FA93EFB79A
:10936C00EA93A9E8BEE008C0AA93BA93EA93FA93E9
:10937C00EFB7EA93ABE8BEE0ED91FD913196FE9329
:10938C00EE93E991EFBFF991E991B991A9911895F3
:10939C000E9461E4EBEBF7E0FA93EA93E0E0EA93E6
:1093AC00A7E8B0E00E9460DDA8E3B1E00E9430E6DF
:1093BC00E093BB07E0E1F5E060E070E00E94EEE5D1
:1093CC0080E00E94E8E32496E091BB07F0E0E130F6
:1093DC00A0E0FA0709F028C100E0023008F007C14C
:1093EC00AAE7B8E0E02FF0E0BD01A1E7B0E00E94F1
:1093FC0016E5DB01AE0FBF1F0E9430E6E03009F42A
:10940C00F4C0ACEBB7E0E02FF0E0BD01A9E1B0E0B7
:10941C000E9416E5E60FF71FFF93EF93AAE7B8E05B
:10942C00E02FF0E0BD01A1E7B0E00E9416E5DB0102
:10943C00AE0FBF1F11960E9430E6E295EF70AF9110
:10944C00BF91EF770E2EEC91E078E029EC93ACEB2A
:10945C00B7E0E02FF0E0BD01A9E1B0E00E9416E515
:10946C00DB01AE0FBF1F1296E5E0EC9331E0E0E0BC
:10947C001E2F5E2F2E2F183008F040C0AAE7B8E040
:10948C00E02FF0E0BD01A1E7B0E00E9416E5DB01A2
:10949C00AE0FBF1F1E96E12FF0E00E94DDE4AE0F71
:1094AC00BF1F16960E9430E6F0E0F695E795E37044
:1094BC00F070E130A0E0FA0721F0E330A0E0FA0709
:1094CC0009F4232BAAE7B8E0E02FF0E0BD01A1E7F7
:1094DC00B0E00E9416E5DB01AE0FBF1F1E96E12F18
:1094EC00F0E00E94DDE4AE0FBF1F16960E9430E63E
:1094FC00E17009F0532B1F5F330FBDCFACEBB7E01E
:10950C00E02FF0E0BD01A9E1B0E00E9416E5E60F06
:10951C00F71F2187ACEBB7E0E02FF0E0BD01A9E12C
:10952C00B0E00E9416E5E60FF71F558331E0E0E04E
:10953C005E2F2E2F1C3008F040C0AAE7B8E0E02FB9
:10954C00F0E0BD01A1E7B0E00E9416E5DB01AE0F33
:10955C00BF1F1E96E12FF0E00E94DDE4AE0FBF1F8F
:10956C0016960E9430E6F0E0F695E795E370F07001
:10957C00E130A0E0FA0721F0E330A0E0FA0709F4AB
:10958C00232BAAE7B8E0E02FF0E0BD01A1E7B0E0A3
:10959C000E9416E5DB01AE0FBF1F1E96E12FF0E017
:1095AC000E94DDE4AE0FBF1F16960E9430E6E170FC
:1095BC0009F0532B1F5F330FBDCFACEBB7E0E02F9F
:1095CC00F0E0BD01A9E1B0E00E9416E5E60FF71F3F
:1095DC002287ACEBB7E0E02FF0E0BD01A9E1B0E0F1
:1095EC000E9416E5E60FF71F56830F5FF6CEE8E1F3
:1095FC00F5E060E070E00E94EEE5AAE7B8E00E94BA
:10960C0030E6FF27662777270E94EEE5ABEEB8E041
:10961C000E9430E6FF27662777270E94EEE588E058
:10962C000E94E8E32C963DC0E230A0E0FA0769F412
:10963C00E9E2F5E060E070E00E94EEE580E00E9477
:10964C00E8E324960E94A2592CC0E330A0E0FA076C
:10965C0069F4EBE3F5E060E070E00E94EEE580E099
:10966C000E94E8E324960E94A2591BC0E430A0E0BB
:10967C00FA0769F4EBE4F5E060E070E00E94EEE5D7
:10968C0080E00E94E8E324960E9402620AC0E3E5AF
:10969C00F5E060E070E00E94EEE580E00E94E8E317
:1096AC0024960E9468E426960895E0E0E093BB07B8
:1096BC00A8E3B1E00E944CE60895BA93AA932597CB
:1096CC000E9461E4AB85BC85EC91E07109F0E2C1CC
:1096DC00EB85FC85A181EFE7EA235E2F503009F47E
:1096EC00D9C130E0323008F0D5C1AAE7B8E0E32F99
:1096FC00F0E0BD01A1E7B0E00E9416E5DB01AE0F82
:10970C00BF1F0E9430E65E1709F0C2C1ACEBB7E098
:10971C00E32FF0E0BD01A9E1B0E00E9416E5DB010A
:10972C00AE0FBF1F1296EAE0EC93EB85FC85A1818E
:10973C00B281E7E00E949CE4EE83F0E0EE30A0E022
:10974C00FA0709F4A5C1E330A0E0FA0709F0A0C1BB
:10975C00ACEBB7E0E32FF0E0BD01A9E1B0E00E9473
:10976C0016E5DB01AE0FBF1FEC91E07889F5ACEB91
:10977C00B7E0E32FF0E0BD01A9E1B0E00E9416E5EF
:10978C00DB01AE0FBF1FEC91E068EC93ACEBB7E0E4
:10979C00E32FF0E0BD01A9E1B0E00E9416E5DB018A
:1097AC00AE0FBF1F1196E0E0EC93EAE5F5E060E048
:1097BC0070E00E94EEE5E32FF0E031966F2F660F1C
:1097CC00660B762F0E94EEE584E00E94E8E3289673
:1097DC00ACEBB7E0E32FF0E0BD01A9E1B0E00E94F3
:1097EC0016E5DB01AE0FBF1F1296E1E1EC93ACEB7B
:1097FC00B7E0E32FF0E0BD01A9E1B0E00E9416E56F
:10980C00DB01AE0FBF1FEC91EF772E2FACEBB7E067
:10981C00E32FF0E0BD01A9E1B0E00E9416E5DB0109
:10982C00AE0FBF1F1996EC91E987ACEBB7E0E32FB5
:10983C00F0E0BD01A9E1B0E00E9416E5DB01AE0F3E
:10984C00BF1F1796EC91E887ACEBB7E0E32FF0E085
:10985C00BD01A9E1B0E00E9416E5DB01AE0FBF1F10
:10986C001596EC91EF83EB85FC854581022F093031
:10987C0008F008E010E0E1E0EA87101758F5EA85F7
:10988C00AF81EA23B1F0EA85E42369F0EA85A88583
:10989C00EA2341F4EA85A985EA27E987EA85A885C0
:1098AC00EA2BE88705C0EA85E095A885EA23E887D6
:1098BC000CC0EA85E42321F0EA85A985EA2B04C0D3
:1098CC00EA85E095A985EA23E9871F5FEA85EE0F13
:1098DC00EA87D3CFACEBB7E0E32FF0E0BD01A9E111
:1098EC00B0E00E9416E5DB01AE0FBF1F1996AC91DC
:1098FC00E985EA17E9F0ACEBB7E0E32FF0E0BD0146
:10990C00A9E1B0E00E9416E5E60FF71F3996A9858C
:10991C00A083ACEBB7E0E32FF0E0BD01A9E1B0E030
:10992C000E9416E5DB01AE0FBF1F1396E0E0EC932F
:10993C00ACEBB7E0E32FF0E0BD01A9E1B0E00E9491
:10994C0016E5E60FF71F3796A885A083293008F493
:10995C009FC0ACEBB7E0E32FF0E0BD01A9E1B0E0B4
:10996C000E9416E5DB01AE0FBF1F1A96EC91E9873A
:10997C00ACEBB7E0E32FF0E0BD01A9E1B0E00E9451
:10998C0016E5DB01AE0FBF1F1896EC91E887ACEB28
:10999C00B7E0E32FF0E0BD01A9E1B0E00E9416E5CD
:1099AC00DB01AE0FBF1F1696EC91EF83EB85FC85A8
:1099BC004681E22FE8500E2F10E0E1E0EA87101705
:1099CC0058F5EA85AF81EA23B1F0EA85E42369F022
:1099DC00EA85A885EA2341F4EA85A985EA27E9877F
:1099EC00EA85A885EA2BE88705C0EA85E095A88575
:1099FC00EA23E8870CC0EA85E42321F0EA85A985EF
:109A0C00EA2B04C0EA85E095A985EA23E9871F5F64
:109A1C00EA85EE0FEA87D3CFACEBB7E0E32FF0E0AB
:109A2C00BD01A9E1B0E00E9416E5DB01AE0FBF1F3E
:109A3C001A96AC91E985EA17E9F0ACEBB7E0E32FA5
:109A4C00F0E0BD01A9E1B0E00E9416E5E60FF71FBA
:109A5C003A96A985A083ACEBB7E0E32FF0E0BD010B
:109A6C00A9E1B0E00E9416E5DB01AE0FBF1F139613
:109A7C00E0E0EC93ACEBB7E0E32FF0E0BD01A9E143
:109A8C00B0E00E9416E5E60FF71F3896A885A08374
:109A9C003F5F28CE0E9468E42D9608956F970E9430
:109AAC0061E4E0916304E07421F40E9468E4A596FB
:109ABC00089540E0423010F00C94EA57ACEBB7E05C
:109ACC00E42FF0E0BD01A9E1B0E00E9416E5DB0156
:109ADC00AE0FBF1F1296AC91A13010F40C94E75747
:109AEC00ACEBB7E0E42FF0E0BD01A9E1B0E00E94DF
:109AFC0016E5DB01AE0FBF1FEC91EF775E2FACEBE1
:109B0C00B7E0E42FF0E0BD01A9E1B0E00E9416E55A
:109B1C00DB01AE0FBF1F1396AC91A13088F0ACEBFC
:109B2C00B7E0E42FF0E0BD01A9E1B0E00E9416E53A
:109B3C00DB01AE0FBF1F1396EC91E1500C94D05586
:109B4C00ACEBB7E0E42FF0E0BD01A9E1B0E00E947E
:109B5C0016E5DB01AE0FBF1F1396E4E0EC93FE019C
:109B6C003C96FA93EA93E0E0EA93A6E0B0E00E9418
:109B7C0060DDFE013696FA93EA93E0E0EA93A6E004
:109B8C00B0E00E9460DD20E0E1E0EE8BE0E1ED8BE7
:109B9C00251708F086C700E030E0AAE7B8E0E42F0C
:109BAC00F0E0BD01A1E7B0E00E9416E5DB01AE0FCD
:109BBC00BF1F1E96E22FF0E00E94DDE4AE0FBF1F28
:109BCC0015960E9430E61E2FA12F0E943A8D3E2F33
:109BDC003030E9F4AAE7B8E0E42FF0E0BD01A1E7EA
:109BEC00B0E00E9416E5DB01AE0FBF1F1E96E22F00
:109BFC00F0E00E94DDE4AE0FBF1F14960E9430E629
:109C0C001E2F103021F0A12F0E943A8D3E2F3030A4
:109C1C00E9F4AAE7B8E0E42FF0E0BD01A1E7B0E079
:109C2C000E9416E5DB01AE0FBF1F1E96E22FF0E07F
:109C3C000E94DDE4AE0FBF1F13960E9430E61E2F6C
:109C4C00103021F0A12F0E943A8D3E2F303011F0B0
:109C5C00353009F4A1C0E32FF0E0E130A0E0FA07C1
:109C6C0029F5AAE7B8E0E42FF0E0BD01A1E7B0E0E8
:109C7C000E9416E5DB01AE0FBF1F1C960E9430E65A
:109C8C00E295E7700E2FAAE7B8E0E42FF0E0BD01F3
:109C9C00A1E7B0E00E9416E5DB01AE0FBF1F1C96DA
:109CAC000E9430E6EE1FE0E0EE1F73C0E230A0E051
:109CBC00FA07F9F4AAE7B8E0E42FF0E0BD01A1E758
:109CCC00B0E00E9416E5DB01AE0FBF1F1C960E9490
:109CDC0030E6E7700E2FAAE7B8E0E42FF0E0BD0104
:109CEC00A1E7B0E00E9416E5DB01AE0FBF1F1C968A
:109CFC004BC0E330A0E0FA0729F5AAE7B8E0E42F5F
:109D0C00F0E0BD01A1E7B0E00E9416E5DB01AE0F6B
:109D1C00BF1F1B960E9430E6E295E7700E2FAAE754
:109D2C00B8E0E42FF0E0BD01A1E7B0E00E9416E539
:109D3C00DB01AE0FBF1F1B960E9430E6EE1FE0E06A
:109D4C00EE1F27C0E430A0E0FA0729F5AAE7B8E037
:109D5C00E42FF0E0BD01A1E7B0E00E9416E5DB01C5
:109D6C00AE0FBF1F1B960E9430E6E7700E2FAAE7BE
:109D7C00B8E0E42FF0E0BD01A1E7B0E00E9416E5E9
:109D8C00DB01AE0FBF1F1B960E9430E6E695E695F1
:109D9C00E695E170EF8BF0C0AAE7B8E0E42FF0E0B5
:109DAC00BD01A1E7B0E00E9416E5DB01AE0FBF1FBD
:109DBC001E96E22FF0E00E94DDE4AE0FBF1F12965C
:109DCC000E9430E61E2F103029F0A12F0E94EE3E8B
:109DDC00E03009F42EC0AAE7B8E0E42FF0E0BD01B2
:109DEC00A1E7B0E00E9416E5DB01AE0FBF1F1E9687
:109DFC00E22FF0E00E94DDE4AE0FBF1F17960E9429
:109E0C0030E6E295E7700E2FAAE7B8E0E42FF0E019
:109E1C00BD01A1E7B0E00E9416E5DB01AE0FBF1F4C
:109E2C001E96E22FF0E00E94DDE4AE0FBF1F1796E6
:109E3C009CC0AAE7B8E0E42FF0E0BD01A1E7B0E0D8
:109E4C000E9416E5DB01AE0FBF1F1E96E22FF0E05D
:109E5C000E94DDE4AE0FBF1F11960E9430E61E2F4C
:109E6C00103029F0A12F0E94EE3EE03009F432C0F0
:109E7C00AAE7B8E0E42FF0E0BD01A1E7B0E00E9452
:109E8C0016E5DB01AE0FBF1F1E96E22FF0E00E941D
:109E9C00DDE4AE0FBF1F17960E9430E6E7700E2F61
:109EAC00AAE7B8E0E42FF0E0BD01A1E7B0E00E9422
:109EBC0016E5DB01AE0FBF1F1E96E22FF0E00E94ED
:109ECC00DDE4AE0FBF1F17960E9430E6E695E695CF
:109EDC00E69550C0AAE7B8E0E42FF0E0BD01A1E799
:109EEC00B0E00E9416E5DB01AE0FBF1F1E96E22FFD
:109EFC00F0E00E94DDE4AE0FBF1F0E9430E61E2F83
:109F0C00103029F0A12F0E94EE3EE03009F434C04D
:109F1C00AAE7B8E0E42FF0E0BD01A1E7B0E00E94B1
:109F2C0016E5DB01AE0FBF1F1E96E22FF0E00E947C
:109F3C00DDE4AE0FBF1F16960E9430E6E295E77087
:109F4C000E2FAAE7B8E0E42FF0E0BD01A1E7B0E0E6
:109F5C000E9416E5DB01AE0FBF1F1E96E22FF0E04C
:109F6C000E94DDE4AE0FBF1F16960E9430E6EE1F76
:109F7C00E0E0EE1FE170EF8B003011F4353009F0AA
:109F8C0025C0AAE7B8E0E42FF0E0BD01A1E7B0E0FE
:109F9C000E9416E5DB01AE0FBF1F1D960E9430E636
:109FAC00E7700E2FAAE7B8E0E42FF0E0BD01A1E7BF
:109FBC00B0E00E9416E5DB01AE0FBF1F1D960E949C
:109FCC0030E6E695E695E695E170EF8BEF89E030AB
:109FDC0009F4ABC2593008F047C0E02FF0E0E13093
:109FEC00A0E0FA0729F4EE89AE81EA2BEE833BC0A0
:109FFC00E230A0E0FA0719F4FE0137962EC0E330E8
:10A00C00A0E0FA0741F1E430A0E0FA0739F4EE8958
:10A01C00AE81EA2BEE83FE0137961FC0E530A0E03F
:10A02C00FA0789F0E630A0E0FA0729F4EE89AE8150
:10A03C00EA2BEE8310C0E730A0E0FA07A1F4EE891A
:10A04C00AE81EA2BEE83FE0137960F01E081AE89DB
:10A05C00EA2BD001EC93FE0138960F01E081AE891A
:10A06C00EA2BD001EC9360C25A3009F0C9C0E02F42
:10A07C00F0E0E130A0E0FA0781F4283028F4EE8912
:10A08C00AE81EA2BEE8308C0FE0137960F01E0810A
:10A09C00AE89EA2BD001EC93B2C0E230A0E0FA0713
:10A0AC0071F4283018F4FE01389602C0FE0139967E
:10A0BC000F01E081AE89EA2BD001EC93A0C0E33014
:10A0CC00A0E0FA0771F4283018F4FE013A9602C0A9
:10A0DC00FE013B960F01E081AE89EA2BD001EC9397
:10A0EC008EC0E430A0E0FA07E9F4283028F4EE89B9
:10A0FC00AE81EA2BEE8308C0FE0137960F01E0819A
:10A10C00AE89EA2BD001EC93283018F4FE01389676
:10A11C0002C0FE0139960F01E081AE89EA2BD00115
:10A12C00EC936DC0E530A0E0FA07D9F4283018F4B0
:10A13C00FE01389602C0FE0139960F01E081AE890E
:10A14C00EA2BD001EC93283018F4FE013A9602C0A9
:10A15C00FE013B960F01E081AE89EA2BD001EC9316
:10A16C004EC0E630A0E0FA07E9F4283028F4EE8976
:10A17C00AE81EA2BEE8308C0FE0137960F01E08119
:10A18C00AE89EA2BD001EC93283018F4FE013A96F4
:10A19C0002C0FE013B960F01E081AE89EA2BD00193
:10A1AC00EC932DC0E730A0E0FA0749F5283018F4FD
:10A1BC00FE01389602C0FE0139960F01E081AE898E
:10A1CC00EA2BD001EC93283028F4EE89AE81EA2BEF
:10A1DC00EE8308C0FE0137960F01E081AE89EA2BB1
:10A1EC00D001EC93283018F4FE013A9602C0FE011F
:10A1FC003B960F01E081AE89EA2BD001EC9394C120
:10A20C005C3009F0C9C0E02FF0E0E130A0E0FA07C3
:10A21C0081F4283028F4EE89AE81EA2BEE8308C055
:10A22C00FE0137960F01E081AE89EA2BD001EC9349
:10A23C00B2C0E230A0E0FA0771F4243018F4FE0149
:10A24C00379602C0FE0138960F01E081AD89EA2BEA
:10A25C00D001EC93A0C0E330A0E0FA0771F42830F1
:10A26C0018F4FE01399602C0FE013A960F01E08106
:10A27C00AE89EA2BD001EC938EC0E430A0E0FA0753
:10A28C00E9F4283028F4EE89AE81EA2BEE8308C07D
:10A29C00FE0137960F01E081AE89EA2BD001EC93D9
:10A2AC00243018F4FE01379602C0FE0138960F01D7
:10A2BC00E081AD89EA2BD001EC936DC0E530A0E0D4
:10A2CC00FA07D9F4243018F4FE01379602C0FE01C7
:10A2DC0038960F01E081AD89EA2BD001EC93283040
:10A2EC0018F4FE01399602C0FE013A960F01E08186
:10A2FC00AE89EA2BD001EC934EC0E630A0E0FA0711
:10A30C00E9F4283028F4EE89AE81EA2BEE8308C0FC
:10A31C00FE0137960F01E081AE89EA2BD001EC9358
:10A32C00283018F4FE01399602C0FE013A960F014E
:10A33C00E081AE89EA2BD001EC932DC0E730A0E090
:10A34C00FA0749F5283028F4EE89AE81EA2BEE8322
:10A35C0008C0FE0137960F01E081AE89EA2BD001CF
:10A36C00EC93243018F4FE01379602C0FE013896A7
:10A37C000F01E081AD89EA2BD001EC93283018F461
:10A38C00FE01399602C0FE013A960F01E081AE89BA
:10A39C00EA2BD001EC93C8C0E02FF0E0E130A0E054
:10A3AC00FA0781F4283028F4EE89AE81EA2BEE838B
:10A3BC0008C0FE0137960F01E081AE89EA2BD0016F
:10A3CC00EC93B2C0E230A0E0FA0771F4283018F434
:10A3DC00FE01389602C0FE0139960F01E081AD896D
:10A3EC00EA2BD001EC93A0C0E330A0E0FA0771F4A3
:10A3FC00283018F4FE013A9602C0FE013B960F017C
:10A40C00E081AE89EA2BD001EC938EC0E430A0E061
:10A41C00FA07E9F4283028F4EE89AE81EA2BEE83B2
:10A42C0008C0FE0137960F01E081AE89EA2BD001FE
:10A43C00EC93283018F4FE01389602C0FE013996D0
:10A44C000F01E081AD89EA2BD001EC936DC0E530B2
:10A45C00A0E0FA07D9F4283018F4FE01389602C0AF
:10A46C00FE0139960F01E081AD89EA2BD001EC9306
:10A47C00283018F4FE013A9602C0FE013B960F01FB
:10A48C00E081AE89EA2BD001EC934EC0E630A0E01F
:10A49C00FA07E9F4283028F4EE89AE81EA2BEE8332
:10A4AC0008C0FE0137960F01E081AE89EA2BD0017E
:10A4BC00EC93283018F4FE013A9602C0FE013B964C
:10A4CC000F01E081AE89EA2BD001EC932DC0E7306F
:10A4DC00A0E0FA0749F5283028F4EE89AE81EA2B82
:10A4EC00EE8308C0FE0137960F01E081AE89EA2B9E
:10A4FC00D001EC93283018F4FE01389602C0FE010E
:10A50C0039960F01E081AD89EA2BD001EC9328300C
:10A51C0018F4FE013A9602C0FE013B960F01E08151
:10A52C00AE89EA2BD001EC93AAC2593008F047C08F
:10A53C00E02FF0E0E130A0E0FA0729F4EE89AC85D9
:10A54C00EA2BEC873BC0E230A0E0FA0719F4FE01DD
:10A55C003D962EC0E330A0E0FA0741F1E430A0E0D4
:10A56C00FA0739F4EE89AC85EA2BEC87FE013D96AF
:10A57C001FC0E530A0E0FA0789F0E630A0E0FA074A
:10A58C0029F4EE89AC85EA2BEC8710C0E730A0E00B
:10A59C00FA07A1F4EE89AC85EA2BEC87FE013D9617
:10A5AC000F01E081AE89EA2BD001EC93FE013E96BF
:10A5BC000F01E081AE89EA2BD001EC9360C25A30D6
:10A5CC0009F0C9C0E02FF0E0E130A0E0FA0781F417
:10A5DC00283028F4EE89AC85EA2BEC8708C0FE0104
:10A5EC003D960F01E081AE89EA2BD001EC93B2C00D
:10A5FC00E230A0E0FA0771F4283018F4FE013E9620
:10A60C0002C0FE013F960F01E081AE89EA2BD0011A
:10A61C00EC93A0C0E330A0E0FA0771F4283018F4F2
:10A62C00FE01709602C0FE0171960F01E081AE89A9
:10A63C00EA2BD001EC938EC0E430A0E0FA07E9F4E9
:10A64C00283028F4EE89AC85EA2BEC8708C0FE0193
:10A65C003D960F01E081AE89EA2BD001EC932830B6
:10A66C0018F4FE013E9602C0FE013F960F01E081F8
:10A67C00AE89EA2BD001EC936DC0E530A0E0FA076F
:10A68C00D9F4283018F4FE013E9602C0FE013F9624
:10A69C000F01E081AE89EA2BD001EC93283018F43D
:10A6AC00FE01709602C0FE0171960F01E081AE8929
:10A6BC00EA2BD001EC934EC0E630A0E0FA07E9F4A7
:10A6CC00283028F4EE89AC85EA2BEC8708C0FE0113
:10A6DC003D960F01E081AE89EA2BD001EC93283036
:10A6EC0018F4FE01709602C0FE0171960F01E08114
:10A6FC00AE89EA2BD001EC932DC0E730A0E0FA072D
:10A70C0049F5283018F4FE013E9602C0FE013F9632
:10A71C000F01E081AE89EA2BD001EC93283028F4AC
:10A72C00EE89AC85EA2BEC8708C0FE013D960F0143
:10A73C00E081AE89EA2BD001EC93283018F4FE01AD
:10A74C00709602C0FE0171960F01E081AE89EA2B72
:10A75C00D001EC9394C15C3009F0C9C0E02FF0E05B
:10A76C00E130A0E0FA0781F4283028F4EE89AC85BA
:10A77C00EA2BEC8708C0FE013D960F01E081AE8903
:10A78C00EA2BD001EC93B2C0E230A0E0FA0771F4EE
:10A79C00243018F4FE013D9602C0FE013E960F01D6
:10A7AC00E081AD89EA2BD001EC93A0C0E330A0E0AE
:10A7BC00FA0771F4283018F4FE013F9602C0FE012E
:10A7CC0070960F01E081AE89EA2BD001EC938EC01C
:10A7DC00E430A0E0FA07E9F4283028F4EE89AC85DF
:10A7EC00EA2BEC8708C0FE013D960F01E081AE8993
:10A7FC00EA2BD001EC93243018F4FE013D9602C0F4
:10A80C00FE013E960F01E081AD89EA2BD001EC935D
:10A81C006DC0E530A0E0FA07D9F4243018F4FE013D
:10A82C003D9602C0FE013E960F01E081AD89EA2BF8
:10A83C00D001EC93283018F4FE013F9602C0FE01C3
:10A84C0070960F01E081AE89EA2BD001EC934EC0DB
:10A85C00E630A0E0FA07E9F4283028F4EE89AC855C
:10A86C00EA2BEC8708C0FE013D960F01E081AE8912
:10A87C00EA2BD001EC93283018F4FE013F9602C06D
:10A88C00FE0170960F01E081AE89EA2BD001EC93AA
:10A89C002DC0E730A0E0FA0749F5283028F4EE89FE
:10A8AC00AC85EA2BEC8708C0FE013D960F01E081D8
:10A8BC00AE89EA2BD001EC93243018F4FE013D96BE
:10A8CC0002C0FE013E960F01E081AD89EA2BD0015A
:10A8DC00EC93283018F4FE013F9602C0FE017096EE
:10A8EC000F01E081AE89EA2BD001EC93C8C0E02FB8
:10A8FC00F0E0E130A0E0FA0781F4283028F4EE898A
:10A90C00AC85EA2BEC8708C0FE013D960F01E08177
:10A91C00AE89EA2BD001EC93B2C0E230A0E0FA078A
:10A92C0071F4283018F4FE013E9602C0FE013F96E9
:10A93C000F01E081AE89EA2BD001EC93A0C0E3308B
:10A94C00A0E0FA0771F4283018F4FE01709602C0EA
:10A95C00FE0171960F01E081AE89EA2BD001EC93D8
:10A96C008EC0E430A0E0FA07E9F4283028F4EE8930
:10A97C00AC85EA2BEC8708C0FE013D960F01E08107
:10A98C00AE89EA2BD001EC93283018F4FE013E96E8
:10A99C0002C0FE013F960F01E081AE89EA2BD00187
:10A9AC00EC936DC0E530A0E0FA07D9F4283018F428
:10A9BC00FE013E9602C0FE013F960F01E081AE897A
:10A9CC00EA2BD001EC93283018F4FE01709602C0EB
:10A9DC00FE0171960F01E081AE89EA2BD001EC9358
:10A9EC004EC0E630A0E0FA07E9F4283028F4EE89EE
:10A9FC00AC85EA2BEC8708C0FE013D960F01E08187
:10AA0C00AE89EA2BD001EC93283018F4FE01709635
:10AA1C0002C0FE0171960F01E081AE89EA2BD001D4
:10AA2C00EC932DC0E730A0E0FA0749F5283028F464
:10AA3C00EE89AC85EA2BEC8708C0FE013D960F0130
:10AA4C00E081AE89EA2BD001EC93283018F4FE019A
:10AA5C003E9602C0FE013F960F01E081AE89EA2BC3
:10AA6C00D001EC93283018F4FE01709602C0FE0160
:10AA7C0071960F01E081AE89EA2BD001EC93EE893F
:10AA8C00EE0FEE8BED89EE0FED8BEE89E03011F4CD
:10AA9C00E1E0EE8BED89E03011F4E1E0ED8B2F5F1E
:10AAAC0077C8ACEBB7E0E42FF0E0BD01A9E1B0E072
:10AABC000E9416E5E60FF71F3B96FA93EA93FE0108
:10AACC003E96FA93EA93A6E0B0E00E9435DDE030C2
:10AADC0029F1ACEBB7E0E42FF0E0BD01A9E1B0E067
:10AAEC000E9416E5E60FF71F3B96FA93EA93FE01D8
:10AAFC003E96FA93EA93A6E0B0E00E944EDDACEBF2
:10AB0C00B7E0E42FF0E0BD01A9E1B0E00E9416E54A
:10AB1C00DB01AE0FBF1F5796E0E0EC93ACEBB7E058
:10AB2C00E42FF0E0BD01A9E1B0E00E9416E5E60FCC
:10AB3C00F71F7196FA93EA93FE013896FA93EA930B
:10AB4C00A6E0B0E00E9435DDE03029F1ACEBB7E0D7
:10AB5C00E42FF0E0BD01A9E1B0E00E9416E5E60F9C
:10AB6C00F71F7196FA93EA93FE013896FA93EA93DB
:10AB7C00A6E0B0E00E944EDDACEBB7E0E42FF0E0D5
:10AB8C00BD01A9E1B0E00E9416E5DB01AE0FBF1FCD
:10AB9C005896E0E0EC93ACEBB7E0E42FF0E0BD01AD
:10ABAC00A9E1B0E00E9416E5DB01AE0FBF1F1496C1
:10ABBC00AC91A13088F0ACEBB7E0E42FF0E0BD0134
:10ABCC00A9E1B0E00E9416E5DB01AE0FBF1F1496A1
:10ABDC00EC91E150EC9330C1ACEBB7E0E42FF0E03A
:10ABEC00BD01A9E1B0E00E9416E5DB01AE0FBF1F6D
:10ABFC005796AC91A13080F0ACEBB7E0E42FF0E0CD
:10AC0C00BD01A9E1B0E00E9416E5DB01AE0FBF1F4C
:10AC1C005896AC91A13008F40FC1ACEBB7E0E42F1F
:10AC2C00F0E0BD01A9E1B0E00E9416E5DB01AE0F3A
:10AC3C00BF1F1496E4E6EC93AAE7B8E0E42FF0E02B
:10AC4C00BD01A1E7B0E00E9416E5DB01AE0FBF1F0E
:10AC5C0017960E9430E6AE2F0E94EE3EE03081F156
:10AC6C00AAE7B8E0E42FF0E0BD01A1E7B0E00E9454
:10AC7C0016E5DB01AE0FBF1F18960E9430E6EC8B79
:10AC8C00AAE7B8E0E42FF0E0BD01A1E7B0E00E9434
:10AC9C0016E5DB01AE0FBF1F1A960E9430E6E29557
:10ACAC00EF70EB8BAAE7B8E0E42FF0E0BD01A1E771
:10ACBC00B0E00E9416E5DB01AE0FBF1F199671C004
:10ACCC00AAE7B8E0E42FF0E0BD01A1E7B0E00E94F4
:10ACDC0016E5DB01AE0FBF1F14960E9430E6AE2FB7
:10ACEC000E94EE3EE03079F1AAE7B8E0E42FF0E004
:10ACFC00BD01A1E7B0E00E9416E5DB01AE0FBF1F5E
:10AD0C0015960E9430E6EC8BAAE7B8E0E42FF0E051
:10AD1C00BD01A1E7B0E00E9416E5DB01AE0FBF1F3D
:10AD2C001A960E9430E6EF70EB8BAAE7B8E0E42F9E
:10AD3C00F0E0BD01A1E7B0E00E9416E5DB01AE0F2B
:10AD4C00BF1F16962EC0AAE7B8E0E42FF0E0BD01B5
:10AD5C00A1E7B0E00E9416E5DB01AE0FBF1F129613
:10AD6C000E9430E6EC8BAAE7B8E0E42FF0E0BD01DE
:10AD7C00A1E7B0E00E9416E5DB01AE0FBF1F1196F4
:10AD8C000E9430E6EF70EB8BAAE7B8E0E42FF0E01E
:10AD9C00BD01A1E7B0E00E9416E5DB01AE0FBF1FBD
:10ADAC0013960E9430E6EA8BE88DE07FE860E88F2E
:10ADBC00EF7EE88FAAE7B8E0E42FF0E0BD01A1E751
:10ADCC00B0E00E9416E5DB01AE0FBF1F0E9430E61B
:10ADDC00F0E0F660E98FFA8FEFE2ED8FE3E0EE8FB3
:10ADEC00E0E2EF8FE1E0E8A3EA89E9A3E0E0EAA37F
:10ADFC00EBA3ECA3DE0158960E94BE09E88DE07F20
:10AE0C00E260E88FAAE7B8E0E42FF0E0BD01A1E72B
:10AE1C00B0E00E9416E5DB01AE0FBF1F0E9430E6CA
:10AE2C00F0E0F560E98FFA8FEC89ED8FEB89EE8F0E
:10AE3C00DE0158960E94BE09593010F0E6E001C0C0
:10AE4C00E3E0EF700E2EE88DE07FE029E88FEF7ED7
:10AE5C00E88FACEBB7E0E42FF0E0BD01A9E1B0E086
:10AE6C000E9416E5DB01AE0FBF1F5796AC91A130C7
:10AE7C0088F0ACEBB7E0E42FF0E0BD01A9E1B0E065
:10AE8C000E9416E5DB01AE0FBF1F5796EC91E15007
:10AE9C00EC933BC0ACEBB7E0E42FF0E0BD01A9E1D3
:10AEAC00B0E00E9416E5DB01AE0FBF1F5796EAEF2C
:10AEBC00EC93AAE7B8E0E42FF0E0BD01A1E7B0E025
:10AECC000E9416E5DB01AE0FBF1F0E9430E6F0E0DA
:10AEDC00F260E98FFA8FFE017D96FA93EA93ACEB60
:10AEEC00B7E0E42FF0E0BD01A9E1B0E00E9416E567
:10AEFC00E60FF71F3B96FA93EA93A6E0B0E00E94A8
:10AF0C004EDDDE0158960E94BE09ACEBB7E0E42F93
:10AF1C00F0E0BD01A9E1B0E00E9416E5DB01AE0F47
:10AF2C00BF1F5896AC91A13088F0ACEBB7E0E42F82
:10AF3C00F0E0BD01A9E1B0E00E9416E5DB01AE0F27
:10AF4C00BF1F5896EC91E150EC933BC0ACEBB7E0D3
:10AF5C00E42FF0E0BD01A9E1B0E00E9416E5DB01B1
:10AF6C00AE0FBF1F5896EAEFEC93AAE7B8E0E42FB8
:10AF7C00F0E0BD01A1E7B0E00E9416E5DB01AE0FE9
:10AF8C00BF1F0E9430E6F0E0F360E98FFA8FFE01FC
:10AF9C007D96FA93EA93ACEBB7E0E42FF0E0BD01B9
:10AFAC00A9E1B0E00E9416E5E60FF71F7196FA933F
:10AFBC00EA93A6E0B0E00E944EDDDE0158960E94B6
:10AFCC00BE094F5F0C94604D0E9468E4A5960895ED
:10AFDC002D970E9463E4E0916304E07409F4A8C126
:10AFEC0000E0023008F0A4C1AAE7B8E0E02FF0E0DE
:10AFFC00BD01A1E7B0E00E9416E5DB01AE0FBF1F5B
:10B00C000E9430E6E03081F4ACEBB7E0E02FF0E0EA
:10B01C00BD01A9E1B0E00E9416E5DB01AE0FBF1F38
:10B02C001296E0E0EC9382C1ACEBB7E0E02FF0E0DD
:10B03C00BD01A9E1B0E00E9416E5DB01AE0FBF1F18
:10B04C001296AC91A13008F46CC0ACEBB7E0E02FD9
:10B05C00F0E0BD01A9E1B0E00E9416E5DB01AE0F06
:10B06C00BF1F1296EC91E150EC93ACEBB7E0E02FE4
:10B07C00F0E0BD01A9E1B0E00E9416E5DB01AE0FE6
:10B08C00BF1F1196AC91A13088F0ACEBB7E0E02F6C
:10B09C00F0E0BD01A9E1B0E00E9416E5DB01AE0FC6
:10B0AC00BF1F1196EC91E150EC933AC0ACEBB7E0BA
:10B0BC00E02FF0E0BD01A9E1B0E00E9416E5DB0154
:10B0CC00AE0FBF1F1196E2E3EC93EC81E07FE860DA
:10B0DC00EC83EF7EEC83AAE7B8E0E02FF0E0BD0153
:10B0EC00A1E7B0E00E9416E5DB01AE0FBF1F0E9486
:10B0FC0030E6F0E0F660ED83FE83EBE2E987E0E01A
:10B10C00EA87E8E1EB87E5E0EC87E4EFED87E1E047
:10B11C00EE87E0E0EF87E88BDE0114960E94BE0913
:10B12C0005C1ACEBB7E0E02FF0E0BD01A9E1B0E068
:10B13C000E9416E5DB01AE0FBF1FEC91E07809F41D
:10B14C00C8C0ACEBB7E0E02FF0E0BD01A9E1B0E086
:10B15C000E9416E5DB01AE0FBF1FEC91EF773E2F7F
:10B16C00ACEBB7E0E02FF0E0BD01A9E1B0E00E944C
:10B17C0016E5DB01AE0FBF1FEC91EF77EC93EAE61F
:10B18C00F5E060E070E00E94EEE5E02FF0E0319633
:10B19C006F2F660F660B762F0E94EEE584E00E94FF
:10B1AC00E8E3289621E010E0131708F047C0AAE75F
:10B1BC00B8E0E02FF0E0BD01A1E7B0E00E9416E599
:10B1CC00DB01AE0FBF1F1E96E12FF0E00E94DDE405
:10B1DC00AE0FBF1F16960E9430E6F0E0F695E7958D
:10B1EC00E370F070309799F4ACEBB7E0E02FF0E03F
:10B1FC00BD01A9E1B0E00E9416E5E60FF71F3996F4
:10B20C000F01A081E22FE095EA23D00113C0E130B9
:10B21C00A0E0FA0781F4ACEBB7E0E02FF0E0BD0161
:10B22C00A9E1B0E00E9416E5DB01AE0FBF1F199635
:10B23C00EC91E22BEC931F5F220FB6CF21E013179A
:10B24C0008F047C0AAE7B8E0E02FF0E0BD01A1E7A5
:10B25C00B0E00E9416E5DB01AE0FBF1F1E96E12F7A
:10B26C00F0E00E94DDE4AE0FBF1F16960E9430E6A0
:10B27C00F0E0F695E795E370F070309799F4ACEB4D
:10B28C00B7E0E02FF0E0BD01A9E1B0E00E9416E5C7
:10B29C00E60FF71F3A960F01A081E22FE095EA2303
:10B2AC00D00113C0E130A0E0FA0781F4ACEBB7E0B9
:10B2BC00E02FF0E0BD01A9E1B0E00E9416E5DB0152
:10B2CC00AE0FBF1F1A96EC91E22BEC931F5F220F6F
:10B2DC00B6CFACEBB7E0E02FF0E0BD01A9E1B0E0F8
:10B2EC000E9416E5DB01AE0FBF1F1296EAE0EC934D
:10B2FC00EC81E07FE260EC83EF7EEC83E0E0ED83B9
:10B30C00EE83E1E0E987AAE7B8E0E02FF0E0BD01C9
:10B31C00A1E7B0E00E9416E5DB01AE0FBF1F0E9453
:10B32C0030E6EA87DE0114960E94BE090F5F59CE03
:10B33C000E946AE4619608950E9463E410E0133061
:10B34C0008F081C0AEEBB7E0E12FF0E0BD01ACE05E
:10B35C00B0E00E9416E5E60FF71F3196FF93EF93CE
:10B36C00AAE7B8E0E12FF0E0BD01AAE0B0E00E944E
:10B37C0016E5DB01AE0FBF1F0E9430E6AF91BF9107
:10B38C00EC93AEEBB7E0E12FF0E0BD01ACE0B0E048
:10B39C000E9416E5E60FF71F3296FF93EF93AAE78C
:10B3AC00B8E0E12FF0E0BD01AAE0B0E00E9416E5A4
:10B3BC00DB01AE0FBF1F11960E9430E6AF91BF911B
:10B3CC00EC93AEEBB7E0E12FF0E0BD01ACE0B0E008
:10B3DC000E9416E5E60FF71F3596FF93EF93AAE749
:10B3EC00B8E0E12FF0E0BD01AAE0B0E00E9416E564
:10B3FC00DB01AE0FBF1F12960E9430E6AF91BF91DA
:10B40C00EC93AEEBB7E0E12FF0E0BD01ACE0B0E0C7
:10B41C000E9416E5E60FF71F3696FF93EF93AAE707
:10B42C00B8E0E12FF0E0BD01AAE0B0E00E9416E523
:10B43C00DB01AE0FBF1F15960E9430E6AF91BF9196
:10B44C00EC931F5F7CCFE091C007E093CD07A091F8
:10B45C00C007E091CC07EA0FE093D907A091D90778
:10B46C00E091D807EA0FE093BD0710E0183108F01F
:10B47C00E1C0E0E03E2F0E2FA8E9B8E0E12FF0E0AC
:10B48C00BD01ACE0B0E00E9416E5DB01AE0FBF1FC2
:10B49C0011960E9430E6E03009F031E0A8E9B8E0FE
:10B4AC00E12FF0E0BD01ACE0B0E00E9416E5DB015D
:10B4BC00AE0FBF1F12960E9430E6E03009F03260EA
:10B4CC00A8E9B8E0E12FF0E0BD01ACE0B0E00E94EB
:10B4DC0016E5DB01AE0FBF1F15960E9430E6E0307B
:10B4EC0009F03460A8E9B8E0E12FF0E0BD01ACE070
:10B4FC00B0E00E9416E5DB01AE0FBF1F16960E944E
:10B50C0030E6E03009F03860A8E9B8E0E12FF0E06F
:10B51C00BD01ACE0B0E00E9416E5DB01AE0FBF1F31
:10B52C0019960E9430E6E03009F03061A8E9B8E0E5
:10B53C00E12FF0E0BD01ACE0B0E00E9416E5DB01CC
:10B54C00AE0FBF1F1A960E9430E6E03009F0306251
:10B55C00A8E9B8E0E12FF0E0BD01ACE0B0E00E945A
:10B56C0016E5DB01AE0FBF1F13960E9430E6E030EC
:10B57C0009F000E1A8E9B8E0E12FF0E0BD01ACE092
:10B58C00B0E00E9416E5DB01AE0FBF1F17960E94BC
:10B59C0030E6E03009F00062A8E9B8E0E12FF0E015
:10B5AC00BD01ACE0B0E00E9416E5DB01AE0FBF1FA1
:10B5BC001B960E9430E6E03009F00064A2EEB7E082
:10B5CC00E12FF0E00E94DFE4EA0FFB1F0283A2EE02
:10B5DC00B7E0E12FF0E00E94DFE4EA0FFB1F3383BA
:10B5EC00A2EEB7E0E12FF0E00E94DFE4EA0FFB1FD0
:10B5FC003296FF93EF93A8E9B8E0E12FF0E0BD019C
:10B60C00ACE0B0E00E9416E5DB01AE0FBF1F0E945C
:10B61C0030E6E295EF70E695E695E170AF91BF915B
:10B62C00E170EE0FEE0F0E2EEC91EB7FE029EC9318
:10B63C001F5F1CCF0E946AE424960895BA93AA93C4
:10B64C0025970E9461E4E091BB07F0E0E230A0E0B6
:10B65C00FA0739F4AB85BC85EC91E07109F02AC18D
:10B66C000AC0E330A0E0FA0731F4AB85BC85EC915D
:10B67C00E07109F41FC1E091BB07F0E0E230A0E0FB
:10B68C00FA0729F0E330A0E0FA0709F013C110E043
:10B69C00133008F00FC1AEEBB7E0E12FF0E0BD01C5
:10B6AC00ACE0B0E00E9416E5E60FF71F22812130D6
:10B6BC0008F4FDC0AEEBB7E0E12FF0E0BD01ACE06B
:10B6CC00B0E00E9416E5E60FF71F3181A091BB0791
:10B6DC00A23089F4E32FF0E0E058FE4F0F01AB8568
:10B6EC00BC851196ED91FC911197E015F10509F0CF
:10B6FC00DFC0E1E007C0EB85FC85E181E31709F0D1
:10B70C00D7C0E3E0EA87AEEBB7E0E12FF0E0BD0194
:10B71C00ACE0B0E00E9416E5DB01AE0FBF1FEC9170
:10B72C00E03079F4AEEBB7E0E12FF0E0BD01ACE036
:10B73C00B0E00E9416E5DB01AE0FBF1F1496EFEFD1
:10B74C00EC93AEEBB7E0E12FF0E0BD01ACE0B0E084
:10B75C000E9416E5DB01AE0FBF1FECE0EC93AEEBE5
:10B76C00B7E0E12FF0E0BD01ACE0B0E00E9416E5DF
:10B77C00E60FF71F5381E0E04E2FE8870E2F42179C
:10B78C0008F094C0A091BB07A230A1F4003069F47A
:10B79C0007E0AB85BC851596E885EF5FE887E1503F
:10B7AC00F0E0AE0FBF1FEC9103C00150E985E695A8
:10B7BC00E98714C0003069F403E0AB85BC851596AD
:10B7CC00E885EF5FE887E150F0E0AE0FBF1FEC912A
:10B7DC0004C00150E985E695E695E987A2EEB7E04D
:10B7EC00E52FF0E00E94DFE4AE0FBF1F1296EC9144
:10B7FC00E47009F43FC0A2EEB7E0E52FF0E00E9440
:10B80C00DFE4AE0FBF1F1296EC91E170EF83A2EE56
:10B81C00B7E0E52FF0E00E94DFE4AE0FBF1F1296F9
:10B82C00EC91E695E170EE83EA85A985EA23E13097
:10B83C0069F4EE81E03049F4E1E0EE83EF81E03031
:10B84C0011F0E0E001C0E1E0EF8302C0E0E0EE8344
:10B85C00A2EEB7E0E52FF0E00E94DFE4AE0FBF1FD1
:10B86C001296EE81E170EE0F0E2EEC91ED7FE02939
:10B87C00EC9309C0EA85A985EA23E13011F4E1E0F3
:10B88C0001C0E0E0EF83A2EEB7E0E52FF0E00E940C
:10B89C00DFE4AE0FBF1F1296EF81E1700E2EEC911C
:10B8AC00EE7FE029EC934F5F5F5F69CF03C002C06E
:10B8BC001F5FEECE0E9468E42D9608952D970E948E
:10B8CC0063E41A2F09893A89EC81E061EC83E07F0B
:10B8DC00E860EC83F32FE0E066277727E060F06008
:10B8EC006F6E7861DF01CB01E0915C04FF27662766
:10B8FC007727EA2BFB2B682B792BED83FE836F8349
:10B90C007887E02FEF5FE987A2EEB7E0E12FF0E058
:10B91C000E94DFE4AE0FBF1FEC91EA87A2EEB7E006
:10B92C00E12FF0E00E94DFE4AE0FBF1F1196EC9107
:10B93C00EB87C9C02D970E9461E44A2FEE81EF7E00
:10B94C00EE83E07FE860EE83EC89F0E0E050FE4FA0
:10B95C00EF83F887FE013B96FA93EA93E0E0EA93D3
:10B96C00A8E0B0E00E9460DD51E020E031E0E0E0D2
:10B97C000E2F1E2F141708F04BC030E0333008F098
:10B98C0042C0503051F4E02F0F5FF0E0DE011B9607
:10B99C00EA0FFB1F208351E020E0E32FF0E030970B
:10B9AC0069F4A2EEB7E0EB89F0E00E94DFE4AE0FA1
:10B9BC00BF1FEC91EF7009F0252B22C0E130A0E005
:10B9CC00FA0769F4A2EEB7E0EB89F0E00E94DFE43D
:10B9DC00AE0FBF1FEC91E07F09F0252B11C0E230B8
:10B9EC00A0E0FA0769F4A2EEB7E0EB89F0E00E9460
:10B9FC00DFE4AE0FBF1F1196EC91E03009F0252B60
:10BA0C00550F3F5FBBCF1F5FEB89EF5FEB8BB2CF67
:10BA1C00E02FF0E0DE011B96EA0FFB1F2083DE0116
:10BA2C0016960E94BE090E9468E4659608952D97AB
:10BA3C000E9463E41A2F09893A89FE013996FA9318
:10BA4C00EA93E0E0EA93A0E0B0E00E9460DDEC81D4
:10BA5C00EF7EEC83E07FE860EC83E32FF0E0E050D6
:10BA6C00FD4FED83FE831987FE013B96008335C0A5
:10BA7C002D970E9463E41A2F09893A89EC81E061C1
:10BA8C00EC83E07FE860EC83F32FE0E06627772718
:10BA9C00E060F060606D7861DF01CB01E0915C04E7
:10BAAC00FF2766277727EA2BFB2B682B792BED8357
:10BABC00FE836F837887E0E0E987FE013A96008386
:10BACC00FE013B961083FE013C96FA93EA93EFEF4E
:10BADC00EA93A5E0B0E00E9460DDDE0114960E94BE
:10BAEC00BE090E946AE46396089562970E9461E41D
:10BAFC00E0916304E07409F47BC4A091BC07A4300A
:10BB0C0038F4E091BC07EF5FE093BC07E15003C051
:10BB1C00E0E0E093BC07A091BC07A33008F068C438
:10BB2C00AEEBB7E0E091BC07F0E0BD01ACE0B0E0FB
:10BB3C000E9416E5E60FF71F5181AEEBB7E0E091DE
:10BB4C00BC07F0E0BD01ACE0B0E00E9416E5E60FEA
:10BB5C00F71F1281AEEBB7E0E091BC07F0E0BD013E
:10BB6C00ACE0B0E00E9416E5E60FF71F3381113010
:10BB7C0010F0103108F03CC4E091BB07F0E0E2306B
:10BB8C00A0E0FA0729F0E330A0E0FA0709F030C48E
:10BB9C00AEEBB7E0E091BC07F0E0BD01ACE0B0E08B
:10BBAC000E9416E5DB01AE0FBF1FAC91A13008F46B
:10BBBC0040C0AEEBB7E0E091BC07F0E0BD01ACE0FB
:10BBCC00B0E00E9416E5DB01AE0FBF1FEC91E15017
:10BBDC00EC93AEEBB7E0E091BC07F0E0BD01ACE05C
:10BBEC00B0E00E9416E5DB01AE0FBF1FEC91E03018
:10BBFC00F9F400E0232F0117D8F4A2EEB7E0E22FFE
:10BC0C00F0E00E94DFE4AE0FBF1F1296EC91EE7FC6
:10BC1C00EC93A2EEB7E0E22FF0E00E94DFE4AE0F6F
:10BC2C00BF1F1296EC91E260EC930F5F2F5FE3CF96
:10BC3C0048C0A091BB07A23009F043C0AEEBB7E0FF
:10BC4C00E091BC07F0E0BD01ACE0B0E00E9416E56D
:10BC5C00DB01AE0FBF1F1A96AC91A13088F0AEEB92
:10BC6C00B7E0E091BC07F0E0BD01ACE0B0E00E94B1
:10BC7C0016E5DB01AE0FBF1F1A96EC91E15020C008
:10BC8C00EE81E07FE260EE83EF7EEE83E0E0EF8317
:10BC9C00E887E1E0EB87E0E0EC87DE0116960E9496
:10BCAC00BE09AEEBB7E0E091BC07F0E0BD01ACE043
:10BCBC00B0E00E9416E5DB01AE0FBF1F1A96E4E15F
:10BCCC00EC93AEEBB7E0E091BC07F0E0BD01ACE06B
:10BCDC00B0E00E9416E5DB01AE0FBF1F1696AC91CB
:10BCEC000E94EE3EE03011F1AAE7B8E0E091BC070B
:10BCFC00F0E0BD01AAE0B0E00E9416E5DB01AE0F5A
:10BD0C00BF1F16960E9430E64E2FAAE7B8E0E091CE
:10BD1C00BC07F0E0BD01AAE0B0E00E9416E5DB0133
:10BD2C00AE0FBF1F17960E9430E637C0AEEBB7E0E0
:10BD3C00E091BC07F0E0BD01ACE0B0E00E9416E57C
:10BD4C00DB01AE0FBF1F1596AC910E94EE3EE030AA
:10BD5C0011F1AAE7B8E0E091BC07F0E0BD01AAE060
:10BD6C00B0E00E9416E5DB01AE0FBF1F13960E94D8
:10BD7C0030E64E2FAAE7B8E0E091BC07F0E0BD0139
:10BD8C00AAE0B0E00E9416E5DB01AE0FBF1F1496CF
:10BD9C000E9430E602C040E0E0E0EF8BAEEBB7E093
:10BDAC00E091BC07F0E0BD01ACE0B0E00E9416E50C
:10BDBC00DB01AE0FBF1F1796AC914A1799F4AEEB8F
:10BDCC00B7E0E091BC07F0E0BD01ACE0B0E00E9450
:10BDDC0016E5DB01AE0FBF1F1896AC91EF89EA1781
:10BDEC0009F447C0AEEBB7E0E091BC07F0E0BD0151
:10BDFC00ACE0B0E00E9416E5E60FF71F4783AEEB10
:10BE0C00B7E0E091BC07F0E0BD01ACE0B0E00E940F
:10BE1C0016E5E60FF71F3896AF89A083A091BB07F4
:10BE2C00A23011F55A93AEEBB7E0E091BC07F0E00D
:10BE3C00BD01ACE0B0E00E9416E5DB01AE0FBF1F08
:10BE4C001896EC91EA93AEEBB7E0E091BC07F0E00A
:10BE5C00BD01ACE0B0E00E9416E5DB01AE0FBF1FE8
:10BE6C001796AC91E4DD05C05A93E88DEA93A42FA4
:10BE7C00FFDD00E0232F011708F0E8C1A2EEB7E0C8
:10BE8C00E22FF0E00E94DFE4AE0FBF1F1296EC91A0
:10BE9C00EE8BA2EEB7E0E22FF0E00E94DFE4AE0FF3
:10BEAC00BF1F1396EC91ED8BEE89E071A1F0A8E920
:10BEBC00B8E0E22FF0E0BD01ACE0B0E00E9416E586
:10BECC00DB01AE0FBF1F13960E9430E6AE2F0E940F
:10BEDC00F56AE03009F412C0A8E9B8E0E22FF0E00E
:10BEEC00BD01ACE0B0E00E9416E5DB01AE0FBF1F58
:10BEFC000E9430E6E295E370EF5F55C0ED89E27089
:10BF0C00A1F0A8E9B8E0E22FF0E0BD01ACE0B0E0B0
:10BF1C000E9416E5DB01AE0FBF1F12960E9430E6A1
:10BF2C00AE2F0E94EE3EE03009F413C0A8E9B8E051
:10BF3C00E22FF0E0BD01ACE0B0E00E9416E5DB01C1
:10BF4C00AE0FBF1F0E9430E6E695E695E370EF5FFB
:10BF5C002AC0ED89E170A1F0A8E9B8E0E22FF0E089
:10BF6C00BD01ACE0B0E00E9416E5DB01AE0FBF1FD7
:10BF7C0011960E9430E6AE2F0E94EE3EE03009F49E
:10BF8C0011C0A8E9B8E0E22FF0E0BD01ACE0B0E0F0
:10BF9C000E9416E5DB01AE0FBF1F0E9430E6E37076
:10BFAC00EF5F01C0E0E0EC8BEE89E072A1F0A8E954
:10BFBC00B8E0E22FF0E0BD01ACE0B0E00E9416E585
:10BFCC00DB01AE0FBF1F17960E9430E6AE2F0E940A
:10BFDC00F56AE03009F411C0A8E9B8E0E22FF0E00E
:10BFEC00BD01ACE0B0E00E9416E5DB01AE0FBF1F57
:10BFFC0014960E9430E6E29551C0ED89E870A1F0EC
:10C00C00A8E9B8E0E22FF0E0BD01ACE0B0E00E949E
:10C01C0016E5DB01AE0FBF1F16960E9430E6AE2F61
:10C02C000E94EE3EE03009F412C0A8E9B8E0E22F1D
:10C03C00F0E0BD01ACE0B0E00E9416E5DB01AE0F14
:10C04C00BF1F14960E9430E6E695E69527C0ED8951
:10C05C00E470A1F0A8E9B8E0E22FF0E0BD01ACE09B
:10C06C00B0E00E9416E5DB01AE0FBF1F15960E94D3
:10C07C0030E6AE2F0E94EE3EE03009F416C0A8E97F
:10C08C00B8E0E22FF0E0BD01ACE0B0E00E9416E5B4
:10C09C00DB01AE0FBF1F14960E9430E6E370EF5F1A
:10C0AC00E295E07FAC89EA2BEC8BEE89E074A1F091
:10C0BC00A8E9B8E0E22FF0E0BD01ACE0B0E00E94EE
:10C0CC0016E5DB01AE0FBF1F1B960E9430E6AE2FAC
:10C0DC000E94F56AE03009F413C0A8E9B8E0E22F39
:10C0EC00F0E0BD01ACE0B0E00E9416E5DB01AE0F64
:10C0FC00BF1F18960E9430E6E295E370EF5F57C0C1
:10C10C00ED89E072A1F0A8E9B8E0E22FF0E0BD0102
:10C11C00ACE0B0E00E9416E5DB01AE0FBF1F1A9633
:10C12C000E9430E6AE2F0E94EE3EE03009F414C0BF
:10C13C00A8E9B8E0E22FF0E0BD01ACE0B0E00E946D
:10C14C0016E5DB01AE0FBF1F18960E9430E6E69590
:10C15C00E695E370EF5F2BC0ED89E071A1F0A8E9E3
:10C16C00B8E0E22FF0E0BD01ACE0B0E00E9416E5D3
:10C17C00DB01AE0FBF1F19960E9430E6AE2F0E9456
:10C18C00EE3EE03009F412C0A8E9B8E0E22FF0E08E
:10C19C00BD01ACE0B0E00E9416E5DB01AE0FBF1FA5
:10C1AC0018960E9430E6E370EF5F01C0E0E0EB8B85
:10C1BC00A2EEB7E0E22FF0E00E94DFE4AE0FBF1F6B
:10C1CC00AC91EC89EA1769F4A2EEB7E0E22FF0E04B
:10C1DC000E94DFE4AE0FBF1F1196AC91EB89EA17FA
:10C1EC0091F1A2EEB7E0E22FF0E00E94DFE4EA0F5B
:10C1FC00FB1FAC89A083A2EEB7E0E22FF0E00E9417
:10C20C00DFE4EA0FFB1F3196AB89A083AEEBB7E0FE
:10C21C00E091BC07F0E0BD01ACE0B0E00E9416E597
:10C22C00DB01AE0FBF1F1996E4E1EC93A091BB07A5
:10C23C00A23029F45A933A93A12F7CDB04C05A9371
:10C24C000A93A22F3BDB0F5F2F5F15CEAEEBB7E04F
:10C25C00E091BC07F0E0BD01ACE0B0E00E9416E557
:10C26C00DB01AE0FBF1F1996AC91A13088F0AEEB7D
:10C27C00B7E0E091BC07F0E0BD01ACE0B0E00E949B
:10C28C0016E5DB01AE0FBF1F1996EC91E150AFC064
:10C29C00A091BB07A230B1F5AEEBB7E0E091BC07C3
:10C2AC00F0E0BD01ACE0B0E00E9416E5DB01AE0FA2
:10C2BC00BF1F1996E9E0EC935A933A93A12F3ADBFE
:10C2CC005A93AEEBB7E0E091BC07F0E0BD01ACE0F7
:10C2DC00B0E00E9416E5DB01AE0FBF1F1896EC9183
:10C2EC00EA93AEEBB7E0E091BC07F0E0BD01ACE047
:10C2FC00B0E00E9416E5DB01AE0FBF1F1796AC91A4
:10C30C0096DB76C0AEEBB7E0E091BC07F0E0BD0188
:10C31C00ACE0B0E00E9416E5DB01AE0FBF1F199632
:10C32C00EAE0EC93AEEBB7E0E091BC07F0E0BD01C6
:10C33C00ACE0B0E00E9416E5DB01AE0FBF1F149617
:10C34C00AC91A11790F1AEEBB7E0E091BC07F0E037
:10C35C00BD01ACE0B0E00E9416E5DB01AE0FBF1FE3
:10C36C001496E0E0EC935A93AEEBB7E0E091BC0787
:10C37C00F0E0BD01ACE0B0E00E9416E5DB01AE0FD1
:10C38C00BF1F1896EC91EA93AEEBB7E0E091BC07B7
:10C39C00F0E0BD01ACE0B0E00E9416E5DB01AE0FB1
:10C3AC00BF1F1796AC9164DB23C0AEEBB7E0E091F6
:10C3BC00BC07F0E0BD01ACE0B0E00E9416E5E60F72
:10C3CC00F71F04815A930A93A02FA30F77DAAEEBD1
:10C3DC00B7E0E091BC07F0E0BD01ACE0B0E00E943A
:10C3EC0016E5DB01AE0FBF1F1496EC91EF5FEC93DB
:10C3FC000E9468E4689608950E9463E4ECEBF7E011
:10C40C00FA93EA93E0E0EA93A9E6B0E00E9460DDDB
:10C41C00AAE7B8E00E9430E6E093BD07ABE7B8E0CE
:10C42C000E9430E6E093E50710E0123008F0A2C05D
:10C43C00ACE7B8E0E12FF0E0BD01AAE0B0E00E946B
:10C44C0016E5DB01AE0FBF1F0E942CE69F01ADEB82
:10C45C00B7E0E12FF0E0BD01A8E2B0E00E9416E5E4
:10C46C00E60FF71F3496FF93EF93ACE7B8E0E12F9C
:10C47C00F0E0BD01AAE0B0E00E9416E5DB01AE0FD2
:10C48C00BF1F12960E9430E6AF91BF91EC93ADEBBB
:10C49C00B7E0E12FF0E0BD01A8E2B0E00E9416E5A4
:10C4AC00E60FF71F3596FF93EF93ACE7B8E0E12F5B
:10C4BC00F0E0BD01AAE0B0E00E9416E5DB01AE0F92
:10C4CC00BF1F16960E9430E6AF91BF91EC93ADEB77
:10C4DC00B7E0E12FF0E0BD01A8E2B0E00E9416E564
:10C4EC00E60FF71F2787308BADEBB7E0E12FF0E0BD
:10C4FC00BD01A8E2B0E00E9416E5DB01AE0FBF1F44
:10C50C001E96EC91E07FE460EC93ADEBB7E0E12F8D
:10C51C00F0E0BD01A8E2B0E00E9416E5DB01AE0F31
:10C52C00BF1F1196F9013196ED93FC93ADEBB7E07B
:10C53C00E12FF0E0BD01A8E2B0E00E9416E5DB01BE
:10C54C00AE0FBF1F5C96F9013496ED93FC93ADEBE7
:10C55C00B7E0E12FF0E0BD01A8E2B0E00E9416E5E3
:10C56C00DB01AE0FBF1F5B96EC91E07FE860EC93B4
:10C57C001F5F5BCFA0E9B8E00E9430E6E093C507EF
:10C58C00A1E9B8E00E9430E6E093C807A2E9B8E060
:10C59C000E9430E6E093ED07A3E9B8E00E9430E694
:10C5AC00E093F00710E01831A0F500E0A4E9B8E042
:10C5BC00E12FF0E00E94DFE4AE0FBF1F11960E9446
:10C5CC0030E6E03009F001E0A4E9B8E0E12FF0E05A
:10C5DC000E94DFE4AE0FBF1F12960E9430E6E030DF
:10C5EC0009F00260A4E9B8E0E12FF0E00E94DFE47A
:10C5FC00AE0FBF1F13960E9430E6E03009F00460C6
:10C60C00ADE0B8E0E12FF0E0EA0FFB1F00831F5F05
:10C61C00CACF0E946AE424960895BA93AA930E9402
:10C62C0061E410E0123008F0CDC0ADEBB7E0E12FC3
:10C63C00F0E0BD01A8E2B0E00E9416E5DB01AE0F10
:10C64C00BF1FEC91E030B1F0ADEBB7E0E12FF0E0C3
:10C65C00BD01A8E2B0E00E9416E5E60FF71F0180CD
:10C66C001280AE81BF811196ED91FC911197E0156E
:10C67C00F10509F0A5C0EE81FF810581ADEBB7E0B6
:10C68C00E12FF0E0BD01A8E2B0E00E9416E5E60F54
:10C69C00F71F2681ADEBB7E0E12FF0E0BD01A8E27A
:10C6AC00B0E00E9416E5E60FF71F5085ADEBB7E042
:10C6BC00E12FF0E0BD01A8E2B0E00E9416E5E60F24
:10C6CC00F71F37812523A02FA523EFEFE327EA23BC
:10C6DC002E27E52FE095E0232E2BADEBB7E0E12FD5
:10C6EC00F0E0BD01A8E2B0E00E9416E5E60FF71FEE
:10C6FC002683ADEBB7E0E12FF0E0BD01A8E2B0E09E
:10C70C000E9416E5E60FF71F0783EE81FF81E68195
:10C71C00EF700E2FADEBB7E0E12FF0E0BD01A8E21A
:10C72C00B0E00E9416E5E60FF71F2185ADEBB7E0F0
:10C73C00E12FF0E0BD01A8E2B0E00E9416E5E60FA3
:10C74C00F71F5385ADEBB7E0E12FF0E0BD01A8E298
:10C75C00B0E00E9416E5E60FF71F32852523A02FC7
:10C76C00A523EFEFE327EA232E27E52FE095E0231F
:10C77C002E2BADEBB7E0E12FF0E0BD01A8E2B0E06D
:10C78C000E9416E5E60FF71F2187ADEBB7E0E12F0E
:10C79C00F0E0BD01A8E2B0E00E9416E5E60FF71F3D
:10C7AC000287ADEBB7E0E12FF0E0BD01A8E2B0E00D
:10C7BC000E9416E5DB01AE0FBF1F1396EAE0EC9367
:10C7CC001F5F30CF0E9468E42896089524970E943A
:10C7DC0061E4E0916304E07409F4BCC3A091BC076C
:10C7EC00A43038F4E091BC07EF5FE093BC07E15054
:10C7FC0003C0E0E0E093BC07A091BC07A23008F0B6
:10C80C00A9C3ADEBB7E0E091BC07F0E0BD01A8E235
:10C81C00B0E00E9416E5DB01AE0FBF1FEC91E030DB
:10C82C0009F498C3ADEBB7E0E091BC07F0E0BD01B3
:10C83C00A8E2B0E00E9416E5DB01AE0FBF1F139615
:10C84C00AC91A13008F463C0ADEBB7E0E091BC074C
:10C85C00F0E0BD01A8E2B0E00E9416E5DB01AE0FEE
:10C86C00BF1F1396EC91E150EC93ADEBB7E0E09168
:10C87C00BC07F0E0BD01A8E2B0E00E9416E5DB01C8
:10C88C00AE0FBF1F1396EC91E03009F040C0ADEB3A
:10C89C00B7E0E091BC07F0E0BD01A8E2B0E00E9477
:10C8AC0016E5DB01AE0FBF1F1696E0E0EC93ADEB87
:10C8BC00B7E0E091BC07F0E0BD01A8E2B0E00E9457
:10C8CC0016E5DB01AE0FBF1F1796E0E0EC93ADEB66
:10C8DC00B7E0E091BC07F0E0BD01A8E2B0E00E9437
:10C8EC0016E5DB01AE0FBF1F1996E0E0EC93ADEB44
:10C8FC00B7E0E091BC07F0E0BD01A8E2B0E00E9417
:10C90C0016E5DB01AE0FBF1F1A96E0E0EC93E0E0FA
:10C91C002E2F3E2FE091BC07E03011F450E001C007
:10C92C005CE040E011E0103009F47DC0ADE0B8E00F
:10C93C00EE27A50FBE1F0C9102FF10C0A4E9B8E0B2
:10C94C00E52FF0E00E94DFE4AE0FBF1F13960E94AC
:10C95C0030E6AE2F0E94F56AE03009F40EC0A4E96F
:10C96C00B8E0E52FF0E00E94DFE4AE0FBF1F0E949D
:10C97C0030E6E295E370EE8343C001FF10C0A4E9FA
:10C98C00B8E0E52FF0E00E94DFE4AE0FBF1F129677
:10C99C000E9430E6AE2F0E94EE3EE03009F40FC04C
:10C9AC00A4E9B8E0E52FF0E00E94DFE4AE0FBF1F72
:10C9BC000E9430E6E695E695E370EE8321C000FF19
:10C9CC0010C0A4E9B8E0E52FF0E00E94DFE4AE0F60
:10C9DC00BF1F11960E9430E6AE2F0E94EE3EE03053
:10C9EC0009F40DC0A4E9B8E0E52FF0E00E94DFE403
:10C9FC00AE0FBF1F0E9430E6E370EE8301C010C083
:10CA0C00EE81F0E0309711F4312B0AC0E130A0E058
:10CA1C00FA0729F0E230A0E0FA0711F4312B212BB0
:10CA2C005F5F110F80CFADEBB7E0E091BC07F0E09A
:10CA3C00BD01A8E2B0E00E9416E5E60FF71FA0A129
:10CA4C003A1771F0ADEBB7E0E091BC07F0E0BD0137
:10CA5C00A8E2B0E00E9416E5E60FF71F30A341E014
:10CA6C00ADEBB7E0E091BC07F0E0BD01A8E2B0E0AF
:10CA7C000E9416E5E60FF71FA2A12A1771F0ADEB85
:10CA8C00B7E0E091BC07F0E0BD01A8E2B0E00E9485
:10CA9C0016E5E60FF71F22A341E0E0E02E2F3E2F14
:10CAAC0011E0103109F47DC0ADE0B8E0EE27A50F20
:10CABC00BE1F0C9102FF10C0A4E9B8E0E52FF0E016
:10CACC000E94DFE4AE0FBF1F13960E9430E6AE2F1C
:10CADC000E94F56AE03009F40EC0A4E9B8E0E52F35
:10CAEC00F0E00E94DFE4AE0FBF1F0E9430E6E2953B
:10CAFC00E370EE8343C001FF10C0A4E9B8E0E52F5A
:10CB0C00F0E00E94DFE4AE0FBF1F12960E9430E6E9
:10CB1C00AE2F0E94EE3EE03009F40FC0A4E9B8E05D
:10CB2C00E52FF0E00E94DFE4AE0FBF1F0E9430E65D
:10CB3C00E695E695E370EE8321C000FF10C0A4E9F2
:10CB4C00B8E0E52FF0E00E94DFE4AE0FBF1F1196B6
:10CB5C000E9430E6AE2F0E94EE3EE03009F40DC08C
:10CB6C00A4E9B8E0E52FF0E00E94DFE4AE0FBF1FB0
:10CB7C000E9430E6E370EE8301C010C0EE81F0E05D
:10CB8C00309711F4312B0AC0E130A0E0FA0729F0FC
:10CB9C00E230A0E0FA0711F4312B212B5F5F110F6B
:10CBAC0080CFADEBB7E0E091BC07F0E0BD01A8E2AF
:10CBBC00B0E00E9416E5E60FF71FA1A13A1771F03D
:10CBCC00ADEBB7E0E091BC07F0E0BD01A8E2B0E04E
:10CBDC000E9416E5E60FF71F31A341E0ADEBB7E07D
:10CBEC00E091BC07F0E0BD01A8E2B0E00E9416E5C0
:10CBFC00E60FF71FA3A12A1771F0ADEBB7E0E09198
:10CC0C00BC07F0E0BD01A8E2B0E00E9416E5E60F1B
:10CC1C00F71F23A341E0403089F4ADEBB7E0E0917E
:10CC2C00BC07F0E0BD01A8E2B0E00E9416E5DB0114
:10CC3C00AE0FBF1F1D96AC91A13008F412C0ADEB26
:10CC4C00B7E0E091BC07F0E0BD01A8E2B0E00E94C3
:10CC5C0016E5DB01AE0FBF1F1D96EC91E150EC9376
:10CC6C0020C0ADEBB7E0E091BC07F0E0BD01A8E25D
:10CC7C00B0E00E9416E5DB01AE0FBF1F1D96E0E190
:10CC8C00EC93ADEBB7E0E091BC07F0E0BD01A8E29E
:10CC9C00B0E00E9416E5DB01AE0FBF1F5B960E9451
:10CCAC00BE09ADEBB7E0E091BC07F0E0BD01A8E236
:10CCBC00B0E00E9416E5DB01AE0FBF1F1496AC91DD
:10CCCC00A03091F4ADEBB7E0E091BC07F0E0BD0112
:10CCDC00A8E2B0E00E9416E5DB01AE0FBF1F15966F
:10CCEC00AC91A03009F436C140E0E1E0E987EFE017
:10CCFC00E887EF83ADEBB7E0E091BC07F0E0BD0156
:10CD0C00A8E2B0E00E9416E5DB01AE0FBF1F15963E
:10CD1C00AC910E94EE3EE03089F1ACE7B8E0E091D6
:10CD2C00BC07F0E0BD01AAE0B0E00E9416E5DB0113
:10CD3C00AE0FBF1F17960E9430E6E987ACE7B8E04C
:10CD4C00E091BC07F0E0BD01AAE0B0E00E9416E55E
:10CD5C00DB01AE0FBF1F18960E9430E6E887ACE7E8
:10CD6C00B8E0E091BC07F0E0BD01AAE0B0E00E94A1
:10CD7C0016E5DB01AE0FBF1F199643C0ADEBB7E054
:10CD8C00E091BC07F0E0BD01A8E2B0E00E9416E51E
:10CD9C00DB01AE0FBF1F1496AC910E94EE3EE0304B
:10CDAC0099F1ACE7B8E0E091BC07F0E0BD01AAE076
:10CDBC00B0E00E9416E5DB01AE0FBF1F13960E9478
:10CDCC0030E6E987ACE7B8E0E091BC07F0E0BD01E4
:10CDDC00AAE0B0E00E9416E5DB01AE0FBF1F14966F
:10CDEC000E9430E6E887ACE7B8E0E091BC07F0E0E1
:10CDFC00BD01AAE0B0E00E9416E5DB01AE0FBF1F3B
:10CE0C0015960E9430E6EF83ADEBB7E0E091BC07DE
:10CE1C00F0E0BD01A8E2B0E00E9416E5E60FF71FB6
:10CE2C00A489E985EA1781F0ADEBB7E0E091BC0786
:10CE3C00F0E0BD01A8E2B0E00E9416E5E60FF71F96
:10CE4C007496A985A08341E0ADEBB7E0E091BC07F7
:10CE5C00F0E0BD01A8E2B0E00E9416E5E60FF71F76
:10CE6C00A589E885EA1781F0ADEBB7E0E091BC0746
:10CE7C00F0E0BD01A8E2B0E00E9416E5E60FF71F56
:10CE8C007596A885A08341E0ADEBB7E0E091BC07B7
:10CE9C00F0E0BD01A8E2B0E00E9416E5E60FF71F36
:10CEAC00A689EF81EA1781F0ADEBB7E0E091BC0702
:10CEBC00F0E0BD01A8E2B0E00E9416E5E60FF71F16
:10CECC007696AF81A08341E0403089F4ADEBB7E0BA
:10CEDC00E091BC07F0E0BD01A8E2B0E00E9416E5CD
:10CEEC00DB01AE0FBF1F1C96AC91A13008F412C031
:10CEFC00ADEBB7E0E091BC07F0E0BD01A8E2B0E01B
:10CF0C000E9416E5DB01AE0FBF1F1C96EC91E150A1
:10CF1C00EC9320C0ADEBB7E0E091BC07F0E0BD01B5
:10CF2C00A8E2B0E00E9416E5DB01AE0FBF1F1C9615
:10CF3C00E0E1EC93ADEBB7E0E091BC07F0E0BD01B4
:10CF4C00A8E2B0E00E9416E5DB01AE0FBF1F1E96F3
:10CF5C000E94BE090E9468E42A96089508951A93C7
:10CF6C001A2FAAE01A9FF001EC5CF64FA081A73BA8
:10CF7C0021F4A12F0E94DE9730C31730D0F410306B
:10CF8C0011F4139815C0113011F4769811C01230A9
:10CF9C0011F42C980DC0133011F4109809C01430F2
:10CFAC0011F4179805C0153011F4A39801C02F98EF
:10CFBC003DC01D30B0F4173011F4169811C0183064
:10CFCC0011F411980DC0193011F48E9809C01A3053
:10CFDC0011F48C9805C01B3011F42D9801C02E98BB
:10CFEC0025C0123190F41D3011F474980DC01E3010
:10CFFC0011F4759809C01F3011F4A49805C01031B4
:10D00C0011F4729801C0739811C0163170F412317A
:10D01C0011F4149809C0133111F45F9805C0143140
:10D02C0011F48D9801C0129801C01598D6C21A93AC
:10D03C001A2F1730D0F4103011F4139A15C0113088
:10D04C0011F4769A11C0123011F42C9A0DC01330D1
:10D05C0011F4109A09C0143011F4179A05C0153048
:10D06C0011F4A39A01C02F9AA7C01D30B0F4173049
:10D07C0011F4169A11C0183011F4119A0DC0193010
:10D08C0011F48E9A09C01A3011F48C9A05C01B3019
:10D09C0011F42D9A01C02E9A8FC0123190F41D30CC
:10D0AC0011F4749A0DC01E3011F4759A09C01F301A
:10D0BC0011F4A49A05C0103111F4729A01C0739A3C
:10D0CC007BC0173190F4123111F4149A0DC0133146
:10D0DC0011F45F9A09C0143111F48D9A05C0153101
:10D0EC0011F4129A01C0159A67C01F3198F51731C7
:10D0FC0021F4E0911E09E16027C0183121F4E09180
:10D10C001E09E26021C0193121F4E0911E09E4608E
:10D11C001BC01A3121F4E0911E09E86015C01B31C7
:10D12C0021F4E0911E09E0680FC01C3121F4E0915C
:10D13C001E09E06409C01D3121F4E0911E09E06272
:10D14C0003C0E0911E09E061E0931E09E8E0E09362
:10D15C00180932C01F3121F4E0911D09E06827C085
:10D16C00103221F4E0911D09E06421C0113221F448
:10D17C00E0911D09E0621BC0123221F4E0911D09FF
:10D18C00E06115C0133221F4E0911D09E1600FC07C
:10D19C00143221F4E0911D09E26009C0153221F42A
:10D1AC00E0911D09E46003C0E0911D09E860E09383
:10D1BC001D09E8E0E093170910C21A931A2F1730D3
:10D1CC00D0F4103011F4139815C0113011F4769876
:10D1DC0011C0123011F42C980DC0133011F41098AA
:10D1EC0009C0143011F4179805C0153011F4A39828
:10D1FC0001C02F98A7C01D30B0F4173011F4169849
:10D20C0011C0183011F411980DC0193011F48E980A
:10D21C0009C01A3011F48C9805C01B3011F42D98EC
:10D22C0001C02E988FC0123190F41D3011F47498F7
:10D23C000DC01E3011F4759809C01F3011F4A4985C
:10D24C0005C0103111F4729801C073987BC017316E
:10D25C0090F4123111F414980DC0133111F45F983D
:10D26C0009C0143111F48D9805C0153111F41298C0
:10D27C0001C0159867C01F3198F5173121F4E09162
:10D28C001E09EE7F27C0183121F4E0911E09ED7FB5
:10D29C0021C0193121F4E0911E09EB7F1BC01A311A
:10D2AC0021F4E0911E09E77F15C01B3121F4E091B8
:10D2BC001E09EF770FC01C3121F4E0911E09EF7BA2
:10D2CC0009C01D3121F4E0911E09EF7D03C0E091EE
:10D2DC001E09EF7EE0931E09E8E0E093180932C0C6
:10D2EC001F3121F4E0911D09EF7727C0103221F492
:10D2FC00E0911D09EF7B21C0113221F4E0911D0951
:10D30C00EF7D1BC0123221F4E0911D09EF7E15C098
:10D31C00133221F4E0911D09EE7F0FC0143221F479
:10D32C00E0911D09ED7F09C0153221F4E0911D0932
:10D33C00EB7F03C0E0911D09E77FE0931D09E8E056
:10D34C00E09317094AC11A931A2FEEE7F5E060E053
:10D35C0070E00E94EEE5E12FFF27662777270E94F9
:10D36C00EEE584E00E94E8E32896E12FF0E0E2305D
:10D37C00A0E0FA0749F4E0912209E061E093220968
:10D38C00E0912109EF7E9AC0E330A0E0FA0749F45E
:10D39C00E0912209E460E0932209E0912109EB7FFE
:10D3AC008DC0E430A0E0FA0749F4E0912209E06274
:10D3BC00E0932209E0912109EF7D80C0E530A0E0E7
:10D3CC00FA0749F4E0912209E068E0932209E09120
:10D3DC002109EF7773C0EB30A0E0FA0771F4E0910C
:10D3EC002009E160E0932009E0911F09EE7FE093B2
:10D3FC001F09E0E0E093190966C0EC30A0E0FA07E1
:10D40C0049F4E0912209E860E0932209E0912109B6
:10D41C00E77F54C0ED30A0E0FA0771F4E0912009E9
:10D42C00E460E0932009E0911F09EB7FE0931F0972
:10D43C00E0E0E093190947C0EE30A0E0FA0771F480
:10D44C00E0912009E260E0932009E0911F09ED7F53
:10D45C00E0931F09E0E0E093190935C0E031A0E04A
:10D46C00FA0771F4E0912009E061E0932009E09162
:10D47C001F09EF7EE0931F09E0E0E093190923C038
:10D48C00E131A0E0FA0771F4E0912009E860E09343
:10D49C002009E0911F09E77FE0931F09E0E0E0938A
:10D4AC00190911C0E631A0E0FA0769F4E0912209EC
:10D4BC00E064E0932209E0912109EF7BE0932109DC
:10D4CC00E0E0E0931A0989C01A931A2FEFE8F5E00F
:10D4DC0060E070E00E94EEE5E12FFF2766277727DA
:10D4EC000E94EEE584E00E94E8E32896E12FF0E04C
:10D4FC00E230A0E0FA0721F4E0912109E06168C074
:10D50C00E330A0E0FA0721F4E0912109E46060C067
:10D51C00E430A0E0FA0721F4E0912109E06258C060
:10D52C00E530A0E0FA0721F4E0912109E06850C051
:10D53C00EB30A0E0FA0749F4E0911F09E160E093B9
:10D54C001F09E0E0E093190948C0EC30A0E0FA07AD
:10D55C0021F4E0912109E8603BC0ED30A0E0FA072E
:10D56C0049F4E0911F09E460E0931F09E0E0E093C7
:10D57C00190933C0EE30A0E0FA0749F4E0911F0915
:10D58C00E260E0931F09E0E0E093190926C0E03166
:10D59C00A0E0FA0749F4E0911F09E061E0931F094C
:10D5AC00E0E0E093190919C0E131A0E0FA0749F471
:10D5BC00E0911F09E860E0931F09E0E0E09319098E
:10D5CC000CC0E631A0E0FA0741F4E0912109E064D7
:10D5DC00E0932109E0E0E0931A09199108950E9463
:10D5EC0063E43A2F3F3010F0363208F01FC0E32FBF
:10D5FC00EF501E2FAAE01A9FF001EF5CF64FE0816E
:10D60C00E47011F0E1E079C3AAE01A9FF001EF5C3D
:10D61C00F64FE081E295E7700E2F013021F00430D7
:10D62C0011F0053011F4E1E068C31BC0363210F084
:10D63C00363308F016C0E32FE6521E2FA7E1BAE0EE
:10D64C00F0E00E94DFE4AE0FBF1FEC91E295E770B3
:10D65C000E2F013021F0043011F0053011F4E1E00F
:10D66C004CC3A32F0E941C9048C30E9463E4E0911A
:10D67C002409EF7EE0932409EF7DE0932409E4E193
:10D68C00E0932809E0912409EF7BE0932409E091D1
:10D69C002509EE7FE0932509ED7FE0932509A2EDA6
:10D6AC00B9E00E9430E6E0932D09A3EDB9E00E94A9
:10D6BC0030E6E0932E09E1E3F9E0FA93EA93E0E037
:10D6CC00EA93A6EEB0E00E9460DDA4EDB9E00E9402
:10D6DC0030E6E0932F09A5EDB9E00E9430E6E09327
:10D6EC0030096E9A089A6A9A6B9A0C9A579A0D9A04
:10D6FC0010E0173108F018C1AAE01A9FF001EC5C99
:10D70C00F64FFF93EF93A5E4B1E0E12FF0E0BD01FC
:10D71C00A7E0B0E00E9416E5DB01AE0FBF1F0E9430
:10D72C0030E6AF91BF91EC93AAE01A9FF001EF5C49
:10D73C00F64FFF93EF93A5E4B1E0E12FF0E0BD01CC
:10D74C00A7E0B0E00E9416E5DB01AE0FBF1F1296FA
:10D75C000E9430E6E07121F5A5E4B1E0E12FF0E0A4
:10D76C00BD01A7E0B0E00E9416E5DB01AE0FBF1FC4
:10D77C0012960E9430E6E07299F4A5E4B1E0E12F34
:10D78C00F0E0BD01A7E0B0E00E9416E5DB01AE0FB2
:10D79C00BF1F12960E9430E6E07411F4E0E001C065
:10D7AC00E1E0AF91BF91E170EE0F0E2EEC91ED7FA9
:10D7BC00E029EC93A5E4B1E0E12FF0E0BD01A7E096
:10D7CC00B0E00E9416E5DB01AE0FBF1F15960E945C
:10D7DC0030E6E07249F0AAE01A9FF001EE5CF64FD9
:10D7EC00DF01EC91E061EC93A5E4B1E0E12FF0E016
:10D7FC00BD01A7E0B0E00E9416E5DB01AE0FBF1F34
:10D80C0015960E9430E6E07449F0AAE01A9FF001E8
:10D81C00EE5CF64FDF01EC91E062EC93A5E4B1E035
:10D82C00E12FF0E0BD01A7E0B0E00E9416E5DB01BE
:10D83C00AE0FBF1F12960E9430E6E07829F0E091FF
:10D84C002409E061E0932409A8EBB9E0E12FF0E0B2
:10D85C00F595E795AE0FBF1F0E9430E60E2F10FF17
:10D86C000DC0E02FE07F49F0AAE01A9FF001EF5CB9
:10D87C00F64FDF01EC91E068EC930CC0E02FEF70F9
:10D88C0049F0AAE01A9FF001EF5CF64FDF01EC9132
:10D89C00E068EC93AAE01A9FF001EC5CF64FA081D3
:10D8AC00A63309F03FC0E12FFF2766277727EC52FC
:10D8BC00FF4F6F4F6BBF36913731A0F5AAE03A9FFF
:10D8CC00F001EE5CF64FDF01EC91E064EC93E12F9C
:10D8DC00F0E0E130A0E0FA0711F46E9823C0E330D9
:10D8EC00A0E0FA0711F408981DC0E031A0E0FA0797
:10D8FC0011F46A9817C0E131A0E0FA0711F46B98A3
:10D90C0011C0E231A0E0FA0711F40C980BC0E3311E
:10D91C00A0E0FA0711F4579805C0E631A0E0FA0729
:10D92C0009F40D981F5FE5CEE7E1FAE0FA93EA936C
:10D93C00E0E0EA93A0E4B0E00E9460DD10E010317A
:10D94C0008F097C0E12FA7E1BAE0F0E00E94DFE415
:10D95C00EA0FFB1F32960F01A6EEB1E0E12FF0E0CB
:10D96C00EE0FFF1FAE0FBF1F0E9430E6D001EC93ED
:10D97C00E12FA7E1BAE0F0E00E94DFE4EA0FFB1F21
:10D98C000F01A6EEB1E0E12FF0E0EE0FFF1FAE0F9E
:10D99C00BF1F11960E9430E6E170E1F4A6EEB1E0F3
:10D9AC00E12FF0E0EE0FFF1FAE0FBF1F11960E948C
:10D9BC0030E6E27079F4A6EEB1E0E12FF0E0EE0F84
:10D9CC00FF1FAE0FBF1F11960E9430E6E47011F4DA
:10D9DC00E0E001C0E1E0D001E170EE0F0E2EEC9121
:10D9EC00ED7FE029EC93A6EEB1E0E12FF0E0EE0F35
:10D9FC00FF1FAE0FBF1F11960E9430E6E87069F052
:10DA0C00A0915E0EA33420F0E0912409E06203C0E3
:10DA1C00E0912409E061E0932409A4ECB9E0E12F42
:10DA2C00F0E0F595E795AE0FBF1F0E9430E60E2F84
:10DA3C0010FF0FC0E02FE07F59F0E12FA7E1BAE013
:10DA4C00F0E00E94DFE4AE0FBF1FEC91E068EC93B6
:10DA5C000EC0E02FEF7059F0E12FA7E1BAE0F0E033
:10DA6C000E94DFE4AE0FBF1FEC91E068EC931F5FE8
:10DA7C0066CFA2E2B9E0E0912409E295E1700E2EA6
:10DA8C00EC91EE7FE029EC93ABE1B9E0E091240955
:10DA9C00E295EF70E695E170E295E07FEE0FEE0F08
:10DAAC000E2EEC91EF7BE029EC93E0912009E07EC7
:10DABC00E0932009E091B409E07481F0A4EAB1E0AC
:10DACC000E942CE6DF01EEE00E949CE4E17029F05C
:10DADC00E0912009E061E09320090FC0A9EBB1E0CF
:10DAEC000E942CE6DF01EEE00E949CE4E17029F03C
:10DAFC00E0912009E061E0932009E091A009E07435
:10DB0C0081F0A6E9B1E00E942CE6DF01EEE00E9474
:10DB1C009CE4E17029F0E0912009E860E093200991
:10DB2C000FC0A0ECB1E00E942CE6DF01EEE00E94F9
:10DB3C009CE4E17029F0E0912009E860E093200971
:10DB4C00A4EAB1E00E942CE6DF01EEE00E949CE426
:10DB5C00E17029F0E0912009E460E0932009E09164
:10DB6C005009E07481F0AEE5B1E00E942CE6DF01D3
:10DB7C00EEE00E949CE4E17029F0E0912009E26063
:10DB8C00E09320090FC0ABEAB1E00E942CE6DF0164
:10DB9C00EEE00E949CE4E17029F0E0912009E26043
:10DBAC00E0932009A6E9B1E00E942CE6DF01EEE04B
:10DBBC000E949CE4E17029F0E0912009E160E0937F
:10DBCC002009E0911F09E07EE0931F09A0911F0935
:10DBDC00E0912009E095EF71EA2BE0931F09E0E05A
:10DBEC00E0931909E0912209E370E0932209ACE675
:10DBFC00B1E00E942CE6DF01EEE00E949CE4E170B3
:10DC0C0029F0E0912209E068E0932209E091AA0949
:10DC1C00E07481F0ADE9B1E00E942CE6DF01EEE0AA
:10DC2C000E949CE4E17029F0E0912209E064E09309
:10DC3C0022090FC0A3EEB1E00E942CE6DF01EEE05A
:10DC4C000E949CE4E17029F0E0912209E064E093E9
:10DC5C002209A5E6B1E00E942CE6DF01EEE00E946D
:10DC6C009CE4E17029F0E0912209E062E093220942
:10DC7C00E0913C09E07451F4A7E5B1E00E942CE678
:10DC8C00DF01EEE00E949CE4E17009F405C0E09134
:10DC9C002209E061E0932209ADE9B1E00E942CE693
:10DCAC00DF01EEE00E949CE4E17029F0E091220992
:10DCBC00E860E0932209AEE5B1E00E942CE6DF01BA
:10DCCC00EEE00E949CE4E17029F0E0912209E4600E
:10DCDC00E0932209E0912109E370E0932109A091DE
:10DCEC002109E0912209E095EC7FEA2BE0932109D0
:10DCFC00E0E0E0931609E0931A090E946AE4249686
:10DD0C00089527970E9461E4E0912609EF73E731AB
:10DD1C0060F1E0912209EE7FE0932209E0911B096A
:10DD2C00EF7BE0931B09E0E0E0931609E0931A09FE
:10DD3C00E0912609E07CE0932609E0912309E77045
:10DD4C00E063E0932309E0E0E2B9E5B1EF70E5B9F7
:10DD5C005F98EEB1E378EEB9E1B3EF78E1BBE4B3F1
:10DD6C00E77EE4BBA0E063D9C9C2E0912309E87F58
:10DD7C00E83008F4C3C2A3E2B9E083E0EFE10E940B
:10DD8C0022E6E0912309E87FE830D1F4A1E5B8E080
:10DD9C00E0912609EF73FF2766277727EC5FFE4F8C
:10DDAC006F4F6BBFE691F0E0EE0FFF1FAE0FBF1F82
:10DDBC00ED91FC911197E0932A09F0932B099EC2E7
:10DDCC00E0912309E87F09F099C2A1E5B8E0E09160
:10DDDC002609EF73FF2766277727EC5FFE4F6F4FFF
:10DDEC006BBFE691F0E0EE0FFF1FAE0FBF1FED9182
:10DDFC00FD91A0912A09B0912B09EA0FFB1FE0932A
:10DE0C002A09F0932B09A0912A09B0912B09E091D2
:10DE1C002B09F070EA0FFB1FE0932A09F0932B09F2
:10DE2C000E94F1E4E0932A09F0932B09E091230975
:10DE3C00F0E0E770F070E230A0E0FA07E1F5A2E361
:10DE4C00B0E0E0912609EF73F0E0BD01AAE0B0E08C
:10DE5C000E9416E5DB01AE0FBF1FE0912A09F0917D
:10DE6C002B090E9444E6E0912609EF73FF276627F1
:10DE7C007727E45EFE4F6F4F6BBFE691E03061F4A5
:10DE8C00EAEAF1E060E070E00E94D9E59F01E8ED7C
:10DE9C00F1E060E070E00BC0E6E0F2E060E070E022
:10DEAC000E94D9E59F01E4E3F2E060E070E00E949B
:10DEBC00D9E5AF0103C1E330A0E0FA07E9F5A2E32D
:10DECC00B0E0E0912609EF73F0E0BD01AAE0B0E00C
:10DEDC000E9416E5DB01AE0FBF1F1296E0912A09D6
:10DEEC00F0912B090E9444E6E0912609EF73FF277D
:10DEFC0066277727E45EFE4F6F4F6BBFE691E030ED
:10DF0C0061F4ECEAF1E060E070E00E94D9E59F0179
:10DF1C00EAEDF1E060E070E00BC0E8E0F2E060E018
:10DF2C0070E00E94D9E59F01E6E3F2E060E070E06A
:10DF3C000E94D9E5AF01C2C0E430A0E0FA07E9F5D0
:10DF4C00A2E3B0E0E0912609EF73F0E0BD01AAE096
:10DF5C00B0E00E9416E5DB01AE0FBF1F1496E091F6
:10DF6C002A09F0912B090E9444E6E0912609EF73EF
:10DF7C00FF2766277727E45EFE4F6F4F6BBFE69156
:10DF8C00E03061F4EEEAF1E060E070E00E94D9E587
:10DF9C009F01ECEDF1E060E070E00BC0EAE0F2E034
:10DFAC0060E070E00E94D9E59F01E8E3F2E060E0F8
:10DFBC0070E00E94D9E5AF0181C0E530A0E0FA071E
:10DFCC00E9F5A2E3B0E0E0912609EF73F0E0BD01C2
:10DFDC00AAE0B0E00E9416E5DB01AE0FBF1F16965B
:10DFEC00E0912A09F0912B090E9444E6E091260960
:10DFFC00EF73FF2766277727E45EFE4F6F4F6BBFEB
:10E00C00E691E03061F4E0EBF1E060E070E00E945A
:10E01C00D9E59F01EEEDF1E060E070E00BC0ECE0C3
:10E02C00F2E060E070E00E94D9E59F01EAE3F2E0E3
:10E03C0060E070E00E94D9E5AF0140C0E630A0E09E
:10E04C00FA07E1F5A2E3B0E0E0912609EF73F0E006
:10E05C00BD01AAE0B0E00E9416E5DB01AE0FBF1FC8
:10E06C001896E0912A09F0912B090E9444E6E09160
:10E07C002609EF73FF2766277727E45EFE4F6F4F65
:10E08C006BBFE691E03061F4E2EBF1E060E070E050
:10E09C000E94D9E59F01E0EEF1E060E070E00BC07A
:10E0AC00EEE0F2E060E070E00E94D9E59F01ECE365
:10E0BC00F2E060E070E00E94D9E5AF01E4EAF5E03F
:10E0CC0060E070E00E94EEE5E0912609EF73F0E06D
:10E0DC0031966F2F660F660B762F0E94EEE5E0915E
:10E0EC002A09F0912B09662777270E94EEE588E034
:10E0FC000E94E8E32C96A0912A09B0912B09A21753
:10E10C00B30718F04A175B0708F402C011E013C0FC
:10E11C0010E0E0912709EC7771F4A7E2B9E0E09107
:10E12C002609EF73EF5FEF71EE0FEE0F0E2EEC91F1
:10E13C00E378E029EC93A12F0E94CCD4E7E0EF83A5
:10E14C00E9EFE887E985E160E987E12FE170EE0FFF
:10E15C000E2EE985ED7FE029E987E0912609EF7322
:10E16C00EF5FEF73EE0FEE0F0E2EE985E370E029F3
:10E17C00E987E0912A09F0912B09EB87FC87E09164
:10E18C002309F0E0E770F070E230A0E0FA0711F438
:10E19C00E1E019C0E330A0E0FA0711F4E2E013C0AB
:10E1AC00E430A0E0FA0711F4E3E00DC0E530A0E0A4
:10E1BC00FA0711F4E4E007C0E630A0E0FA0711F426
:10E1CC00E5E001C0E0E0EA87E0E0E2B9E5B1EF703C
:10E1DC00E5B95F98EEB1E378EEB9E1B3EF78E1BB66
:10E1EC00E4B3E77EE4BBDE0116960E9483A7E091C0
:10E1FC002609EF73E63198F4A6E2B9E080E0EFE38C
:10E20C000E941EE6E0912309E770E062E093230987
:10E21C00E0912609EF73AE2F0E941D686FC0A2E239
:10E22C00B0E00E9430E61E2EE0912309E770E25028
:10E23C00A1E00E9483E4E129A2E2B0E00E944CE656
:10E24C00EFEAF5E060E070E00E94EEE580E00E940D
:10E25C00E8E32496E0912709EC7791F4EAEBF5E0FA
:10E26C0060E070E00E94EEE580E00E94E8E3249616
:10E27C00E0912309E770E23011F40E94D73914C001
:10E28C00EEEBF5E060E070E00E94EEE5E09127092E
:10E29C00E695E695EF71FF27662777270E94EEE556
:10E2AC0084E00E94E8E32896A2E2B9E0E091240918
:10E2BC00E295E1700E2EEC91EE7FE029EC93ABE150
:10E2CC00B9E0E0912409E295EF70E695E170E295F2
:10E2DC00E07FEE0FEE0F0E2EEC91EF7BE029EC932E
:10E2EC00E0E0E0931609E0931A09E0912309E87F36
:10E2FC00E160E0932309E6E0E093630E0E9468E49A
:10E30C002D9608952F970E9461E4E0912609EF73F2
:10E31C00E73260F1E0912609E07CE0932609E09178
:10E32C002309E770E062E0932309E0912209EE7F74
:10E33C00E0932209E0911B09EF7BE0931B09E0E0DD
:10E34C00E0931609E0931A09E2B9E5B1EF70E5B96B
:10E35C005F98EEB1E378EEB9E1B3EF78E1BBE4B3EB
:10E36C00E77EE4BBA0E00E941D68D0C2E0912309C7
:10E37C00E87FE83008F4CAC2E0912609EF730E2F4B
:10E38C00A3E2B9E083E0EFE10E9422E6E0912309E9
:10E39C00E87FE830D1F40731B8F4A1E5B8E0E02F1C
:10E3AC00FF2766277727EC5FFE4F6F4F6BBFE69119
:10E3BC00F0E0EE0FFF1FAE0FBF1FED91FC91119718
:10E3CC00E0932A09F0932B09A1C2E0912309E87F7D
:10E3DC0009F09CC2E7E0EF83E9EFE887E6E0EA8723
:10E3EC00E985E160E987E260E987E0912609EF734E
:10E3FC00EF5FEF73EE0FEE0F0E2EE985E370E02961
:10E40C00E987E0E0EB87EC87073108F0ABC1A1E5C9
:10E41C00B8E0E02FFF2766277727EC5FFE4F6F4FA2
:10E42C006BBFE691F0E0EE0FFF1FAE0FBF1FED913B
:10E43C00FD91A0912A09B0912B09AE0FBF1FFD01D0
:10E44C000E94F1E49F01A2E3B0E0E02FF0E0BD01F7
:10E45C00AAE0B0E00E9416E5DB01AE0FBF1F0E94E0
:10E46C002CE6AF014217530718F020E030E0E1C072
:10E47C00A2E3B0E0E02FF0E0BD01AAE0B0E00E9422
:10E48C0016E5DB01AE0FBF1F12960E942CE6EB8B3C
:10E49C00FC8BE217F30708F1241B350BF9016627F7
:10E4AC0077276E2F7F2FE0E0F0E07F936F93FF9341
:10E4BC00EF93EB89FC89E41BF50B66277727AFE814
:10E4CC00B2E080E090E00E941EE5AF91BF918F9189
:10E4DC009F910E9474E59F01ACC0A2E3B0E0E02FD5
:10E4EC00F0E0BD01AAE0B0E00E9416E5DB01AE0F42
:10E4FC00BF1F14960E942CE6E98BFA8BE217F307E8
:10E50C0030F1AB89BC892A1B3B0BD9018827992791
:10E51C00E1E10E94ADE47F936F93FF93EF93AB899E
:10E52C00BC89E989FA89EA1BFB0B66277727AFE8D8
:10E53C00B2E080E090E00E941EE5AF91BF918F9118
:10E54C009F910E9474E59F012C593F4F72C0A2E32A
:10E55C00B0E0E02FF0E0BD01AAE0B0E00E9416E5CB
:10E56C00DB01AE0FBF1F16960E942CE6EF87F88BCF
:10E57C00E217F30730F1A989BA892A1B3B0BD901A1
:10E58C0088279927E1E10E94ADE47F936F93FF9375
:10E59C00EF93A989BA89EF85F889EA1BFB0B6627EB
:10E5AC007727A4EBB1E080E090E00E941EE5AF91EC
:10E5BC00BF918F919F910E9474E59F01245D3E4F06
:10E5CC0038C0A2E3B0E0E02FF0E0BD01AAE0B0E07B
:10E5DC000E9416E5DB01AE0FBF1F18960E942CE6B9
:10E5EC00ED87FE87AF85B8892A1B3B0BD90188279D
:10E5FC009927E3E10E94ADE47F936F93FF93EF9330
:10E60C00AF85B889ED85FE85EA1BFB0BF695E79582
:10E61C0066277727ACEEB2E080E090E00E941EE522
:10E62C00AF91BF918F919F910E9474E59F01285AE1
:10E63C003D4FE3EDF5E060E070E00E94EEE5E02F89
:10E64C00F0E031966F2F660F660B762F0E94EEE589
:10E65C00F901662777270E94C9E6DF01CB01E0E0CC
:10E66C00F0E068EC72E40E94A0E70E94EEE588E01E
:10E67C000E94E8E32C96F6982B873C8710E0173124
:10E68C0008F06FC00117B1F5A5EBB8E0E12FFF273B
:10E69C0066277727E451FF4F6F4F6BBFE691F0E091
:10E6AC00AE0FBF1FEC91E07421F5E2EEF5E060E0F7
:10E6BC0070E00E94EEE5E02FF0E031966F2F660FD0
:10E6CC00660B762F0E94EEE5E12FF0E031966F2F6E
:10E6DC00660F660B762F0E94EEE588E00E94E8E359
:10E6EC002C96E0912709E260E0932709E985ED7FFC
:10E6FC00E98735C0A5EBB8E0E12FFF276627772720
:10E70C00E451FF4F6F4F6BBFE691F0E0AE0FBF1FB0
:10E71C00EC91E07421F1ECEFF5E060E070E00E9428
:10E72C00EEE5E02FF0E031966F2F660F660B762F3B
:10E73C000E94EEE5E12FF0E031966F2F660F660B2D
:10E74C00762F0E94EEE588E00E94E8E32C96E0919B
:10E75C002709E260E0932709E985ED7FE9871F5FD0
:10E76C008ECF78C0075110E0103108F073C001173C
:10E77C00C1F5A5EBB8E0E12FFF2766277727EE560A
:10E78C00FD4F6F4F6BBFE691F0E0AE0FBF1FEC91EA
:10E79C00E07831F5E2EEF5E060E070E00E94EEE545
:10E7AC00E0912609EF73F0E031966F2F660F660B40
:10E7BC00762F0E94EEE5E12FF0E077966F2F660F33
:10E7CC00660B762F0E94EEE588E00E94E8E32C961B
:10E7DC00E0912709E260E0932709E985ED7FE9875D
:10E7EC0037C0A5EBB8E0E12FFF2766277727EE5659
:10E7FC00FD4F6F4F6BBFE691F0E0AE0FBF1FEC917A
:10E80C00E07831F1ECEFF5E060E070E00E94EEE5CD
:10E81C00E0912609EF73F0E031966F2F660F660BCF
:10E82C00762F0E94EEE5E12FF0E077966F2F660FC2
:10E83C00660B762F0E94EEE588E00E94E8E32C96AA
:10E84C00E0912709E260E0932709E985ED7FE987EC
:10E85C001F5F8ACFE0912609EF730E2FA02F0E9425
:10E86C00E368DE0116960E9483A7063298F4A6E2AE
:10E87C00B9E080E0EFE30E941EE6E0912609EF7319
:10E88C00AE2F0E941D68E0912309E770E062E093CF
:10E89C0023093CC0E9E1F6E060E070E00E94EEE59F
:10E8AC0080E00E94E8E32496E0912709E695E17068
:10E8BC00A0E0EA17E1E009F0EE27AE2F0E94CCD4DD
:10E8CC00E0912309E87FE0932309A2E2B9E0E0910B
:10E8DC002409E295E1700E2EEC91EE7FE029EC9389
:10E8EC00ABE1B9E0E0912409E295EF70E695E170B7
:10E8FC00E295E07FEE0FEE0F0E2EEC91EF7BE02910
:10E90C00EC93E0E0E0931609E0931A090E9468E4A6
:10E91C006596089526970E9461E4E5E2F6E060E0D2
:10E92C0070E00E94EEE5ABE1B0E00E942CE66627B9
:10E93C0077270E94EEE584E00E94E8E32896ABE19D
:10E94C00B0E00E942CE6E03CA3E3FA0740F0ABE118
:10E95C00B0E00E942CE6E134AFE3FA0708F002C005
:10E96C0021E001C020E0A22F0E94CCD4E6E3F6E027
:10E97C0060E070E00E94EEE5ADE1B0E00E942CE6B4
:10E98C00662777270E94EEE5AFE1B0E00E942CE607
:10E99C00662777270E94EEE588E00E94E8E32C9634
:10E9AC00ADE1B0E00E942CE6E53AA7E1FA07C0F031
:10E9BC00ADE1B0E00E942CE6E73EACE1FA0780F452
:10E9CC00AFE1B0E00E942CE6E53AA7E1FA0740F08F
:10E9DC00AFE1B0E00E942CE6E73EACE1FA0708F0AC
:10E9EC0002C051E001C050E0A52F0E94CCD4EFE44E
:10E9FC00F6E060E070E00E94EEE5A2E2B0E00E947A
:10EA0C0030E6FF27662777270E94EEE584E00E9418
:10EA1C00E8E32896E0E01E2F3E2F173108F03EC1A8
:10EA2C00E4E6F6E060E070E00E94EEE5E12FF0E055
:10EA3C0031966F2F660F660B762F0E94EEE5A2E3E0
:10EA4C00B0E0E12FF0E0BD01AAE0B0E00E9416E5D5
:10EA5C00DB01AE0FBF1F0E942CE6662777270E94B2
:10EA6C00EEE5A2E3B0E0E12FF0E0BD01AAE0B0E0FA
:10EA7C000E9416E5DB01AE0FBF1F12960E942CE61A
:10EA8C00662777270E94EEE5A2E3B0E0E12FF0E0E5
:10EA9C00BD01AAE0B0E00E9416E5DB01AE0FBF1F7E
:10EAAC0014960E942CE6662777270E94EEE5A2E3D7
:10EABC00B0E0E12FF0E0BD01AAE0B0E00E9416E565
:10EACC00DB01AE0FBF1F16960E942CE66627772738
:10EADC000E94EEE5A2E3B0E0E12FF0E0BD01AAE078
:10EAEC00B0E00E9416E5DB01AE0FBF1F18960E9426
:10EAFC002CE6662777270E94EEE588E10E94E8E382
:10EB0C006C9600E0053008F0B6C0E02FF0E03097CE
:10EB1C0069F4A2E3B0E0E12FF0E0BD01AAE0B0E0BF
:10EB2C000E9416E5DB01AE0FBF1F47C0E130A0E02D
:10EB3C00FA0771F4A2E3B0E0E12FF0E0BD01AAE026
:10EB4C00B0E00E9416E5DB01AE0FBF1F129635C078
:10EB5C00E230A0E0FA0771F4A2E3B0E0E12FF0E0BC
:10EB6C00BD01AAE0B0E00E9416E5DB01AE0FBF1FAD
:10EB7C00149623C0E330A0E0FA0771F4A2E3B0E0EE
:10EB8C00E12FF0E0BD01AAE0B0E00E9416E5DB0148
:10EB9C00AE0FBF1F169611C0E430A0E0FA0789F43F
:10EBAC00A2E3B0E0E12FF0E0BD01AAE0B0E00E94EA
:10EBBC0016E5DB01AE0FBF1F18960E942CE6EE8304
:10EBCC00FF83E12FFF2766277727E45EFE4F6F4F09
:10EBDC006BBFE691E030C1F4E02FAAEAB1E080E02F
:10EBEC00FF2766277727EE0FFF1F661F771FEA0F99
:10EBFC00FB1F681F791F0E94D9E5EA87FB87E02F6E
:10EC0C00A8EDB1E080E017C0E02FA6E0B2E080E014
:10EC1C00FF2766277727EE0FFF1F661F771FEA0F68
:10EC2C00FB1F681F791F0E94D9E5EA87FB87E02F3D
:10EC3C00A4E3B2E080E0FF2766277727EE0FFF1FE3
:10EC4C00661F771FEA0FFB1F681F791F0E94D9E50B
:10EC5C00E887F987EE81FF81AA85BB85EA17FB0758
:10EC6C0038F0E885F985AE81BF81EA17FB0708F417
:10EC7C0002C00F5F47CFA02FE5E0EA17E1E009F0F3
:10EC8C00EE27AE2F0E94CCD4053010F4303009F0B2
:10EC9C0003C0E12FEF5F3E2F1F5FBFCEEFEAF5E021
:10ECAC0060E070E00E94EEE580E00E94E8E32496CC
:10ECBC00A2E2B0E00E9430E6EF3181F5203029F479
:10ECCC00EEE7F6E060E070E022C0503029F4E1E9B4
:10ECDC00F6E060E070E01BC03130A8F0EEEBF5E040
:10ECEC0060E070E00E94EEE5E0912709E695E6957C
:10ECFC00EF71FF27662777270E94EEE584E00E94DC
:10ED0C00E8E328960AC0EAEBF5E060E070E00E94C8
:10ED1C00EEE580E00E94E8E324960AC0E3EAF6E020
:10ED2C0060E070E00E94EEE580E00E94E8E324964B
:10ED3C000E9468E42C9608950E9463E40A2F3C819B
:10ED4C00373108F091C0AAE03A9FF001EF5CF64F22
:10ED5C00DF01EC91E068EC93AAE03A9FF001ED5CE6
:10ED6C00F64FDF01EC91E061EC9330FF1CC036955F
:10ED7C00A8EBB9E0EE27A30FBE1F0E9430E61E2FB2
:10ED8C00023019F4E07FE03169F01F70E02FE2955A
:10ED9C00E07F1E2BA8EBB9E0EE27A30FBE1FE12FDF
:10EDAC000E944CE618C03695A8EBB9E0EE27A30FED
:10EDBC00BE1F0E9430E61E2F023019F4EF70E130B6
:10EDCC0051F0107F102BA8EBB9E0EE27A30FBE1F5C
:10EDDC00E12F0E944CE648C00E9463E40A2F3C815C
:10EDEC00373108F041C0E32FA7E1BAE0F0E00E9410
:10EDFC00DFE4AE0FBF1FEC91E068EC9330FF1CC05A
:10EE0C003695A4ECB9E0EE27A30FBE1F0E9430E6A6
:10EE1C001E2F023019F4E07FE03169F01F70E02FF3
:10EE2C00E295E07F1E2BA4ECB9E0EE27A30FBE1FEA
:10EE3C00E12F0E944CE618C03695A4ECB9E0EE2701
:10EE4C00A30FBE1F0E9430E61E2F023019F4EF7084
:10EE5C00E13051F0107F102BA4ECB9E0EE27A30F9A
:10EE6C00BE1FE12F0E944CE60E946AE4259608958D
:10EE7C001A930A930A2FE6EBF6E060E070E00E942A
:10EE8C00EEE5E02FFF27662777270E94EEE584E06A
:10EE9C000E94E8E32896073108F047C0AAE00A9FD1
:10EEAC00F001EF5CF64FDF01EC91EF77EC93AAE009
:10EEBC000A9FF001ED5CF64FDF01EC91E07FEC93E3
:10EECC0000FF02C01FE001C010EFA8EBB9E0E02F7B
:10EEDC00F0E0F595E795AE0FBF1F0E9430E6E123F9
:10EEEC000E944CE6AAE00A9FF001EF5CF64FE0812D
:10EEFC00E17089F00A9FF001EF5CF64FE081E0775A
:10EF0C00E03440F00A9FF001EF5CF64FDF01EC912A
:10EF1C00EF78EC9309C0AAE00A9FF001EF5CF64F82
:10EF2C00DF01EC91EF78EC9359C00751003108F0F8
:10EF3C0055C0E02FA7E1BAE0F0E00E94DFE4AE0F8D
:10EF4C00BF1FEC91EF77EC93E02FA7E1BAE0F0E074
:10EF5C000E94DFE4AE0FBF1F1196EC91EF70EC93A3
:10EF6C0000FF02C01FE001C010EFA4ECB9E0E02FDD
:10EF7C00F0E0F595E795AE0FBF1F0E9430E6E12358
:10EF8C000E944CE6E02FA7E1BAE0F0E00E94DFE43B
:10EF9C00AE0FBF1FEC91E170C1F0E02FA7E1BAE01A
:10EFAC00F0E00E94DFE4AE0FBF1FEC91E077E0349D
:10EFBC0058F0E02FA7E1BAE0F0E00E94DFE4AE0FDA
:10EFCC00BF1FEC91EF78EC9309C0AAE00A9FF00107
:10EFDC00EF5CF64FDF01EC91EF78EC93099119910E
:10EFEC0008950E9461E4E0912309E770E23008F093
:10EFFC00FBC3A7E2B1E00E9430E6E03079F0A7E273
:10F00C00B1E00E9430E6AE2F0E94EE3EA5E2B9E0E0
:10F01C00E1700E2EEC91EE7FE029EC93A8E2B1E0CA
:10F02C000E9430E6E03081F0A8E2B1E00E9430E6C8
:10F03C00AE2F0E94EE3EA5E2B9E0E170EE0F0E2E6F
:10F04C00EC91ED7FE029EC9316E1173108F0E3C168
:10F05C00AAE01A9FF001EC5CF64F2081263309F4EC
:10F06C00D8C1AAE01A9FF001EF5CF64FE081E2955F
:10F07C00E7705E2F40E0E0912309E770E13041F446
:10F08C001A9FF001EF5CF64FE081E1703E2F73C0E8
:10F09C00273B09F4BEC1AAE01A9FF001EF5CF64FC2
:10F0AC00E081E27009F441C0A5E4B1E0E12FF0E0A9
:10F0BC00BD01A7E0B0E00E9416E5DB01AE0FBF1F5B
:10F0CC0012960E9430E6E07121F0E0912509E17082
:10F0DC0059F5A5E4B1E0E12FF0E0BD01A7E0B0E007
:10F0EC000E9416E5DB01AE0FBF1F12960E9430E6A0
:10F0FC00E07221F0E0912509E270B1F4A5E4B1E0F1
:10F10C00E12FF0E0BD01A7E0B0E00E9416E5DB01C5
:10F11C00AE0FBF1F12960E9430E6E07421F0E09112
:10F12C002409E07809F401C001C002C030E016C027
:10F13C00A22F0E94EE3E3E2FAAE01A9FF001EE5C39
:10F14C00F64FE081E07121F0E091600EE17009F47E
:10F15C0005C0303011F030E001C031E0AAE01A9F58
:10F16C00F001EF5CF64FDF01E32FE1700E2EEC9116
:10F17C00EE7FE029EC93303069F1E52FF0E0309729
:10F18C0021F0E130A0E0FA07D9F4E0912409E7700E
:10F19C00E23098F0E5ECF6E060E070E00E94EEE51D
:10F1AC00E12FF0E031966F2F660F660B762F0E94E1
:10F1BC00EEE584E00E94E8E3289641E052E009C0C5
:10F1CC00E430A0E0FA0721F0E530A0E0FA0709F4FA
:10F1DC0042E032C0503011F0513009F42DC042E001
:10F1EC0050E0AAE01A9FF001EF5CF64FDF01EC91C2
:10F1FC00EB7FEC93AAE01A9FF001E85CF64FA0E0DD
:10F20C00B0E0A083B183AAE01A9FF001EB5CF64F4B
:10F21C00A0E0A083AAE01A9FF001ED5CF64FDF019D
:10F22C00EC91E07FEC93AAE01A9FF001E65CF64FBC
:10F23C00DF01EC91EF71EC93E42FF0E0309709F4DF
:10F24C0097C0E130A0E0FA0709F06FC0A12F0E942F
:10F25C001D68AAE01A9FF001EE5CF64FDF01EC91FD
:10F26C00E068EC93AAE01A9FF001EB5CF64FA0E08B
:10F27C00A083AAE01A9FF001ED5CF64FDF01EC9140
:10F28C00E07FEC93AAE01A9FF001E65CF64FDF01F9
:10F29C00EC91E07EEC93AAE01A9FF001EE5CF64F45
:10F2AC00E081E07409F440C0E12FFF27662777273F
:10F2BC00EC52FF4F6F4F6BBF06910A9FF001EF5C52
:10F2CC00F64FDF01EC91E160EC93AAE00A9FF001AC
:10F2DC00EF5CF64FDF01EC91EF78E062EC93AAE083
:10F2EC000A9FF001EE5CF64FDF01EC91E068EC93C5
:10F2FC00AAE00A9FF001EB5CF64FA0E0A083AAE025
:10F30C000A9FF001ED5CF64FDF01EC91E07FEC938E
:10F31C00AAE00A9FF001E65CF64FDF01EC91E07E7B
:10F32C00EC93A02F0E941D6823C0E230A0E0FA07E6
:10F33C00F9F4A12F0E94B567AAE01A9FF001EE5CC8
:10F34C00F64FE081E074A1F0E12FFF2766277727C5
:10F35C00EC52FF4F6F4F6BBF06910A9FF001EF5CB1
:10F36C00F64FDF01EC91EE7FEC93A02F0E94B56776
:10F37C00E0912409E770E23050F0AAE01A9FF00106
:10F38C00EF5CF64FE081E295E7705E1709F432C04E
:10F39C00E1EDF6E060E070E00E94EEE5E12FF0E0D8
:10F3AC0031966F2F660F660B762F0E94EEE5AAE062
:10F3BC001A9FF001EF5CF64FE081E295E770FF27B2
:10F3CC00662777270E94EEE5E52FFF27662777272C
:10F3DC000E94EEE5E32FFF27662777270E94EEE5D4
:10F3EC00E42FFF27662777270E94EEE584E10E9431
:10F3FC00E8E36896AAE01A9FF001EF5CF64FDF0194
:10F40C00E52FE770E295E07F0E2EEC91EF78E02986
:10F41C00EC9311501ACE10E0103108F0E5C1E12F39
:10F42C00A7E1BAE0F0E00E94DFE4AE0FBF1F129636
:10F43C002C91E12FA7E1BAE0F0E00E94DFE4AE0FDF
:10F44C00BF1FEC91E295E7705E2F40E0E09123093D
:10F45C00E770E13061F4E12FA7E1BAE0F0E00E943F
:10F46C00DFE4AE0FBF1FEC91E1703E2F66C0A22F00
:10F47C000E94EE3E3E2FE12FA7E1BAE0F0E00E94A1
:10F48C00DFE4AE0FBF1FEC91E27009F447C0E12F2F
:10F49C00A7E1BAE0F0E00E94DFE4AE0FBF1FEC91F1
:10F4AC00E270A9F1A6EEB1E0E12FF0E0EE0FFF1F44
:10F4BC00AE0FBF1F11960E9430E6E17021F0E09173
:10F4CC002509E17019F5A6EEB1E0E12FF0E0EE0FA1
:10F4DC00FF1FAE0FBF1F11960E9430E6E27021F0A5
:10F4EC00E0912509E27091F4A6EEB1E0E12FF0E095
:10F4FC00EE0FFF1FAE0FBF1F11960E9430E6E47097
:10F50C0021F0E0912409E07809F401C001C002C0A7
:10F51C0030E004C0A22F0E94EE3E3E2FE12FA7E167
:10F52C00BAE0F0E00E94DFE4AE0FBF1FE32FE17002
:10F53C000E2EEC91EE7FE029EC93303009F446C0AE
:10F54C00E52FF0E0309721F0E130A0E0FA07E9F583
:10F55C00E0912409E770E23098F0E5ECF6E060E029
:10F56C0070E00E94EEE5E12FF0E031966F2F660F10
:10F57C00660B762F0E94EEE584E00E94E8E3289665
:10F58C0041E052E0E12FA7E1BAE0F0E00E94DFE4B5
:10F59C00AE0FBF1FEC91E37FEC93E12FA7E1BAE034
:10F5AC00F0E00E94DFE4AE0FBF1F1196EC91EF70FC
:10F5BC00EC93E12FA7E1BAE0F0E00E94DFE4AE0F9C
:10F5CC00BF1F1396EC91E07EEC931FC0503011F0EE
:10F5DC00513009F41AC042E050E0E12FA7E1BAE043
:10F5EC00F0E00E94DFE4AE0FBF1F1196EC91EF70BC
:10F5FC00EC93E12FA7E1BAE0F0E00E94DFE4AE0F5C
:10F60C00BF1F1396EC91EF71EC93E42FF0E0309761
:10F61C0009F48FC0E130A0E0FA0709F043C0E12FF4
:10F62C00FF2766277727A3E0B0E00E9416E5EE5986
:10F63C00FD4F6F4F6BBFE691E030D1F0E12FFF270C
:10F64C0066277727A3E0B0E00E9416E5EE59FD4F40
:10F65C006F4FEF5FFF4F6F4F7F4F6BBFE691A091E6
:10F66C001E09EA2BE0931E09E0E0E093180919C08B
:10F67C00E12FFF2766277727A3E0B0E00E9416E56D
:10F68C00EE59FD4F6F4FEF5FFF4F6F4F7F4F6BBFCB
:10F69C00E691A0911D09EA2BE0931D09E0E0E093AF
:10F6AC00170947C0E230A0E0FA0709F042C0E12F89
:10F6BC00FF2766277727A3E0B0E00E9416E5EE59F6
:10F6CC00FD4F6F4F6BBFE691E030D1F0E12FFF277C
:10F6DC0066277727A3E0B0E00E9416E5EE59FD4FB0
:10F6EC006F4FEE5FFF4F6F4F7F4F6BBFE691A09157
:10F6FC001E09EA23E0931E09E0E0E093180919C003
:10F70C00E12FFF2766277727A3E0B0E00E9416E5DC
:10F71C00EE59FD4F6F4FEE5FFF4F6F4F7F4F6BBF3B
:10F72C00E691A0911D09EA23E0931D09E0E0E09326
:10F73C001709E0912409E770E23068F0E12FA7E1A6
:10F74C00BAE0F0E00E94DFE4AE0FBF1FEC91E2954F
:10F75C00E7705E1709F435C0E1EDF6E060E070E0AB
:10F76C000E94EEE5E12FF0E078966F2F660F660BA6
:10F77C00762F0E94EEE5E12FA7E1BAE0F0E00E94BF
:10F78C00DFE4AE0FBF1FEC91E295E770FF27662711
:10F79C0077270E94EEE5E52FFF27662777270E9443
:10F7AC00EEE5E32FFF27662777270E94EEE5E42F8F
:10F7BC00FF27662777270E94EEE584E10E94E8E3A5
:10F7CC006896E12FA7E1BAE0F0E00E94DFE4AE0F0B
:10F7DC00BF1FE52FE770E295E07F0E2EEC91EF78DE
:10F7EC00E029EC931F5F18CE0E9468E426960895DA
:10F7FC0027970E9463E48D013B852C85E7E0ED8320
:10F80C00E9EFEE83EF81E160EF83E32FE170EE0F20
:10F81C000E2EEF81ED7FE029EF83203011F4E7E02D
:10F82C0001C0E8E0E887E22FEF73EE0FEE0F0E2E2B
:10F83C00EF81E370E029EF8309871A87DE011496C4
:10F84C000E9483A7A32F0E94CCD40E946AE42D9619
:10F85C00089563970E9461E4E0912309E770E23018
:10F86C0088F0E0912309E770E73019F40E94887161
:10F87C0002C00E94876EE4E1E09328090E9468E4CC
:10F88C0069960895E0E0F0E0E0932A09F0932B09E3
:10F89C00E0912709E170C9F1E0912709EE7FE0932F
:10F8AC002709E1EFF6E060E070E00E94EEE580E011
:10F8BC000E94E8E32496E0E0EC8BAC89A03210F5D2
:10F8CC00E6EFF6E060E070E00E94EEE5E88DFF27E1
:10F8DC00662777270E94EEE5A1E5B8E0EC8DF0E015
:10F8EC00EE0FFF1FAE0FBF1FED91FD91662777271F
:10F8FC000E94EEE588E00E94E8E32C96EC89EF5F2D
:10F90C00EC8BDBCFAAE00E94C1A6ABE1B0E00E9479
:10F91C002CE6EE87FF87A091660EB091670EE09102
:10F92C007D08F0917E080E94F1E4EA0FFB1FE09342
:10F93C00660EF093670EE091650EEF70E93038F4C7
:10F94C00A5E6BEE080E0EFE00E941EE66BC0E09111
:10F95C00650EE071D1F1E091650EEF7EE093650EDE
:10F96C00ABE1B0E0E091660EF091670E0E9444E6C8
:10F97C00E6E0E093630EEDEFF6E060E070E00E94ED
:10F98C00EEE5E091660EF091670E662777270E94F0
:10F99C00EEE584E00E94E8E32896E0E0EA93A0918B
:10F9AC00660EB091670EA03CE3E3BE0730F0A134C5
:10F9BC00EFE3BE0710F4E1E001C0E0E0EA93A091B0
:10F9CC00660EB091670E14DF22C0E091660EF091C6
:10F9DC00670E66277727EA87FB876C877D87A0EE03
:10F9EC00BEE280E090E00E941EE5EA87FB876C8710
:10F9FC007D87EE85FF85AA85BB858C859D856627D1
:10FA0C0077270E9474E5E093680EF093690EE091FD
:10FA1C00650EE07FE093650EE0E0F0E0E093660EAB
:10FA2C00F093670EE0917D08F0917E0866277727AA
:10FA3C00EA87FB876C877D87ACE2B1E080E090E0E1
:10FA4C000E941EE5EA87FB876C877D87EE85FF8524
:10FA5C00F695E795AA85BB858C859D8566277727C6
:10FA6C00EA0FFB1F681F791FEA87FB876C877D876E
:10FA7C00EE85FF85AA85BB858C859D8566277727B6
:10FA8C000E9474E5E0936A0EAAE2B1E00E9430E6AF
:10FA9C00E13008F4A1C0E0912409E07809F443C0F6
:10FAAC00A091680EB091690EE4E6F0E00E945CE56E
:10FABC000F01ACE2B1E00E9430E6D001F0E0AE17ED
:10FACC00BF0768F1ADE2B1E00E9430E6A0912909D0
:10FADC00AE1738F4E0912909EF5FE0932909E15062
:10FAEC001DC0E7E0F7E060E070E00E94EEE5E09119
:10FAFC00680EF091690E662777270E94EEE584E088
:10FB0C000E94E8E32896A9E00E94C92BE091240901
:10FB1C00EF77E0932409E0E0E093290903C0E0E0EB
:10FB2C00E093290959C0E0E0EB8BABE2B1E00E9415
:10FB3C0030E6EA3058F4AAE2B1E00E9430E6A09137
:10FB4C006A0EAE1710F4E1E0EB8B14C0A091680EB6
:10FB5C00B091690EE4E6F0E00E945CE50F01AAE2C8
:10FB6C00B1E00E9430E6D001F0E0AE17BF0710F410
:10FB7C00E1E0EB8BEB89E03061F1ABE2B1E00E94AC
:10FB8C0030E6A0912909AE1738F4E0912909EF5F0E
:10FB9C00E0932909E1501CC0E7E1F7E060E070E078
:10FBAC000E94EEE5E0916A0EFF27662777270E94F8
:10FBBC00EEE584E00E94E8E32896A8E00E94C92BB9
:10FBCC00E0912409E068E0932409E0E0E09329093E
:10FBDC0003C0E0E0E0932909A0915E0EA53420F467
:10FBEC00A0916A0EAB3520F0A0916A0EAD3330F5C2
:10FBFC00E0912809E030E9F4E8E2F7E060E070E039
:10FC0C000E94EEE5E0916A0EF0E06F2F660F660B36
:10FC1C00762F0E94C9E6DF01CB01E0E0F0E060E264
:10FC2C0071E40E94A0E70E94EEE584E00E94E8E304
:10FC3C002896EAE0E0932809F19A35C0A0912809AA
:10FC4C00A13088F1E0912809E150E0932809EF5F99
:10FC5C00E0912809E03039F5E0912409E07411F1C4
:10FC6C00E0912409EF7BE0932409E0E4F7E060E005
:10FC7C0070E00E94EEE5E0916A0EF0E06F2F660FE7
:10FC8C00660B762F0E94C9E6DF01CB01E0E0F0E0C5
:10FC9C0060E271E40E94A0E70E94EEE584E00E941D
:10FCAC00E8E32896F198A0912809E0E0EA17E1E052
:10FCBC0008F0EE27E98BA0916D0EB0916E0EE091DD
:10FCCC008508F0918608F695E795EA0FFB1FE093FF
:10FCDC006D0EF0936E0EE0916B0EEF70E73038F412
:10FCEC00ABE6BEE080E0EFE00E941EE605C1A0910D
:10FCFC006D0EB0916E0EE0EAF0E060E070E00E94F4
:10FD0C00D9E5AE17BF0720F0E0E0E0936C0EE9C038
:10FD1C00A0916D0EB0916E0EE2EDF0E060E070E03F
:10FD2C000E94D9E5AE17BF0720F4EAEFE0936C0E02
:10FD3C00D8C0E1E0EC8BEC89A0EAB0E080E0FF27D2
:10FD4C0066277727EE0FFF1F661F771FEA0FFB1F33
:10FD5C00681F791F0E94E4E5E0916D0EF0916E0E24
:10FD6C00EA17FB0720F4EC89EF5FEC8BE4CFEC890E
:10FD7C00E150EC8BAAE0EA02F001E0936C0EEC8906
:10FD8C00A0EAB0E080E0FF2766277727EE0FFF1F81
:10FD9C00661F771FEA0FFB1F681F791F0E94D9E5AA
:10FDAC00A0916D0EB0916E0EEA1BFB0BEE87FF87D8
:10FDBC00AE85BF85EAE00E943EE5EE87FF87EC89C1
:10FDCC00A0EAB0E080E0FF2766277727EE0FFF1F41
:10FDDC00661F771FEA0FFB1F681F791F0E94E4E55F
:10FDEC00EC89F0E066277727EE0FFF1F661F771F61
:10FDFC00EE55FF4F6F4F0E94D9E50E94FEE5EA1BBE
:10FE0C00FB0BAE85BF850E945CE5EE87FF87E0911A
:10FE1C006C0EAE85EA0FE0936C0EA6E3B1E00E9487
:10FE2C0030E6EE83AE81A03054F1E0916B0EE072BF
:10FE3C00A1F0E0916C0EF0E0F595E795DF01EE8115
:10FE4C00F0E0E7FDFFEF3197AE17BF072CF4E09120
:10FE5C006B0EEF7DE0936B0E12C0E0916C0EF0E038
:10FE6C00F595E795DF01EE81F0E0E7FDFFEFAE17CA
:10FE7C00BF072CF0E0916B0EE062E0936B0EA7E3F2
:10FE8C00B1E00E9430E6EE83AE81A03054F1E091F7
:10FE9C006B0EE074A1F0E0916C0EF0E0F595E79537
:10FEAC00DF01EE81F0E0E7FDFFEF3197AE17BF0702
:10FEBC002CF4E0916B0EEF7BE0936B0E12C0E09193
:10FECC006C0EF0E0F595E795DF01EE81F0E0E7FDD3
:10FEDC00FFEFAE17BF072CF0E0916B0EE064E093E0
:10FEEC006B0EE0916B0EE07FE0936B0EE0E0F0E0C8
:10FEFC00E0936D0EF0936E0EA0914F08A13008F4B4
:10FF0C0097C0E0914F08F0E0E130A0E0FA07C1F5AE
:10FF1C00E0918F08F091900866277727A8EEB3E060
:10FF2C0080E090E00E941EE57F936F93FF93EF9328
:10FF3C00ADE1B0E00E942CE6AF91BF918F919F9103
:10FF4C00662777270E9474E5E0939108F093920856
:10FF5C00A0919108B0919208139718F4E0E0F0E0AA
:10FF6C000AC0A0919108B0919208A93FE7E0BE07A2
:10FF7C0030F0E8EFF7E0E0939108F093920858C066
:10FF8C00E230A0E0FA0721F4E3E0E0934F0850C020
:10FF9C00E330A0E0FA0709F04BC0E1E0E0934F0832
:10FFAC00E0918F08F0919008F695E795EE87FF8722
:10FFBC00ADE1B0E00E9444E6E7E5F7E060E070E018
:10FFCC000E94EEE5EA89FB89662777270E94EEE519
:10FFDC0084E00E94E8E32896E3E0EA93EF85F88951
:10FFEC00E53AA7E1FA0740F0AF85B889A73EECE106
:04FFFC00BE0710F438
:020000021000EC
:0C000000E1E001C0E0E0EA93A889B989C2
:10000C00F7DBE1E0E0934F08E6E0E093630EA091AC
:10001C005008A23020F4F49B02C0F59B01C008C02C
:10002C00E0911B09E068E0931B09E0E0E0931609FE
:10003C00A0915008A13008F497C0E0915008F0E06E
:10004C00E130A0E0FA07C1F5A0915108B091520837
:10005C0088279927E8EEF3E060E070E00E941EE547
:10006C007F936F93FF93EF93AFE1B0E00E942CE688
:10007C00AF91BF918F919F91662777270E9474E56E
:10008C00E0939308F0939408A0919308B09194088E
:10009C00139718F4E0E0F0E00AC0A0919308B09137
:1000AC009408A93FE7E0BE0730F0E8EFF7E0E093F3
:1000BC009308F093940858C0E230A0E0FA0721F4BA
:1000CC00E3E0E093500850C0E330A0E0FA0709F0F9
:1000DC004BC0E1E0E0935008E0915108F0915208D8
:1000EC00F695E795EE87FF87AFE1B0E00E9444E616
:1000FC00E6E0E093630EE3E6F7E060E070E00E9478
:10010C00EEE5EA89FB89662777270E94EEE584E015
:10011C000E94E8E32896E4E0EA93EF85F889E53A53
:10012C00A7E1FA0740F0AF85B889A73EECE1BE071E
:10013C0010F4E1E001C0E0E0EA93A889B98958DB4A
:10014C00E1E0E0935008A0914F08A23020F4F49B1A
:10015C0002C0F59B01C008C0E0911B09E068E09368
:10016C001B09E0E0E0931609A6EDB9E00E9430E629
:10017C00AE2F0E94EE3EE03061F0E0912509E07474
:10018C0039F4E0912509E064E09325090E945E8C26
:10019C0005C0E0912509EF7BE0932509A0912C097E
:1001AC00A13038F0E0912C09E150E0932C09EF5F7D
:1001BC0003C0E4E0E0932C09E6E1EC8BAC89A731B9
:1001CC0008F0F8C6EC89AAE0EA9FF001EE5CF64F65
:1001DC00E081E07849F0EC89EA9FF001EE5CF64FA3
:1001EC00DF01EC91EF77E1C6EC89AAE0EA9FF00120
:1001FC00EC5CF64FE081E987E0E0EF83E88BA985C2
:10020C00A633D9F4EC89FF2766277727EC52FF4FEA
:10021C006F4F6BBFE691AAE0EA9FF001EF5CF64FDF
:10022C00E081E170EA8BEC89FF2766277727EC5297
:10023C00FF4F6F4F6BBFE6910AC0EC89AAE0EA9FB3
:10024C00F001EF5CF64FE081E170EA8BEC89AAE0FB
:10025C00EA9FF001EF5CF64FE081E295E770E887EA
:10026C00EA89E03009F443C5A1E5B8E0EC89FF2741
:10027C0066277727EC5FFE4F6F4F6BBFE691F0E080
:10028C00EE0FFF1FAE0FBF1FED91FD91F695E79599
:10029C00EE87FF87A2E3B0E0EC89F0E0BD01AAE0B5
:1002AC00B0E00E9416E5DB01AE0FBF1F0E942CE6EA
:1002BC008F01AE85BF850A171B0720F0E0E0EE87A3
:1002CC00EF87F1C0A2E3B0E0EC89F0E0BD01AAE059
:1002DC00B0E00E9416E5DB01AE0FBF1F12960E9424
:1002EC002CE69F01AE85BF852A173B0710F1EE85E2
:1002FC00FF85E01BF10BEE87FF87662777276E2FB4
:10030C007F2FE0E0F0E07F936F93FF93EF93F90181
:10031C00E01BF10B66277727AFE8B2E080E090E0B6
:10032C000E941EE5AF91BF918F919F910E9474E541
:10033C00B8C0A2E3B0E0EC89F0E0BD01AAE0B0E007
:10034C000E9416E5DB01AE0FBF1F14960E942CE62F
:10035C00AF01AE85BF854A175B0738F1EE85FF8587
:10036C00E21BF30BEE87FF87AE85BF8588279927A5
:10037C00E1E10E94ADE47F936F93FF93EF93FA0159
:10038C00E21BF30B66277727AFE8B2E080E090E042
:10039C000E941EE5AF91BF918F919F910E9474E5D1
:1003AC00EE87FF87EC59FF4F7CC0A2E3B0E0EC89ED
:1003BC00F0E0BD01AAE0B0E00E9416E5DB01AE0F53
:1003CC00BF1F16960E942CE6EF8BF88FAE85BF856B
:1003DC00EA17FB0740F1EE85FF85E41BF50BEE8772
:1003EC00FF87AE85BF8588279927E1E10E94ADE4A0
:1003FC007F936F93FF93EF93EF89F88DE41BF50BCD
:10040C0066277727A4EBB1E080E090E00E941EE520
:10041C00AF91BF918F919F910E9474E5EE87FF87FA
:10042C00E45DFE4F3EC0A2E3B0E0EC89F0E0BD011C
:10043C00AAE0B0E00E9416E5DB01AE0FBF1F1896D4
:10044C000E942CE6ED8BFE8BAF89B88DEE85FF8577
:10045C00EA1BFB0BEE87FF87AE85BF8588279927A4
:10046C00E3E10E94ADE47F936F93FF93EF93AF8929
:10047C00B88DED89FE89EA1BFB0BF695E79566278F
:10048C007727ACEEB2E080E090E00E941EE5AF91E1
:10049C00BF918F919F910E9474E5EE87FF87E85A78
:1004AC00FD4FEE87FF87A985A73BA1F0A63389F402
:1004BC00EC89FF2766277727EC52FF4F6F4F6BBFF6
:1004CC00E691AAE0EA9FF001EC5CF64FA081A73B15
:1004DC0009F06EC0A985A73B19F4EC89EB8B0AC017
:1004EC00EC89FF2766277727EC52FF4F6F4F6BBFC6
:1004FC0006900B8AA2E6BAE0EB89FF2766277727DE
:10050C00EC5CFE4F6F4F6BBFE691F0E00E94DDE4B8
:10051C00AE0FBF1F1196AC91A83C11F4E0E001C0E6
:10052C00E1E0E88BAE85BF85A130E0E4BE0720F0AA
:10053C00E0E0F0E4EE87FF87EC89AAE0EA9FF001A7
:10054C00EA5CF64FCF0160817181EC89AAE0EA9FE9
:10055C00F001EA5CF64FDF01ED91FD910E94EDE4B4
:10056C00DF01FB01EA1BFB0BDC01ED93FC93EC8937
:10057C00AAE0EA9FF001EA5CF64F0F01DF01ED9172
:10058C00FD91DF01EE85FF850E94F1E4EA0FFB1F70
:10059C00D001ED93FC93EC89AAE0EA9FF001EA5CB0
:1005AC00F64FDF01ED91FD910E94F1E4EE87FF879C
:1005BC00E0912A09F0912B09AE85BF85EA0FFB1F4C
:1005CC00E0932A09F0932B09EC89AAE0EA9FF00149
:1005DC00EE5CF64FE081E074B1F0EC89FF27662702
:1005EC007727EC52FF4F6F4F6BBFE691EA9FF001FC
:1005FC00E85CF64FDF01ED91FD91AE85BF85EA0F0A
:10060C00FB1FEE87FF87AE85BF85A73FE7E2BE07DE
:10061C0020F0E6EFF7E2EE87FF87EC89AAE0EA9F8D
:10062C00F001E85CF64FAE85BF85A083B183E09105
:10063C002409E870C9F0EFE6F7E060E070E00E9492
:10064C00EEE5E88DF0E031966F2F660F660B762F96
:10065C000E94EEE5EE89FF89662777270E94EEE57A
:10066C0088E00E94E8E32C96E885F0E0E230A0E018
:10067C00FA0709F0ADC0EC89AAE0EA9FF001ED5C45
:10068C00F64FDF01EC91EF7EEC93A989A03039F5A0
:10069C00A5EFB8E0EC89FF2766277727EC5FFE4FC4
:1006AC006F4F6BBFE691F0E0AE0FBF1FAC91A23065
:1006BC00A8F4A889A03089F4A5E9B8E0EC89FF2753
:1006CC0066277727E451FF4F6F4F6BBFE691F0E041
:1006DC00AE0FBF1FEC91E07409F401C001C04FC014
:1006EC00EC89AAE0EA9FF001ED5CF64FE081EF7037
:1006FC00E43058F4EC89EA9FF001ED5CF64FDF0131
:10070C0080E0EFE00E941EE63AC0E5E0E887E2E018
:10071C00EF83EC89EA93A3E00E94A276EC89AAE02D
:10072C00EA9FF001EE5CF64FE081EF70EA3098F44E
:10073C00EC89EA9FF001EE5CF64FDF0180E0EFE020
:10074C000E941EE6E6E6EA93ED89E15FEA93A0E0FB
:10075C00B0E00E94D22BEBE7F7E060E070E00E9483
:10076C00EEE5E88DF0E031966F2F660F660B762F75
:10077C000E94EEE584E00E94E8E3289673C2EC89BF
:10078C00AAE0EA9FF001EB5CF64FA081A53058F48B
:10079C00EC89AAE0EA9FF001EB5CF64FDF01EC91EB
:1007AC00EF5FEC9314C0EC89AAE0EA9FF001EB5CDC
:1007BC00F64FA0E0A083EC89AAE0EA9FF001ED5C83
:1007CC00F64FDF01EC91E07FEC93E3E0E8874AC25F
:1007DC00E330A0E0FA0709F045C2A989A03039F549
:1007EC00A5EFB8E0EC89FF2766277727EC5FFE4F73
:1007FC006F4F6BBFE691F0E0AE0FBF1FAC91A23014
:10080C00A8F4A889A03089F4A5E9B8E0EC89FF2701
:10081C0066277727E451FF4F6F4F6BBFE691F0E0EF
:10082C00AE0FBF1FEC91E07409F401C001C050C0C1
:10083C00EC89AAE0EA9FF001ED5CF64FE081EF70E5
:10084C00E33058F4EC89EA9FF001ED5CF64FDF01E0
:10085C0080E0EFE00E941EE63AC0E5E0E887E2E0C7
:10086C00EF83EC89EA93A3E00E94A276EC89AAE0DC
:10087C00EA9FF001EE5CF64FE081EF70EA3098F4FD
:10088C00EC89EA9FF001EE5CF64FDF0180E0EFE0CF
:10089C000E941EE6E6E6EA93ED89E15FEA93A0E0AA
:1008AC00B0E00E94D22BEAE8F7E060E070E00E9432
:1008BC00EEE5E88DF0E031966F2F660F660B762F24
:1008CC000E94EEE584E00E94E8E32896CBC114C0B8
:1008DC00EC89AAE0EA9FF001ED5CF64FE081EF7045
:1008EC00E13050F0EC89EA9FF001ED5CF64FDF014E
:1008FC0080E0EFE00E9422E6A985A63309F4B2C19C
:10090C00A5E4B1E0EC89F0E0BD01A7E0B0E00E9405
:10091C0016E5DB01AE0FBF1F14960E942CE6FF718B
:10092C00EE87FF87EC89AAE0EA9FF001EC5CF64FBA
:10093C00A081A73B79F4E0912309E770E13049F4F9
:10094C00EC89AAE0EA9FF001EF5CF64FE081E170E0
:10095C0009F401C035C0A2E6BAE0EC89FF2766278E
:10096C007727EC5CFE4F6F4F6BBFE691F0E00E9477
:10097C00DDE4AE0FBF1F1196EC91EB8BE03029F448
:10098C00EE85FF850E94EFE419C0EB89EC5EEB8BE2
:10099C00AB89A83CA8F4AE85BF8588279927F0E0E1
:1009AC006F2F660F660B762F0E941EE5DF01CB01C1
:1009BC00E8ECF0E060E070E00E9474E5EE87FF8701
:1009CC00EC89AAE0EA9FF001E85CF64FDF01ED91BB
:1009DC00FD91DF01EE85FF85AE17BF0708F48CC0D3
:1009EC00EC89AAE0EA9FF001EF5CF64FDF01EC9195
:1009FC00EB7FEC93EC89AAE0EA9FF001EF5CF64FF9
:100A0C00E081E87091F4EC89EA9FF001EF5CF64F1D
:100A1C00DF01EC91E860EC93EC89AAE0EA9FF0012D
:100A2C00EB5CF64FA0E0A08366C0EC89AAE0EA9FDD
:100A3C00F001EB5CF64FDF01EC91EF5FEC93EC898E
:100A4C00AAE0EA9FF001EB5CF64FE081EF93A5E49E
:100A5C00B1E0EC89F0E0BD01A7E0B0E00E9416E542
:100A6C00DB01AE0FBF1F16960E9430E6AF91AE179A
:100A7C0008F441C0E4E0E887E2E0EF83EC89EA9314
:100A8C00A4E00E94A276EC89AAE0EA9FF001EE5C59
:100A9C00F64FE081EF70EA30D8F4EC89EA9FF00170
:100AAC00EE5CF64FDF0180E0EFE00E941EE6E7E629
:100ABC00EA93ED89E15FEA93EE89AAE0EA9FF001FF
:100ACC00E85CF64FDF01ED91FD91DF010E94D22B26
:100ADC00E9E9F7E060E070E00E94EEE5E88DF0E017
:100AEC0031966F2F660F660B762F0E94EEE584E031
:100AFC000E94E8E32896B6C0EC89AAE0EA9FF001D0
:100B0C00EF5CF64FE081E87089F0EC89EA9FF00128
:100B1C00EF5CF64FDF01EC91E77FEC93EC89AAE0F8
:100B2C00EA9FF001EB5CF64FA0E0A083A5E4B1E0F6
:100B3C00EC89F0E0BD01A7E0B0E00E9416E5DB0116
:100B4C00AE0FBF1F11960E942CE6FF70EE87FF8739
:100B5C00AE85BF8500240A160B0608F083C0EC890D
:100B6C00AAE0EA9FF001E85CF64FDF01ED91FD9100
:100B7C00AE85BF85EA17FB0708F062C0EC89AAE0D6
:100B8C00EA9FF001EB5CF64FE081EF93A5E4B1E056
:100B9C00EC89F0E0BD01A7E0B0E00E9416E5DB01B6
:100BAC00AE0FBF1F13960E9430E6AF91AE1758F4EC
:100BBC00EC89AAE0EA9FF001EB5CF64FDF01EC91C7
:100BCC00EF5FEC933CC0EC89AAE0EA9FF001EF5C8C
:100BDC00F64FE081E47099F5EC89EA9FF001EF5C47
:100BEC00F64FDF01EC91E460EC93EC89EA93A2E020
:100BFC000E94A276EC89AAE0EA9FF001EE5CF64F27
:100C0C00E081EF70EA30D8F4EC89EA9FF001EE5CF9
:100C1C00F64FDF0180E0EFE00E941EE6E5E6EA9386
:100C2C00ED89E15FEA93EE89AAE0EA9FF001E85CC6
:100C3C00F64FDF01ED91FD91DF010E94D22B12C026
:100C4C00EC89AAE0EA9FF001EB5CF64FA0E0A083F0
:100C5C00EC89AAE0EA9FF001EF5CF64FDF01EC9122
:100C6C00EB7FEC93A0912C09A03039F4A885A4302B
:100C7C0020F0A0912D09A13008F438C0EC89AAE02D
:100C8C00EA9FF001E65CF64FE081EF71AE2FE09148
:100C9C002D09AE1750F4EC89AAE0EA9FF001E65C4E
:100CAC00F64FDF0180E0EFE11FC0A0912E09A030CC
:100CBC0081F0EC89AAE0EA9FF001E65CF64FE08156
:100CCC00E295EF70E695E770AE2FE0912E09AE1726
:100CDC0068F4E0E0E887EC89AAE0EA9FF001E65CC2
:100CEC00F64FDF0185E0E7E00E941EE6D0C0EC89FC
:100CFC00AAE0EA9FF001E85CF64FA0E0B0E0A08328
:100D0C00B183EC89AAE0EA9FF001EA5CF64FA0E01F
:100D1C00B0E0A083B183A985A63389F0A5E4B1E046
:100D2C00EC89F0E0BD01A7E0B0E00E9416E5DB0124
:100D3C00AE0FBF1F12960E9430E6E07809F4A7C0F0
:100D4C00E885F0E0309709F06CC0E989E03009F0F3
:100D5C009EC0A5EBB8E0EC89FF2766277727E45106
:100D6C00FF4F6F4F6BBFE691F0E0AE0FBF1FEC91E2
:100D7C00E07459F4EC89AAE0EA9FF001ED5CF64FBF
:100D8C00DF01EC91E07FEC934BC0EC89AAE0EA9F89
:100D9C00F001ED5CF64FE081EF70EF3058F4EC8928
:100DAC00EA9FF001ED5CF64FDF0180E0EFE00E947E
:100DBC001EE636C0E1E0E887EC89AAE0EA9FF00184
:100DCC00ED5CF64FDF01EC91E07FEC93EC89EA935C
:100DDC00A1E00E94A276EC89AAE0EA9FF001EE5C09
:100DEC00F64FE081EF70EA30D8F4EC89EA9FF0011D
:100DFC00EE5CF64FDF0180E0EFE00E941EE6E4E6D9
:100E0C00EA93ED89E15FEA93EE89AAE0EA9FF001AB
:100E1C00E85CF64FDF01ED91FD91DF010E94D22BD2
:100E2C0036C0E130A0E0FA0791F5A5EBB8E0EC890B
:100E3C00FF2766277727E451FF4F6F4F6BBFE69173
:100E4C00F0E0AE0FBF1FEC91E07409F5EC89AAE05D
:100E5C00EA9FF001ED5CF64FE081EF70EF3058F453
:100E6C00EC89EA9FF001ED5CF64FDF0180E0EFE0EA
:100E7C000E941EE60CC0E0E0E887EC89AAE0EA9F3D
:100E8C00F001ED5CF64FDF01EC91E07FEC93AF816C
:100E9C00A230B1F5AC890E94B567EC89AAE0EA9F53
:100EAC00F001EE5CF64FE081E07419F4A985A633ED
:100EBC0039F5EC89FF2766277727EC52FF4F6F4FE8
:100ECC006BBF06900B8AEB89AAE0EA9FF001EF5CFE
:100EDC00F64FDF01EC91EE7FEC93EB89AAE0EA9FF1
:100EEC00F001EF5CF64FDF01E885E770E295E07FFB
:100EFC000E2EEC91EF78E029EC93AB890E94B5674C
:100F0C00E0912409E770E23068F0EC89AAE0EA9FEE
:100F1C00F001EF5CF64FE081E295E770AE2FE885CB
:100F2C00EA1709F433C0E8EAF7E060E070E00E94E9
:100F3C00EEE5E88DF0E031966F2F660F660B762F9D
:100F4C000E94EEE5EC8DAAE0EA9FF001EF5CF64F13
:100F5C00E081E295E770FF27662777270E94EEE590
:100F6C00EC89FF27662777270E94EEE5EAA1FF2789
:100F7C00662777270E94EEE5EB8DFF2766277727FC
:100F8C000E94EEE584E10E94E8E36896EC89AAE011
:100F9C00EA9FF001EF5CF64FDF01E885E770E29520
:100FAC00E07F0E2EEC91EF78E029EC93EC89E15088
:100FBC00EC8B04C9E0E0EC8BAC89A03108F0ECC2FE
:100FCC00EC89A7E1BAE0F0E00E94DFE4AE0FBF1FAE
:100FDC00EC91E295E770E887E0E0EF83EC89A7E11C
:100FEC00BAE0F0E00E94DFE4AE0FBF1FEC91E170BD
:100FFC0009F46FC1E885F0E0E230A0E0FA0709F0EF
:10100C0098C0EC89A7E1BAE0F0E00E94DFE4AE0FF3
:10101C00BF1FEC91EC70EC3068F4EC89A7E1BAE0FE
:10102C00F0E00E94DFE4AE0FBF1F82E0E3E00E941D
:10103C001EE67EC0A989A03089F4A5EBB8E0EC8946
:10104C00FF2766277727EE56FD4F6F4F6BBFE69154
:10105C00F0E0AE0FBF1FEC91E07809F05BC0EC89BB
:10106C00A7E1BAE0F0E00E94DFE4AE0FBF1F1196DB
:10107C00EC91E07FE03470F4EC89A7E1BAE0F0E0A9
:10108C000E94DFE4AE0FBF1F119684E0EFE00E94D8
:10109C001EE63FC0E5E0E887E2E0EF83EC89EA93E7
:1010AC00A3E00E94F276EC89A7E1BAE0F0E00E949E
:1010BC00DFE4AE0FBF1F1196EC91EF70EA30B0F485
:1010CC00EC89A7E1BAE0F0E00E94DFE4AE0FBF1FAD
:1010DC00119680E0EFE00E941EE6E6E6EA93ED89C9
:1010EC00EA5DEA93A0E0B0E00E94D22BE9ECF7E0D5
:1010FC0060E070E00E94EEE5E88DF0E078966F2FEE
:10110C00660F660B762F0E94EEE584E00E94E8E302
:10111C0028960EC0EC89A7E1BAE0F0E00E94DFE46B
:10112C00AE0FBF1F1196EC91EF70EC93E3E0E887E4
:10113C0081C0E330A0E0FA0709F07CC0A989A03097
:10114C0089F4A5EBB8E0EC89FF2766277727EE56E4
:10115C00FD4F6F4F6BBFE691F0E0AE0FBF1FEC91F0
:10116C00E07809F05BC0EC89A7E1BAE0F0E00E94FE
:10117C00DFE4AE0FBF1F1196EC91E07FE03370F40B
:10118C00EC89A7E1BAE0F0E00E94DFE4AE0FBF1FEC
:10119C00119684E0EFE00E941EE63FC0E2E0EF8390
:1011AC00E4E0E887EC89EA93A4E00E94F276EC890B
:1011BC00A7E1BAE0F0E00E94DFE4AE0FBF1F11968A
:1011CC00EC91EF70EA30B0F4EC89A7E1BAE0F0E012
:1011DC000E94DFE4AE0FBF1F119680E0EFE00E948B
:1011EC001EE6E7E6EA93ED89EA5DEA93A0E0B0E05B
:1011FC000E94D22BE6EDF7E060E070E00E94EEE595
:10120C00E88DF0E078966F2F660F660B762F0E94B4
:10121C00EEE584E00E94E8E328960CC0EC89A7E197
:10122C00BAE0F0E00E94DFE4AE0FBF1F1196EC9124
:10123C00EF70EC93A0912C09A03039F4A885A43060
:10124C0020F0A0912F09A13008F442C0EC89A7E14D
:10125C00BAE0F0E00E94DFE4AE0FBF1F1396EC91F2
:10126C00EF71AE2FE0912F09AE1760F4EC89A7E176
:10127C00BAE0F0E00E94DFE4AE0FBF1F139680E0EF
:10128C00EFE124C0A0913009A03099F0EC89A7E1DE
:10129C00BAE0F0E00E94DFE4AE0FBF1F1396EC91B2
:1012AC00E295EF70E695E770AE2FE0913009AE173E
:1012BC0078F4E0E0E887EC89A7E1BAE0F0E00E947E
:1012CC00DFE4AE0FBF1F139685E0E7E00E941EE639
:1012DC00C4C0A6EEB1E0EC89F0E0EE0FFF1FAE0F3C
:1012EC00BF1F11960E9430E6E87009F4B6C0E8857D
:1012FC00F0E0309709F073C0E989E03089F4A5EB90
:10130C00B8E0EC89FF2766277727EE56FD4F6F4F25
:10131C006BBFE691F0E0AE0FBF1FEC91E07869F483
:10132C00EC89A7E1BAE0F0E00E94DFE4AE0FBF1F4A
:10133C001196EC91EF70EC9351C0EC89A7E1BAE0F7
:10134C00F0E00E94DFE4AE0FBF1F1196EC91E07F3E
:10135C00E03F70F4EC89A7E1BAE0F0E00E94DFE432
:10136C00AE0FBF1F119684E0EFE00E941EE636C060
:10137C00E1E0E887EC89A7E1BAE0F0E00E94DFE465
:10138C00AE0FBF1F1196EC91EF70EC93EC89EA93C2
:10139C00A1E00E94F276EC89A7E1BAE0F0E00E94AD
:1013AC00DFE4AE0FBF1F1196EC91EF70EA30B0F492
:1013BC00EC89A7E1BAE0F0E00E94DFE4AE0FBF1FBA
:1013CC00119680E0EFE00E941EE6E4E6EA93ED89D8
:1013DC00EA5DEA93A0E0B0E00E94D22B3EC0E1307F
:1013EC00A0E0FA07D1F5A5EBB8E0EC89FF2766275A
:1013FC007727EE56FD4F6F4F6BBFE691F0E0AE0FC7
:10140C00BF1FEC91E07849F5EC89A7E1BAE0F0E078
:10141C000E94DFE4AE0FBF1F1196EC91E07FE03F1E
:10142C0070F4EC89A7E1BAE0F0E00E94DFE4AE0FC3
:10143C00BF1F119684E0EFE00E941EE60EC0E0E0B4
:10144C00E887EC89A7E1BAE0F0E00E94DFE4AE0F98
:10145C00BF1F1196EC91EF70EC93AF81A23009F0A5
:10146C0042C0EC89FF2766277727A3E0B0E00E94F3
:10147C0016E5EE59FD4F6F4F6BBFE691E030D1F0A2
:10148C00EC89FF2766277727A3E0B0E00E9416E5DA
:10149C00EE59FD4F6F4FEE5FFF4F6F4F7F4F6BBF9E
:1014AC00E691A0911E09EA23E0931E09E0E0E09387
:1014BC00180919C0EC89FF2766277727A3E0B0E04D
:1014CC000E9416E5EE59FD4F6F4FEE5FFF4F6F4FC9
:1014DC007F4F6BBFE691A0911D09EA23E0931D0994
:1014EC00E0E0E0931709E0912409E770E23078F02E
:1014FC00EC89A7E1BAE0F0E00E94DFE4AE0FBF1F79
:10150C00EC91E295E770AE2FE885EA1709F42FC04D
:10151C00E5EEF7E060E070E00E94EEE5E88DF0E0CB
:10152C0078966F2F660F660B762F0E94EEE5EC8D8A
:10153C00A7E1BAE0F0E00E94DFE4AE0FBF1FEC9130
:10154C00E295E770FF27662777270E94EEE5EC8986
:10155C00FF27662777270E94EEE5EF89FF2766278E
:10156C0077270E94EEE580E10E94E8E36496EC891F
:10157C00A7E1BAE0F0E00E94DFE4AE0FBF1FE88500
:10158C00E770E295E07F0E2EEC91EF78E029EC937A
:10159C00EC89EF5FEC8B10CDE091CA08E07421F47C
:1015AC00A0912809A03009F018C0E0912609E07438
:1015BC0031F4E0912609E064E09326090DC0E09136
:1015CC002009E07449F0E0912009EF7BE0932009B9
:1015DC00E0E0E09319096CD105C0E0912609E064C4
:1015EC00E0932609E0912409E87009F4B2C0EDEF0C
:1015FC00F7E060E070E00E94EEE580E00E94E8E336
:10160C002496E0E0EC8BAC89A73108F060C0EC8943
:10161C00AAE0EA9FF001EF5CF64FE081E17009F47B
:10162C0052C0E7E0F8E060E070E00E94EEE5E88D83
:10163C00F0E031966F2F660F660B762F0E94EEE569
:10164C00A5EBB8E0EC8DFF2766277727E451FF4F19
:10165C006F4F6BBFE691F0E0AE0FBF1FEC91E074E3
:10166C0011F0E1E001C0E0E00E94F6E40E94EEE53A
:10167C00A1E5B8E0E8A1FF2766277727EC5FFE4FCE
:10168C006F4F6BBFE691F0E0EE0FFF1FAE0FBF1F69
:10169C00ED91FD91662777270E94EEE5ECA1AAE07B
:1016AC00EA9FF001E85CF64FDF01ED91FD91AAE0B5
:1016BC00B0E00E9416E5662777270E94EEE580E1F0
:1016CC000E94E8E36496EC89EF5FEC8B9CCFAC89CD
:1016DC00A732D0F5EC89A7E1BAE0F0E00E94DFE494
:1016EC00AE0FBF1FEC91E17059F1E1E2F8E060E060
:1016FC0070E00E94EEE5E88DF0E078966F2F660FB3
:10170C00660B762F0E94EEE5A5EBB8E0EC8DFF277B
:10171C0066277727EE56FD4F6F4F6BBFE691F0E0D3
:10172C00AE0FBF1FEC91E07811F0E1E001C0E0E0FA
:10173C000E94F6E40E94EEE588E00E94E8E32C9615
:10174C00EC89EF5FEC8BC3CFE0912409E77FE0934A
:10175C0024090C943E910E9461E4E0E05E2F2E2F50
:10176C003E2F0E2F10E01C3040F5A8EBB9E0EE2711
:10177C00A10FBE1F0E9430E6E03009F021E0AAE084
:10178C001A9FF001EF5CF64FE081F0E00E94EDE46F
:10179C00E770F070E130A0E0FA0711F451E00BC0F3
:1017AC00E430A0E0FA0711F431E005C0E530A0E028
:1017BC00FA0709F401E01F5FD6CF10E0183040F5AE
:1017CC00A4ECB9E0EE27A10FBE1F0E9430E6E0307A
:1017DC0009F021E0AAE01A9FF001EF5CF64FE081DE
:1017EC00F0E00E94EDE4E770F070E130A0E0FA0761
:1017FC0011F451E00BC0E430A0E0FA0711F431E031
:10180C0005C0E530A0E0FA0709F401E01F5FD6CF70
:10181C00E0912009E295EF70E695E695E170E2170C
:10182C00A9F0A0E2B9E0E22FE170E295E07FEE0FC3
:10183C00EE0F0E2EEC91EF7BE029EC93E0E0E093C1
:10184C001909E0912609EF7BE0932609A5E2B9E09E
:10185C00E02FE170EE0FEE0F0E2EEC91EB7FE029F6
:10186C00EC93A5E2B9E0E32FE170EE0FEE0FEE0F73
:10187C000E2EEC91E77FE029EC93A5E2B9E0E22F84
:10188C00E170E295E07FEE0F0E2EEC91EF7DE029FA
:10189C00EC93A5E2B9E0E52FE170E295E07F0E2E26
:1018AC00EC91EF7EE029EC930E9468E42696089573
:1018BC001A93EDE2F8E060E070E00E94EEE580E063
:1018CC000E94E8E32496ACECB9E0E0E0F0E00E9482
:1018DC0044E610E0173108F050C0AAE01A9FF0015E
:1018EC00EE5CF64FDF01EC91E07FEC93AAE01A9FDF
:1018FC00F001EF5CF64FDF01EC91EF77EC93AAE08F
:10190C001A9FF001ED5CF64FDF01EC91EF7EEC934A
:10191C00AAE01A9FF001ED5CF64FDF01EC91E07F3D
:10192C00EC93AAE01A9FF001E65CF64FDF01EC9114
:10193C00EF71EC93AAE01A9FF001EF5CF64FE08197
:10194C00F0E00E94EDE4E770F070E130A0E0FA07FF
:10195C0021F0E430A0E0FA0709F404C0E530A0E07F
:10196C00FA0749F4AAE01A9FF001EF5CF64FDF0189
:10197C00EC91EF78EC931F5FADCF10E01C3048F486
:10198C00A8EBB9E0EE27A10FBE1F0E944CE61F5F2B
:10199C00F5CF10E0103108F052C0E12FA7E1BAE00A
:1019AC00F0E00E94DFE4AE0FBF1F1196EC91E07FD8
:1019BC00EC93E12FA7E1BAE0F0E00E94DFE4AE0F78
:1019CC00BF1FEC91EF77EC93E12FA7E1BAE0F0E0C9
:1019DC000E94DFE4AE0FBF1F1196EC91EF70EC93F9
:1019EC00E12FA7E1BAE0F0E00E94DFE4AE0FBF1FE9
:1019FC001396EC91EF71EC93E12FA7E1BAE0F0E0D4
:101A0C000E94DFE4AE0FBF1FEC91F0E00E94EDE40A
:101A1C00E770F070E130A0E0FA0721F0E530A0E0CB
:101A2C00FA0759F4E12FA7E1BAE0F0E00E94DFE4F5
:101A3C00AE0FBF1FEC91EF78EC931F5FABCF10E0B4
:101A4C00183048F4A4ECB9E0EE27A10FBE1F0E9499
:101A5C004CE61F5FF5CFE0912009EF7BE093200966
:101A6C00E0E0E0931909E0C20E9463E43A2F3733B7
:101A7C0010F03C3308F0BBC000E010E0173108F068
:101A8C005DC0AAE01A9FF001EC5CF64FA0813A17FA
:101A9C0009F052C0AAE01A9FF001EF5CF64FE0810A
:101AAC00F0E00E94EDE4E770F070309761F41A9F5B
:101ABC00F001EF5CF64FE081E07811F0003009F0B6
:101ACC0001C005E039C0E230A0E0FA0721F0E330B4
:101ADC00A0E0FA07B9F4AAE01A9FF001EF5CF64F08
:101AEC00E081E47011F002E00CC0AAE01A9FF00152
:101AFC00EF5CF64FE081E07811F0003009F001C0A6
:101B0C0005E01AC0E130A0E0FA0751F4AAE01A9FF0
:101B1C00F001EF5CF64FE081E07809F001E00CC0D9
:101B2C00E430A0E0FA0711F4E4E0CAC2E530A0E02A
:101B3C00FA0711F4E3E0C4C21F5FA0CF10E010312C
:101B4C0008F053C0E12FA7E1BAE0F0E00E94DFE417
:101B5C00AE0FBF1F1296AC913A1709F044C0E12F9B
:101B6C00A7E1BAE0F0E00E94DFE4AE0FBF1FEC91FA
:101B7C00F0E00E94EDE4E770F070309721F0E23075
:101B8C00A0E0FA0709F404C0E330A0E0FA0781F4FE
:101B9C00E12FA7E1BAE0F0E00E94DFE4AE0FBF1F37
:101BAC00EC91E07811F0003009F001C005E01BC0A9
:101BBC00E130A0E0FA0769F4E12FA7E1BAE0F0E028
:101BCC000E94DFE4AE0FBF1FEC91E07809F001E05A
:101BDC000AC0E430A0E0FA0721F0E530A0E0FA07F3
:101BEC0011F4E3E06DC21F5FAACFE02F69C2E32FAF
